:100000000C940D100C942A100C942A100C942A10A5
:100010000C942A100C942B120C9448140C942A1053
:100020000C942A100C942A100C940A180C942A1080
:100030000C942A100C942A100C94CE280C942A109C
:100040000C942A100C945D150C943B120C94F21134
:100050000C942A100C94E5220C942A100C942A106B
:100060000C942A100C942A100C942A100C942A1028
:100070000C942A100C9476290C945C140C940A1499
:100080000C942A100C94FC6A0C942A1040650C669F
:100090007A6449652066AC64C2646E666E666E669C
:1000A000E1646E666E666E666E665D65EC65EC6557
:1000B0000866A165A1659F659D659B656E666E6618
:1000C0006E666E666E666E666E6630656E666E66CF
:1000D0006E666E666E666E666E666E666E666E6680
:1000E0006E666E666E666E666E666E666E666E6670
:1000F0006E666E666E666E666E666E666E666E6660
:100100006E666E666E666E666E665F6651663F66AA
:10011000246645617379436F6E74726F6C00204D75
:100120004300696E636F6D70617469626C6520482D
:100130005700312E342E34005F03AF01D7006B001F
:10014000470035001A0011000102031718040506C4
:10015000151107080916120A000B0C13100F0E0DCB
:10016000140E111116111116100A00111111110E91
:1001700000110E111111110E0011040A11111F119D
:1001800000010101050D1F0C04040E1F04041F0EC5
:10019000041F1F1F001F1F1F001F1F1F001F111FF5
:1001A000001F111F001F1F1F001F111F001F111F05
:1001B00000000609171709060000060912141209A3
:1001C0000603070F1E1C181000030509121418104F
:1001D00000070707070707070707050505050505C2
:1001E000071C101817150705071C10181711020215
:1001F000021C101812140605021C10181714060110
:10020000061C101815150701011C10181611020103
:10021000061C101816110204071C101812160202F0
:1002200007040A110A0A0E00000C17141714170C01
:10023000001C101810160505051F0A0A0A0A0A1FD5
:10024000000E11111F1B1B1F0002060F1F0F0602BD
:1002500000080C1E1F1E0C08000E0E0E0E1F0E04B2
:1002600000040E1F0E0E0E0E0000C030F00CCC3C31
:10027000FC03C333F30FCF3FFFC303F333CF0FFFB1
:100280003FAAC08030F0B020E0A00CCC8C3CFCBC7D
:100290002CECAC08C88838F8B828E8A803C3833326
:1002A000F3B323E3A30FCF8F3FFFBF2FEFAF0BCBF2
:1002B0008B3BFBBB2BEBAB02C28232F2B222E2A23F
:1002C0000ECE8E3EFEBE2EEEAE0ACA8A3AFABA2A8A
:1002D000EA004060977048685878446454744C6CE5
:1002E0005C7C426252724A6A5A7A466656764E6E12
:1002F0005E7E416151714969597945659F754D6DC2
:100300005D7D436353734B6B5B7B476757774F6FE1
:100310005F7F1018141C121A161E1119151D131BBD
:10032000171FD0D8D4DCD2DAD6DED1D9D5DDD3DBD5
:10033000D7DF9098949C929A969E9199959D939BC5
:10034000505504060507C4C6C5C78486858734365C
:100350003537F4F6F5F7B4B6B5B724262527E4E625
:10036000E5E7A4A6A5A701C18131F1B121E1A10D65
:10037000CD8D3DFDBD2DEDAD09C98939F9B929E90D
:10038000A92020202020200000204D4D49202000C1
:1003900000204D4D01202000002044434320200038
:1003A000002053544F5020000053484F5254210016
:1003B000002048414C5420000000000000000000D4
:1003C000002050524F472000005245534554200012
:1003D00000202054504D2000007E0E0E0E0E1B1BE0
:1003E0001C0E1B1B7E0E0E0E0E232D004144523A96
:1003F00020256C6420202020202020202020002D7B
:100400002D2D2D202000252D35640025336400205E
:100410002001022020202020202000252D356400EE
:10042000252D31312E313173000002070B101419C4
:100430001D22262B3035393F43484C51565B5F64B3
:10044000696D72767B7F0002070C10151A1E232837
:100450002C31363A3F44484D52565B6064696E73A6
:10046000797F00020C151D263039434C565F6972A6
:100470007F2530386C75005741524E494E473A201F
:10048000004552524F523A200062616420706172FE
:10049000616D657465722076616C756500706F774B
:1004A0006572206973204F6666007475726E6F7591
:1004B000742071756575652066756C6C00636F6D71
:1004C0006D616E642071756575652066756C6C0074
:1004D0006E6F2064617461006E6F20736C6F7420A6
:1004E000617661696C61626C65006C6F6B2062752E
:1004F000737900696C6C6567616C207475726E6FDE
:10050000757420616472657373004D4320696E20B9
:1005100048414C54004D4320696E2053544F5000C5
:100520004F6B004572726F7200596573004E6F0019
:1005300042757379210053686F727421004E6F20E9
:100540006465636F646572004E6F2061636B004E7B
:100550006F20706167650042697420726561642074
:100560006572726F720054696D656F7574004D4DE0
:1005700031004D4D3200444343004C207B4C6F6BA7
:10058000232C205B53706565645D2C205B464C5DBD
:100590002C205B4469725D2C205B46315D2C205B16
:1005A00046325D2C205B46335D2C205B46345D7DFE
:1005B0000054207B54726E74232C205B436F6C6F4D
:1005C000725D2C205B5374617475735D7D004620F1
:1005D0007B4C6F6B232C205B46315D2C205B4632BD
:1005E0005D2C205B46335D2C205B46345D2C205B0C
:1005F00046355D2C205B46365D2C205B46375D2CF6
:10060000205B46385D7D00484C2048656C70206654
:100610006F72206C6F6B20636F6D6D616E64730D14
:100620000048462048656C7020666F722066756EC3
:100630006374696F6E20636F6D6D616E64730D001E
:1006400048542048656C7020666F72207475726E15
:100650006F757420636F6D6D616E64730050777297
:10066000206F66660048616C746564210050777283
:10067000206F6E004443432070726F6772616D009B
:1006800054504D2070726F6772616D005245534532
:10069000540048616C746564210D5D004C20257523
:1006A00020257520256320256300756E75736564AC
:1006B000004D6F746F726F6C61204F6C64004D6FF2
:1006C000746F726F6C61204E65770044434300463F
:1006D00020257500465820257500542025642025C6
:1006E00063202564004D43205265766973696F6EFF
:1006F0002000312E342E34000D5365724E722E20A0
:1007000025386C75004D5420256420256400535213
:10071000202564004D6F64756C65202325642028B6
:10072000696E70757420312E2E38202620392E2EB9
:10073000313629203D2000534520256400353736C9
:100740003030002575000D5D0025640025642C20E7
:100750002564002C20004D4D31004D4D32004443A6
:1007600043002C202573002A454E442A002573257A
:1007700064002A454E442A00796573006E6F005B61
:10078000494E464F5D0D0056455253494F4E20008D
:10079000312E342E340048415244574152452048AE
:1007A0005725640D004D43552041544D6567613117
:1007B00032380D0053455249414C20256C750D00CF
:1007C0005B4C4F434F5D0D005B5452414B54494FBE
:1007D0004E535D0D005B414343464D545D0D002576
:1007E000642C20004D4D00444343005B5359535447
:1007F000454D5D0D004C4F4E475041555345004E01
:100800004547415449564553484F52540044454684
:1008100041554C544443430053484F525454494D5E
:10082000452025640D007338384D4F44554C4553D1
:100830002025640D004D41474D494E54494D4520FA
:1008400025640D004D41474D415854494D452025E3
:10085000640D0042415544524154452025750D0018
:100860002A454E442A004D4D004D4D00444343005F
:100870004D4D004D4D004C6F6E67204164647220F9
:100880003D2025750041646472202575203D20249B
:100890002530345820203D3E202043563137203D1E
:1008A00020256420282425303258292C2020435626
:1008B0003138203D20256420282425303258290055
:1008C0005041002564203D202425303258203D2011
:1008D000002564005A7A41003F004800484C004817
:1008E00054004846002E0053544F50002100474FFB
:1008F0000048414C54004C004C4300460046580010
:100900005400590056004D540053520053530053A5
:1009100045004040004200534F0043560043410011
:10092000504400504100505452520050545752000D
:10093000505452500050545750005054524400509C
:10094000545744005054524200505457420050549F
:10095000524C005054574C004C53004C4F4344559C
:100960004D50004C4F43414444004C4F43434C4591
:1009700041520054524B44554D500054524B414447
:10098000440054524B434C45415200434647445562
:100990004D50004346474143430043464753595354
:1009A0000054504D00556E6B6E6F776E20636F6D07
:1009B0006D616E64000D5D00313200003234000064
:1009C0003438000039360000313434003139320017
:1009D00033383400353736004142434445464748B2
:1009E000494A4B4C4D4E4F505152535455565758FF
:1009F000595A303132333435363738392E2C3A2D76
:100A00002B232F3D3C7C3E20004D4D2049202031A2
:100A10003420004D4D20492020323761004D4D20BB
:100A2000492020323762004D4D20012020313420F2
:100A3000004D4D20012020323761004D4D20012016
:100A400020323762004443432020203134200044C8
:100A500043432020203238200044434320203132B9
:100A60003820004C6F636D656E750000000000005B
:100A70000000004443432D70726F6772616D6D2EEC
:100A80000000004D6F64656C6261616E7369742E65
:100A9000000000496E7374656C6C696E67656E006A
:100AA000000000536F667477617265205570646151
:100AB0007465004C4344207665726C6963687469A0
:100AC0006E67004D6173746572436F6E74726F6C04
:100AD000000000457869740000000000000000007C
:100AE0000000004B69657A656E2000000000000080
:100AF00000000044617461666F726D6174000000F3
:100B00000000004E61616D202020202020000000A8
:100B1000000000496E766F657220202020000000E2
:100B20000000003132384653204D6F6465000000EC
:100B300000000043562028627974652900000000F7
:100B4000000000435620286269742900000000005C
:100B50000000004261736973616472657300000094
:100B60000000004C616E67206164726573000000D4
:100B70000000005265676973746572000000000030
:100B8000000000506167652D4D6F64650000000036
:100B9000000000486F6F666473706F6F7200000032
:100BA0000000007338382D696E7374656C6C696E63
:100BB00067656E436F6E666967757261746965001B
:100BC000000000426F6F7374657200000000000047
:100BD000000000496E74657266616365204261754C
:100BE00064000057697373656C000000000000002A
:100BF0000000004C6F63666F726D6174000000004E
:100C00000000004D4D207369676E61616C70617505
:100C10007A65007338382D6D6F64756C650000005F
:100C20000000007338382D6D6F64756C65746573E2
:100C30007400004B6F7274736C2E20706F6C2E00FA
:100C40000000004B6F7274736C2E206765762E0067
:100C5000000000616C6C652057697373656C7300EC
:100C600000000057697373656C666F726D61740084
:100C70000000004D696E2E736368616B656C74696A
:100C80006A64004D61782E736368616B656C74698A
:100C90006A64004D656E75204C6F636F0000000044
:100CA00000000050726F6772616D2E204443430054
:100CB00000000045746174205265736561752E00F3
:100CC0000000005265676C616765730000000000FA
:100CD0000000004D414A206C6F67696369656C00D4
:100CE0000000004C756D696E6F73697465000000DB
:100CF0000000004D6173746572436F6E74726F6CA7
:100D00000000004578697400000000000000000049
:100D100000000053656C656374696F6E200000000D
:100D2000000000466F726D617420646F6E6E6565C1
:100D30007300004E6F6D2020202020202000000036
:100D400000000053616973696520202020000000C5
:100D50000000003132384653204D6F6465000000BA
:100D600000000043562028627974652900000000C5
:100D7000000000435620286269742900000000002A
:100D800000000041647265737365206465206261D0
:100D900073650041647265737365206C6F6E67756F
:100DA0006500005265676973746572000000000099
:100DB000000000506167652D4D6F64650000000004
:100DC000000000566F6965207072696E636970611A
:100DD0006C65005265676C61676520733838000088
:100DE000000000436F6E66696775726174696F6EAB
:100DF000000000426F6F7374657200000000000015
:100E0000000000496E746572666163652042617519
:100E1000640000436F6E662E2041696775696C6CD3
:100E2000612E00466F726D6174206C6F636F0000FD
:100E30000000005061757365207369676E616C20F6
:100E40004D4D004D6F64756C65732073383800002C
:100E500000000054657374206D6F64756C652073B9
:100E6000383800506F6C2E6372742D63697263752D
:100E700069740053656E732E206372742D636972FA
:100E8000637400746F75732061696775696C6C6158
:100E90002E0000466F726D61742061696775696C20
:100EA0006C2E00547073206D696E2E696D70756CB8
:100EB000732E00547073206D61782E696D70756C9F
:100EC000732E004C6F6B204D656EFC00000000001F
:100ED0000000004443432D50726F6772616D6D676F
:100EE0002E0000416E6C6167656E7A757374616E79
:100EF00064000045696E7374656C6C756E67656E31
:100F0000000000536F6674776172652055706461EC
:100F10007465004C43442042656C65756368747564
:100F20006E67004D6173746572436F6E74726F6C9F
:100F30000000004578697400000000000000000017
:100F400000000041757377E4686C656E2000000056
:100F5000000000446174656E666F726D617400001C
:100F60000000004E616D6520202020202000000040
:100F700000000045696E7472616720202000000047
:100F80000000003132384653204D6F646500000088
:100F90000000004356202862797465290000000093
:100FA00000000043562028626974290000000000F8
:100FB00000000042617369732D416472657373654B
:100FC0000000006C616E6765204164726573736533
:100FD00000000052656769737465720000000000CC
:100FE000000000506167652D4D6F646500000000D2
:100FF0000000004861757074676C656973000000DB
:101000000000007338382D45696E7374656C6C751B
:101010006E67004B6F6E66696775726174696F6E9B
:10102000000000426F6F73746572000000000000E2
:10103000000000496E7465726661636520426175E7
:101040006400005765696368656E00000000000079
:101050000000004C6F6B666F726D617400000000E1
:101060000000004D4D2D5369676E616C2050617515
:101070007365007338382D4D6F64756C6500000022
:101080000000007338382D4D6F64756C746573748F
:101090000000004B75727A7363686C2E2D506F6C74
:1010A0002E00004B75727A7363686C2E2D456D703F
:1010B000662E00616C6C65205765696368656E001B
:1010C0000000005765696368656E666F726D6174D4
:1010D0000000006D696E2E20536368616C747A6540
:1010E0006974006D61782E20536368616C747A6551
:1010F0006974004C6F636F6D6F74697665206D6500
:101100006E75004443432070726F6772616D6D6944
:101110006E67004C61796F757420737461747573B8
:1011200000000053657474696E677300000000006E
:10113000000000536F6674776172652055706461BA
:101140007465004C4344206261636B6C696768742A
:101150000000004D6173746572436F6E74726F6C42
:1011600000000045786974000000000000000000E5
:1011700000000053656C65637420000000000000EF
:101180000000004461746120666F726D617400003C
:101190000000004E616D652020202020200000000E
:1011A000000000456E74727920202020200000008D
:1011B0000000003132384653204D6F646500000056
:1011C0000000004356202862797465290000000061
:1011D00000000043562028626974290000000000C6
:1011E0000000005072696D617279206164647265FB
:1011F000737300457874656E642E20616464726553
:1012000073730052656769737465720000000000B3
:10121000000000506167652D4D6F6465000000009F
:101220000000004D61696E20747261636B00000004
:101230000000007338382073657474696E6773003A
:1012400000000044656C657465000000000000004B
:10125000000000426F6F73746572000000000000B0
:10126000000000496E7465726661636520426175B5
:10127000640000506F696E7473000000000000008D
:101280000000004C6F632E20666F726D6174000069
:101290000000004D4D207369676E616C20706175B0
:1012A000736500733838206D6F64756C657300006A
:1012B000000000733838206D6F64756C65207465AC
:1012C00073740053686F727420632E20706F6C2EDD
:1012D00000000053686F727420632E2073656E7374
:1012E0002E0000616C6C20506F696E7473000000FA
:1012F000000000506F696E747320666F726D6174C8
:101300000000006D696E2E7377697463682E7469CE
:101310006D65006D61782E7377697463682E7469EA
:101320006D6500202D2D2D2D0025357500536F6620
:1013300074772E205600312E342E34005365724EB1
:10134000722E2025386C75003A2000253575002551
:101350003364002534643A20002D2D2D002533649C
:1013600000204F4B20202020002020202020202063
:101370000043563A20202020204269743A203D2024
:101380000043563A253464204269743A25643D008E
:10139000202D2D2D0025346400202D2D2D2D2D00E8
:1013A00025366400202E2E2E2E20202020202020C6
:1013B0002020002533642C256473002534646D736C
:1013C000003030204261756400446F776E6C6F614D
:1013D00064202E2E2E002564206D7300202532649B
:1013E000004E723A2025326420200073686F7274B8
:1013F0002028312E356D73292000006C6F6E672018
:1014000028342E3032356D732900004D6F746F72A1
:101410006F6C610000000000000000444343202086
:1014200020202000000000000000004D4D200000A2
:1014300000000000000000000000004443430000E2
:101440000000000000000000000000706F7369746D
:1014500069766520284D4D290000006E656761742E
:10146000697665202844434329000053617665204E
:101470002020202020202020202000526573746F1F
:1014800072652020202020202020005361766520D6
:101490002020202020202020202000526573746FFF
:1014A0007265202020202020202000206C61796F90
:1014B0007574207374617475732000206C61796F8A
:1014C00075742073746174757320004B6F72722091
:1014D00028312E356D7329202000004C616E672065
:1014E00028342E3032356D732900004D6F746F72C1
:1014F0006F6C6100000000000000004443432020A6
:1015000020202000000000000000004D4D200000C1
:101510000000000000000000000000444343000001
:101520000000000000000000000000506F736974AC
:1015300069656620284D4D290000004E656761747D
:1015400069656620284443432900004D6F64656C3B
:101550006261616E7369742E2020004D6F64656C4A
:101560006261616E7369742E202000486572737425
:10157000656C6C656E2020202020004F70736C61BC
:10158000616E2020202020202020002068657273BA
:1015900074656C6C656E2020202000206F70736C69
:1015A00061616E2020202020202000436F7572741E
:1015B0002028312E356D73292000004C6F6E672076
:1015C00028342E3032356D732900004D6F746F72E0
:1015D0006F6C6100000000000000004443432020C5
:1015E00020202000000000000000004D4D200000E1
:1015F0000000000000000000000000444343000021
:101600000000000000000000000000706F736974AB
:1016100069766520284D4D290000006E656761746C
:101620006976652028444343290000456E7265674A
:1016300069737472656D656E7420005265737461B0
:1016400075726174696F6E20202000456E72656747
:1016500069737472656D656E742000526573746190
:1016600075726174696F6E2020200020457461746A
:10167000205265736561752E2020002045746174C9
:10168000205265736561752E2020004B75727A209B
:1016900028312E356D7329202000004C616E6720A3
:1016A00028342E3032356D732900004D6F746F72FF
:1016B0006F6C6100000000000000004443432020E4
:1016C00020202000000000000000004D4D20000000
:1016D0000000000000000000000000444343000040
:1016E0000000000000000000000000706F736974CB
:1016F000697620284D4D29000000006E65676174F1
:101700006976202844434329000000416E6C6167DC
:10171000656E7A757374616E642000416E6C6167EA
:10172000656E7A757374616E6420005769656465CF
:10173000726865727374656C6C6E00537065696372
:101740006865726E20202020202000207769656463
:10175000657268657273742E20200020737065694D
:10176000636865726E202020202000696E636F6DB3
:101770007061742E20466F726D617400496E636FE4
:101780006D702E20466F726D6174202000466F725E
:101790006D617420696E636F6D7061742E00696E87
:1017A0006B6F6D7061742E20466F726D6174002EC8
:1017B0002E2E2077616974696E67202E2E2E2000F0
:1017C000233D64656C657465000000000000000046
:1017D00000286E6F20656E74727929000000000089
:1017E00000002E2E2E2064656C6574696E67202EB5
:1017F0002E2E00206661756C740000000000000051
:101800000000000020444343206F6E6C79210000EB
:10181000000000000020707265737320474F20663F
:101820006972737400002A3D43616E63656C202009
:10183000200000000000002070726F6772616D6907
:101840006E670000000000002D73686F72742063E3
:101850006972637569742D2000206E617469766504
:101860002028313A312920202000206C696E6561E2
:10187000722028323A3129202020002070726F67B0
:101880007265737369766520202020002A72656175
:10189000642000000000000000000000002A7772B1
:1018A00069746500000000000000000000002E2E9A
:1018B0002E2077726974696E67202E2E2E20002EDE
:1018C0002E2E2072656164696E67202E2E2E2000F8
:1018D000212121206661756C742021212120202086
:1018E00000204F4B202020202020202020202020BE
:1018F00020002E2E2E20736176696E67202E2E2EEC
:101900002020002E2E20726573746F72696E67201E
:101910002E2E2000233D44656C2E202A3D43616E0F
:1019200063656C2000233D596573202A3D43616E39
:1019300063656C20200020636F6E66696775726155
:1019400074696F6E2020004F4646000000000000C2
:1019500000000000000000002A2A2A206E6F205498
:101960007261696E202A2A2A002A2073686F7274B5
:10197000206369726375697420002A2A2A207469B9
:101980006D65206F7574202A2A2A00506F696E7465
:1019900020202534642F253464000000436F6E66D8
:1019A000696775726174696F6E2020200020636F13
:1019B0006E66696775726174696F6E2020002E2EE5
:1019C0002E207761636874656E202E2E2E200023F2
:1019D0003D77697373656E00000000000000000031
:1019E000286765656E20696E766F65722900000054
:1019F00000202E2E2E2077697373656E202E2E2EDA
:101A0000000020666F7574000000000000000000F8
:101A100000000020416C6C65656E2044434321004A
:101A20000000000020707265737320474F206669C4
:101A300072737400002A3D2041666272656B656EA8
:101A40000000000000002050726F6772616D6D65CC
:101A500072656E000000002D2D4B6F7274736C75F3
:101A60006974696E672D2D00206E6174697665203A
:101A700028313A312920202000206C696E6561727E
:101A80002028323A3129202020002070726F67729E
:101A900065737369766520202020002A4C657A657D
:101AA0006E00000000000000000000002A53636880
:101AB000726900000000000000000000002E2E20CF
:101AC00073636872696A76656E202E2E00002E2E72
:101AD0002E206C657A656E202E2E2E202000002090
:101AE00021212120466F7574202121212020000012
:101AF000204F4B20202020202020202020202000AC
:101B0000002E2E2E204F70736C61616E202E2E2EB3
:101B100000004865727374656C6C656E202020202F
:101B2000200000233D77697373656E202A3D61664E
:101B300062720000233D4A61202A3D41666272655F
:101B40006B656E20002077697373656E20202020FE
:101B500020202020200055495400000000000000F3
:101B6000000000000000002A2A2A206765656E2018
:101B70004C6F63202A2A2A002A2A6B6F7274736CB6
:101B8000756974696E672A2A002A2054696A646F2D
:101B9000766572736368722E2A0057697373656C79
:101BA000732534642F253464000000436F6E66692A
:101BB00067202020202020202020200020436F6E3E
:101BC000666967202020202020202020005061749A
:101BD00069656E74657A0000000000000000233D16
:101BE0007375707072696D65720000000000007698
:101BF00069646500000000000000000000000000B3
:101C00005375707072657373696F6E000000000029
:101C1000002045727265757200000000000000002F
:101C200000002044434320756E697175656D656ED3
:101C300074000020707265737320474F20666972CC
:101C4000737400002A3D4162616E646F6E20200053
:101C500000000000002050726F6772616D6D61744A
:101C6000696F6E0000002D436F7572742D63697289
:101C7000637569742D2000206E6174697665202873
:101C8000313A312920202000206C696E6561722074
:101C900028323A3129202020002070726F67726547
:101CA000737369766520202020002A4C6563742EAA
:101CB00000000000000000000000002A4563726977
:101CC0007400000000000000000000002E2E2E20F6
:101CD0004563726974757265202E2E2E002E2E2E8D
:101CE000204C656374757265202E2E2E20002121F4
:101CF000212045727265757220212121202000204B
:101D00004F4B202020202020202020202020200099
:101D100020456E72656769737472656D656E7420B7
:101D20000020526573746175726174696F6E202052
:101D30002000233D5375707072202A3D4162616E10
:101D4000642E00233D4F7569202A3D4162616E6417
:101D50006F6E2000205375707072696D657220205F
:101D60002020202000496E616374696620202020B5
:101D70002020202020002A20506173206465206CE0
:101D80006F636F202A20002A20436F7572742D63C1
:101D900069726375697420002A2054656D70732020
:101DA00064657061737365200041696775696C2EA5
:101DB0002534642F253464000000456E7265676920
:101DC000737472656D656E74202000526573746162
:101DD00075726174696F6E20202020002E2E2E20D7
:101DE00077617274656E202E2E2E202000233D4CCC
:101DF000F6736368656E0000000000000000286B49
:101E000065696E2045696E74726167290000002063
:101E10002E2E2E206CF673636865202E2E2E200049
:101E2000204665686C65720000000000000000003C
:101E300000206E75722066FC72204443432100002E
:101E40000000206572737420474F206472FC636B3E
:101E5000656E002A203D2041626272756368000051
:101E6000000000002050726F6772616D6D696572CD
:101E7000756E6700002D2D204B75727A7363686C48
:101E800075DF202D2D00204E617469762028313AAF
:101E900031292020202000204C696E6561722028A5
:101EA000323A3129202020002050726F677265730A
:101EB0007369762020202020002A6C6573656E00EF
:101EC000000000000000000000002A736368722E0A
:101ED00000000000000000000000002E2E207363B0
:101EE0006872656962656E202E2E00002E2E2E20EF
:101EF0006C6573656E202E2E2E202000002121217E
:101F0000204665686C657220212121200000204F49
:101F10004B20202020202020202020202000002EC8
:101F20002E2073706569636865726E202E2E000026
:101F30007769656465726865727374656C6C656EEB
:101F400000233D4CF6736368656E202A3D41626252
:101F50007200233D4A61202A3D41626272756368C6
:101F6000000000206CF6736368656E20202020203E
:101F70002020200041555300000000000000000018
:101F800000000000002A2A206B65696E65204C6FF6
:101F90006B202A2A20002A2A204B75727A736368E4
:101FA0006C75DF202A2A002A205A656974FC626554
:101FB00072736368722E2A0057656963686520250D
:101FC00034642F2534640000004B6F6E66696775BA
:101FD000726174696F6E20202000204B6F6E6669FD
:101FE0006775726174696F6E2020005B6E6F206D83
:101FF0006573736167655D005B756E6B6E6F776EA1
:10200000206572726F725D005B756E6B6E6F776EBE
:10201000207374617475735D000011241FBECFEFCF
:10202000D0E1DEBFCDBF12E0A0E0B1E0E0EEFCEF1A
:1020300000E00BBF02C007900D92AA33B107D9F799
:102040001CE0AAE3B2E001C01D92A93AB107E1F792
:102050000C9498100C94000081E080933B0208954A
:10206000982F80913A02891731F0863021F085301F
:1020700029F4963019F080E090E0089590933A02A8
:10208000892F8250823010F0973059F40E9421221B
:1020900010923F0680913A02823051F40E94072F3D
:1020A00007C0943019F40E945F2202C00E944B22A4
:1020B00080913A02863011F40E943A6380913A028C
:1020C000813019F482E00E94C5774AE352E063E070
:1020D0008FEF0E94EF630E942C1081E090E0089542
:1020E000089580913A029927089580E00E94261D64
:1020F0002FEF8F3F920719F0682F80E009C081E031
:102100000E94261D2FEF8F3F920721F0682F81E05C
:102110000E94074C0E9405640E94F7740E94743369
:1021200080913B02882311F40E94CA1BA895089550
:10213000CFEFD0E1DEBFCDBF0E94F7600E947911E2
:102140000E941A2A0E9418740E948D220E943761F0
:1021500021E04EE468E00E94A71121E04EE468E02F
:1021600087E00E94BD130E94501578940E94881742
:102170000E942F61FC0184810E94321C62E171E0A7
:1021800082E00E94A41C0E947A61813059F060E0D4
:1021900081E00E94E01A62E271E082E00E94A41CE9
:1021A000A895FECF6EE171E082E00E94A41C60E081
:1021B00081E00E94E01A66E582E00E94371C62E33B
:1021C00071E082E00E94A41C0E942F618C0181E0DA
:1021D0000E94B119882319F081E00E94326182E0E7
:1021E0000E94B119882319F080E00E94326183E0D7
:1021F0000E94B119882319F082E00E94326184E0C4
:102200000E94B119882319F083E00E94326180E0B6
:102210000E94301081E00E94E16A80E00E94B119C2
:10222000882319F084E10E94BE5F0E94FF6E40E0A7
:1022300050E060E28FEF0E94EF6380E00E94EB4B82
:1022400081E00E94EB4B8091410690914206A09163
:102250004306B0914406805D9740A040B04078F4BA
:102260000E9475108091410690914206A09143060C
:10227000B0914406805D9740A040B04088F3F801DB
:1022800081859285892BC9F00E94532FEC014A96D3
:102290009E012B5E3F4FAC01B901F801818592850B
:1022A0000E94866DBC01892B29F0F80181859285F9
:1022B000888F998F6115710519F4F8016281738116
:1022C0008FEF0E94AA6281E011C00E94AA330E948F
:1022D000771AFFEF8F3F9F07C1F70E94751080911B
:1022E0003B028823A1F310923B0280E00E94E93078
:1022F000EECF8FE78ABB1BBA80E187BB18BA80EFAD
:1023000084BB8FEF85BB8BEB81BB8CEC82BB82E007
:1023100082B987EF83B987E78093610081EF80936B
:1023200062008FE18093640089E1809365000E94E0
:10233000F36A10926A001ABE8AB78A608ABF0E9446
:102340000519A89588E181BD8CE081BD0895E82F2D
:102350001092130680911306809312068091120644
:1023600080933506809135068093340691E09093F2
:102370003E068C9A119A82B18E7E82B9199A83B1E7
:102380008E7E83B982E08BB99498E83008F0E92F0B
:10239000FF27EE0FFF1FE85CFE4FA591B49165305B
:1023A00010F465E003C0693008F068E04F7D6550C7
:1023B000660F453411F4606203C04F3409F4606362
:1023C000223008F068608B2F992787FD9A958F70CF
:1023D00080939000A9B96093950088EB8AB980E05A
:1023E00090E008951F920F920FB60F9211248F93D1
:1023F0009F93EF93FF939091340680913506981741
:1024000061F088B7806188BF0C9B09C080913E064F
:1024100080FF05C089B7806189BF559813C080913E
:102420003506E82FFF27EE5EF94F84A18CB9809125
:1024300035068F5F8093350680913506883010F021
:1024400010923506FF91EF919F918F910F900FBEE3
:102450000F901F9018951F920F920FB60F92112494
:102460008F9389B78F7E89BF559A8F910F900FBE3A
:102470000F901F9018951F920F920FB60F92112474
:102480002F933F934F935F936F937F938F939F937C
:10249000AF93BF93EF93FF9380911206282F3327BA
:1024A00080911306992701972817390741F08091E9
:1024B00012068F3179F480911306882359F48091A4
:1024C00013068F5F8093130680911306803210F0FD
:1024D000109213069BB180911206E82FFF27EE5E43
:1024E000F94F8CB18283228194FD0CC08091120639
:1024F0008F5F80931206809112068032A8F01092AE
:10250000120612C0222381F4209313068091130631
:10251000809312069498822F0E94EB4B21E04EE4A8
:1025200068E0822F0E94A71180911206282F33277E
:1025300080911306281B310937FF02C0205E3F4FF0
:10254000213131050CF0949AFF91EF91BF91AF9139
:102550009F918F917F916F915F914F913F912F91BB
:102560000F900FBE0F901F90189550E060E070E044
:1025700027E0813D920708F051E02FE0813A920771
:1025800008F052E023E28932920708F053E026E394
:10259000813B920708F054E026E48135920708F069
:1025A00055E028E8893B920708F056E0895D964D92
:1025B00008F057E078948BB1992726E09695879597
:1025C0002A95E1F79C012170307080FFB9016F5F9F
:1025D0007F4FA89587E26031780768F321E04EE4E9
:1025E00068E0852F0E94A7110895992783309105EF
:1025F00009F1843091054CF481309105A9F08230C5
:102600009105ACF4892B69F024C085309105C1F0A7
:102610008530910594F086309105A9F00797B1F0C7
:1026200018C080EB94E0089580E699E0089580EC6E
:1026300092E1089580E895E2089580E498E3089592
:1026400080E09BE4089580E096E9089580E091EEB3
:10265000089580E090E00895089589B1282F3327E8
:10266000809190009927982F8827282B392B60E09C
:1026700040E050E0FA01E85CFE4F859194918217AA
:10268000930729F06F5F4E5F5F4F683098F3862F96
:102690000E94F5120895482F06C0809135068823C0
:1026A00091F4559A7894A89580913406282F332771
:1026B00080913506992701972817390791F3809162
:1026C0003406873051F380913406E82FFF27EE5E01
:1026D000F94F44A3809134068F5F80933406809134
:1026E0003406883010F010923406559A80E090E05D
:1026F0000895F89480911206282F332780911306AD
:10270000281B3109789437FF02C0205E3F4F2031EB
:1027100031050CF49498232B19F48FEF9FEF089553
:1027200080911306E82FFF27EE5EF94F8281282F54
:102730003327F894809113068F5F8093130680915E
:102740001306803210F0109213067894C901089590
:10275000089590913E069170882331F080913E0655
:10276000816080933E0606C080913E068E7F8093F6
:102770003E06559A892F99270895E82F1092E6056D
:102780008091E6058093E5058091E5058093080634
:10279000809108068093070691E09093110681B31B
:1027A000886281BB8A981598939A92981D9882E0C6
:1027B00080939B009598E83008F0E92FFF27EE0FF3
:1027C000FF1FE85CFE4FA591B491653010F465E001
:1027D00003C0693008F068E04F7D6550660F8B2FAD
:1027E000992787FD9A958F7080939800A093990000
:1027F000453411F4606203C04F3409F46063223041
:1028000008F0686060939D0088EB80939A0080E0F8
:1028100090E008951F920F920FB60F9211248F939C
:102820009F93EF93FF939091070680910806981766
:1028300061F088B7806288BF0D9B0DC08091110642
:1028400080FF09C089B7806289BF80919A008F7D1F
:1028500080939A0014C080910806E82FFF27EB515F
:10286000FA4F84A180939C00809108068F5F80932B
:10287000080680910806883010F010920806FF9133
:10288000EF919F918F910F900FBE0F901F90189511
:102890001F920F920FB60F9211248F9389B78F7DDD
:1028A00089BF80919A00806280939A008F910F90E7
:1028B0000FBE0F901F9018951F920F920FB60F9298
:1028C00011242F933F934F935F936F937F938F9335
:1028D0009F93AF93BF93EF93FF938091E505282FCC
:1028E00033278091E605992701972817390741F08A
:1028F0008091E5058F3179F48091E605882359F4BC
:102900008091E6058F5F8093E6058091E605803231
:1029100010F01092E60590919B008091E505E82F5C
:10292000FF27EB51FA4F80919C008283828194FDB6
:102930000CC08091E5058F5F8093E5058091E505EA
:10294000803278F01092E5050CC0882351F4809312
:10295000E6058091E6058093E505959881E00E9463
:10296000EB4B8091E505282F33278091E605281B46
:10297000310937FF02C0205E3F4F213131050CF095
:10298000959AFF91EF91BF91AF919F918F917F9118
:102990006F915F914F913F912F910F900FBE0F90CC
:1029A0001F901895482F0AC0809108068823B1F41B
:1029B00080919A00806280939A007894A895809183
:1029C0000706282F33278091080699270197281793
:1029D000390771F380910706873031F3809107063C
:1029E000E82FFF27EB51FA4F44A3809107068F5F32
:1029F0008093070680910706883010F01092070632
:102A000080919A00806280939A0080E090E008951F
:102A1000F8948091E505282F33278091E605281B3F
:102A20003109789437FF02C0205E3F4F20313105D5
:102A30000CF49598232B19F48FEF9FEF0895809154
:102A4000E605E82FFF27EB51FA4F8281282F332725
:102A5000F8948091E6058F5F8093E6058091E60506
:102A6000803210F01092E6057894C9010895089517
:102A700090913E069170882331F08091110681601B
:102A8000809311060AC0809111068E7F80931106F3
:102A900080919A00806280939A00892F99270895E7
:102AA00087B3876087BBBB9888B3896088BB1DB834
:102AB0008EB18FB187E78DB908951F920F920FB62F
:102AC0000F9211242F938F939F93EF93FF937894FA
:102AD0002FB180913C02E82FFF27E45CFD4F228359
:102AE0008F5F80933C02883110F010923C029091ED
:102AF0005702E92FFF27E45CFD4F248D27FDC09A84
:102B000080915602981759F0C098892F8F5F809353
:102B10005702883110F0109257022FB902C0C09AA4
:102B20006F98FF91EF919F918F912F910F900FBE12
:102B30000F901F90189580915702282F332780916E
:102B40005602281B3109C90147968831910514F0B6
:102B5000C901019708950895282F6F9919C0C09849
:102B60008FB16F9A8091560290915702891711F494
:102B70002FB91CC0E92FFF27E45CFD4F848D8FB96E
:102B8000892F8F5F80935702883110F0109257027F
:102B900080915602E82FFF27E45CFD4F248F8F5F62
:102BA00080935602883110F01092560280E090E037
:102BB000089580913C0220913D02821719F48FEF15
:102BC0009FEF0895E22FFF27E45CFD4F8281482F9D
:102BD0005527822F8F5F80933D02883110F010922D
:102BE0003D02CA01907008950895882311F0DD9A7E
:102BF0000895DD9808950895CF93382FA091760217
:102C0000B0917702109711F4882321F4809170021B
:102C1000882361F1809170028F5F80937002992701
:102C20008330910509F475C0843091053CF48130FE
:102C3000910581F0029709F46FC018C086309105A4
:102C400069F0873091051CF4059731F00FC00797A4
:102C500049F00CC0DC9A60C081E001C080E00E94B5
:102C6000F5155AC0DC981092700256C0DE9B4FC01A
:102C7000332309F04CC0CD0153E0969587955A95C2
:102C8000E1F7209176022770932FCF9991E0482F9A
:102C90005527622F7727C091E509992399F0FA010A
:102CA000E959F54F20E830E002C0359527956A953F
:102CB000E2F78081822B8083FA01E95DF54F808104
:102CC000822B0EC0FA01E959F54F80E890E002C06E
:102CD000959587956A95E2F7982F9095808189233D
:102CE00080839D012F5F3F4F3093770220937602C0
:102CF0008C2F992744E0880F991F4A95E1F72817F0
:102D0000390748F0109277021092760204C03323FC
:102D100011F0DE9A01C0DE98CF9108950000000006
:102D2000000000000895882341F0809165008460D0
:102D3000809365000E948E160895809165008B7FB8
:102D400080936500089508951F93182F8AB3807F9C
:102D50008ABB80E00E949316809165008260809318
:102D60006500112321F080916500816003C080918E
:102D700065008E7F809365000000000081E00E9466
:102D8000931619B380E00E9493161295107F0E944B
:102D90008E1681E00E94931689B38F70182B80E005
:102DA0000E949316812F99271F91089580E00E9419
:102DB000A416982F80917402882331F497FD04C0E3
:102DC000892F8F7780937502892F992787FD90959A
:102DD0008827990F881F992708959B01AC0180913E
:102DE000410690914206A0914306B0914406821795
:102DF0009307A407B507A0F0809141069091420681
:102E0000A0914306B0914406821B930BA40BB50B13
:102E100080509041A040B040A0F080E090E0089544
:102E20008091410690914206A0914306B0914406DC
:102E3000281B390B4A0B5B0B2050304F4F4F5F4F15
:102E400018F081E090E0089580E090E00895089502
:102E5000EF92FF920F931F93AA27BB27E0904106A2
:102E6000F09042060091430610914406E80EF91EC8
:102E70000A1F1B1F01C0A895C801B7010E94ED16CB
:102E80008823C9F31F910F91FF90EF9008950F933E
:102E90001F93CF93C82F162F042F809165008D7F2D
:102EA0008093650080E00E9493168AB38F608ABB8E
:102EB0008BB3807F9C2F92959F70892B8BBB1123A6
:102EC00021F080916500816003C0809165008E7F54
:102ED0008093650081E00E94931680E00E94931623
:102EE000002329F088E090E00E9428170DC08BB3E2
:102EF000807FCF708C2B8BBB0E948E1681E00E944E
:102F00009316802F0E949316CF911F910F910895D1
:102F10000F931F93CF9388E290E00E94281741E01F
:102F200060E080E30E94471741E060E080E30E9498
:102F3000471741E060E080E30E94471741E060E00E
:102F400080E20E94471788E20E94D61A80E40E941D
:102F5000D61A8AE00E94921A89E20E94D61A8CE15F
:102F60000E94D61A82E50E94D61A89E60E94D61AD5
:102F700084E70E94D61A80E40E94D61A85E10E9456
:102F8000921A88E20E94D61A80E40E94D61A0E9401
:102F9000532F8C0101C0A89590914506809146065B
:102FA0009817C9F70E94D616C82F8823A1F781E089
:102FB0000E94A4168A3021F481E0F80187A302C0A0
:102FC000F801C7A388E00E94D61A81E00E94D61AB1
:102FD00086E00E94D61A8CE00E94D61A60E0862F06
:102FE0000E94E01A61E672E080E00E940F1C69E333
:102FF00072E081E00E940F1C61E472E082E00E94B6
:103000000F1C69E272E083E00E940F1CCF911F91B8
:103010000F9108951F920F920FB60F9211242F93C4
:103020003F934F935F936F937F938F939F93AF9350
:10303000BF93CF93EF93FF9380917302882309F09E
:10304000D2C081E080937302789480E00E94FC15E6
:10305000809171028F5F8093710280917102837001
:1030600099278130910519F1823091051CF4892B43
:1030700041F0B4C08230910571F1039709F464C046
:10308000ADC08091410690914206A0914306B09157
:1030900044060196A11DB11D8093410690934206FE
:1030A000A0934306B09344060E945D1A97C0809196
:1030B000410690914206A0914306B091440681706A
:1030C0009070A070B070892B19F00E94C41986C04E
:1030D0000E94851983C00E947110833029F00E94DC
:1030E0007110823009F07AC00E94982220913F0628
:1030F000309140068823E9F02E5F3F4F3093400621
:1031000020933F060E942F61FC019681992309F4C8
:1031100065C08AE0989F9001112480913F069091AC
:1031200040068217930708F459C081E00E943010CE
:1031300055C02115310509F451C02150304030935C
:10314000400620933F064AC060917202662319F040
:103150000E94D61641C09091450680914606981768
:1031600089F0C0914606EC2FFF27EB5BF94F2281D7
:10317000CF5FC03108F0C62F203829F58091450671
:103180008C1719F480E090E027C0EC2FFF27EB5B51
:10319000F94F22812F3F19F420917502206827FFF3
:1031A00002C060937402822F9927807C90708034D3
:1031B000910519F481E080937402CF5FC03108F06B
:1031C000C62F462F02C0462F61E0822F0E9447176C
:1031D000C093460681E090E08093720281E00E94F5
:1031E000FC1510927302FF91EF91CF91BF91AF91B7
:1031F0009F918F917F916F915F914F913F912F910F
:103200000F900FBE0F901F90189510927D0080B701
:10321000877F80BF17BE11BE89E683BF82E085BD70
:1032200087B7806487BF82EF8FBD3AE13EBD4FEC28
:1032300050E057BD46BD85EB90E09BBD8ABD99BD72
:1032400088BD22EC20938B0030938A00509381003C
:103250004093800090938700809386000E942F61A6
:10326000FC0180858093E5090895EF92FF920F930A
:103270001F93AA27BB27E0904106F09042060091D9
:10328000430610914406E80EF91E0A1F1B1F02C0D8
:103290000E947510C801B7010E94ED168823C1F382
:1032A0001F910F91FF90EF900895282F220F611129
:1032B0002160822F83708150823028F424FF02C065
:1032C0002E6001C0217F822F9927089590917A0264
:1032D000E92FFF27E658FD4F8283892F8F5F809368
:1032E0007A02883010F010927A0290917B028091DD
:1032F0007A02981741F4892F8F5F80937B02883080
:1033000010F010927B02089508950F931F9311B14E
:10331000812F8074682F809178020E945519082FA0
:10332000809378021078612F809179020E9455195C
:1033300080937902007C807C003829F4882339F05E
:10334000803C61F408C0003449F4803C11F489E108
:1033500003C0882319F48AE10E9466191F910F9116
:103360000895893118F080E090E0089520E030E081
:10337000E82FFF27EC57FD4F8081882311F021E0D3
:1033800030E0C90108950895FF920F931F93CF93E2
:103390008091A202E82FFF27E356FD4F008113B36F
:1033A0001F7081B1880F880F8071182B1083FF2444
:1033B0008091A20225E0829FF0011124EF0DF11D02
:1033C000E85BFE4FC49110FD42C000FF14C0C6313F
:1033D00029F485E10E94B119882331F48C2F0E94D1
:1033E0006619C93108F054C0EC2FFF27EC57FD4F88
:1033F00081E080834DC0C93108F04AC0EC2FFF271F
:10340000DF01AC57BD4F9C919F5F9C93992311F4B2
:103410009F5F9C93E531F105DCF1E731F1056CF03C
:103420007797B1F580919B02853690F181E20E94F9
:10343000661981E080939B022BC0809199028937A5
:1034400038F180919A02893718F1822F1FC0C93153
:1034500028F4EC2FFF27EC57FD4F108200FD18C019
:103460008C2F80680E9466190E947110853081F44B
:10347000C53121F486E10E94B11905C0C63141F47D
:1034800085E10E94B119882319F486E00E9430106A
:1034900016950695F39484E08F1508F089CF8091F6
:1034A000A2028F5F8093A202853010F01092A202D8
:1034B000CF911F910F91FF9008959091A2029430A7
:1034C00029F485B3806F85BB97980895979A85B343
:1034D0008F7020E130E002C0220F331F9A95E2F78F
:1034E000922F9095907F892B85BB089508958091A8
:1034F0007A0220917B02821719F48FEF9FEF0895D3
:10350000E22FFF27E658FD4F8281482F5527822F53
:103510008F5F80937B02883010F010927B02CA018B
:1035200008950895CF93C82F1CC080914606882324
:1035300039F580E00E94261D2FEF8F3F920719F08A
:10354000682F80E009C081E00E94261D2FEF8F3F89
:10355000920721F0682F81E00E94074C0E940564C9
:10356000A89580914506282F3327809146069927F4
:10357000019728173907E9F2809145068F30A9F2A3
:10358000F89480914506E82FFF27EB5BF94FC28343
:10359000809145068F5F8093450680914506803176
:1035A00010F0109245067894CF9108951F93182F2C
:1035B00080E80E94921A812F0E94921A1F9108950A
:1035C0008295880F880F807C860F80680E94D61AAB
:1035D00008950E94E01A8EE00E94D61A08958CE0A9
:1035E0000E94D61A0895FF920F931F93CF93F82E3F
:1035F00060916806809167060E94E01AC0E007E5C6
:1036000016E080916906C81778F4FF2021F0F801D0
:1036100061918F0101C060E282E00E94371CCF5FA0
:1036200080916906C81788F3CF911F910F91FF9081
:1036300008959093720680937106892B89F1709397
:10364000700660936F06CB01AA27BB272091410625
:10365000309142064091430650914406280F391F8D
:103660004A1F5B1F20936B0630936C0640936D06D8
:1036700050936E0680916A068E7F80936A062115AC
:1036800031054105510561F42F5F3F4F4F4F5F4FAB
:1036900020936B0630936C0640936D0650936E0634
:1036A00008950895AF92BF92CF92DF92EF92FF926A
:1036B0000F931F93CF93DF93D82EC62EEA0187E591
:1036C000E82E86E0F82E109272061092710681E0C4
:1036D0008D1568F1EFE0E61750F14115510539F10C
:1036E000FA0101900020E9F731970E2F041B0131F8
:1036F00008F000E16C2D8D2D0E94E01A5701002387
:1037000061F0102F8881F50181935F018991682F05
:1037100082E00E94371C1150A9F7F701D08AC18AB4
:10372000028B64EF71E083EF9AE10E94191BDF9135
:10373000CF911F910F91FF90EF90DF90CF90BF90AE
:10374000AF900895CF93DF93CDB7DEB7A0970FB6B4
:10375000F894DEBF0FBECDBF282FDE01119690E09A
:10376000FA014F5F5F4F8491882321F08D939F5F13
:103770009F31B0F31C92AE014F5F5F4F822F0E94CA
:10378000521BA0960FB6F894DEBF0FBECDBFDF91DF
:10379000CF9108958091710690917206892BA9F1BD
:1037A00060916B0670916C0680916D0690916E062B
:1037B0000E94ED16882349F180916A06E091710616
:1037C000F09172068170099580916A0691E08927CF
:1037D00080936A0680916F06909170069C01442741
:1037E00055278091410690914206A0914306B091E1
:1037F0004406820F931FA41FB51F80936B069093FE
:103800006C06A0936D06B0936E060895089510920D
:1038100072061092710681E00E94D61A08950F93E5
:103820001F93CF93DF93EB018830B8F4992723E0FF
:10383000880F991F2A95E1F780640E94D61A07E045
:1038400010E0FE01219684910E94921A01501040CE
:1038500017FFF7CF8FEF0E94D61ADF91CF911F91FC
:103860000F910895813308F080E381BF0895CF93CD
:10387000C62F99278130910509F461C082309105E6
:1038800024F4892B09F457C05DC0029709F05AC08F
:1038900067FF4DC00E94532FFC0187A18823C1F010
:1038A000C43E11F4C4E843C0C63F11F4C4E93FC0AC
:1038B000CC3F11F4C1E83BC0C43C11F4CEE837C0A2
:1038C000C63D11F4C9E933C0CC3D49F5CAE92FC062
:1038D000C43E11F4C1EE2BC0C63F11F4CFEE27C099
:1038E000CC3F11F4C5EF23C0C43C39F469E771E063
:1038F00084E00E940F1CC4E01AC0C63D39F461E7A1
:1039000071E085E00E940F1CC5E011C0CC3D39F488
:1039100069E671E086E00E940F1CC6E008C0CF3D5A
:1039200031F461E671E087E00E940F1CC7E08C2F44
:103930000E94921A07C0862F0E944B1303C0862F45
:103940000E94D214CF9108951F93CF93DF93182F25
:10395000EB01FB016491662349F0812F0E94371C23
:103960002196FE018491682F8823B9F7DF91CF91CA
:103970001F9108951F93CF93DF93182FEB01888138
:10398000882341F08991682F812F0E94371C8881FC
:103990008823C1F7DF91CF911F9108951F93CF9393
:1039A000DF93CDB7DEB7C055D0400FB6F894DEBF79
:1039B0000FBECDBF67961FAD679769968EAD9FAD61
:1039C0006997AE01475A5F4FBC01CE0101960E9434
:1039D0001A7DBE016F5F7F4F812F0E94BA1CC05BB2
:1039E000DF4F0FB6F894DEBF0FBECDBFDF91CF9192
:1039F0001F9108951F93CF93DF93CDB7DEB7C055C6
:103A0000D0400FB6F894DEBF0FBECDBF67961FAD96
:103A1000679769968EAD9FAD6997AE01475A5F4F24
:103A2000BC01CE0101960E94437DBE016F5F7F4FB6
:103A3000812F0E94BA1CC05BDF4F0FB6F894DEBF27
:103A40000FBECDBFDF91CF911F910895992781308F
:103A5000910571F0823091051CF4892B31F00BC077
:103A6000029749F40E94771A08950E9479130895E5
:103A70000E94081508958FEF9FEF08950895FC01A7
:103A80008F3F910519F010F0E0E0F0E0EF57FD4FA7
:103A900084919927089590E08F3010F08EE001C056
:103AA00081118F5F442311F028E001C0242F772774
:103AB0006230710581F06330710524F46130710565
:103AC00041F00EC06330710541F06430710539F08A
:103AD00007C0236005C0246003C0266001C02760C2
:103AE000281729F4442311F02AE001C025E043E01F
:103AF00050E0990F990F80FD926020FD91608695AE
:103B000026954150504057FFF4CF892F99270895AB
:103B1000982F21E080E067FD282F6F706F3010F044
:103B200061E002C061116F5F913061F423E030E029
:103B3000880F880F60FD836066952150304037FF05
:103B4000F7CF1BC0222331F0683010F045E007C0EA
:103B50004DE005C0683010F44AE001C042E023E0C7
:103B600030E0880F880F60FD826040FD81606695BF
:103B700046952150304037FFF4CF992708959C0196
:103B8000FB018038910528F48F77808388E090E0EE
:103B90000895832F9927806C8183208380E190E0B2
:103BA00008950895FA019C01285F3F4FC90143E041
:103BB000969587954A95E1F78F7380688183C9014F
:103BC0008095909535E0969587953A95E1F7982FF1
:103BD00090779068822F8770982B9083662311F0DE
:103BE00098609083808191E08927808380E190E0D4
:103BF0000895FC014081242F332781819927019763
:103C00002817390729F04F3031F48181882319F4BE
:103C100081E090E0089580E090E0089508951F937A
:103C200083E796E00E94F91D182F85EE96E00E942A
:103C3000F91D182B812F99271F910895AF92BF92DC
:103C4000CF92DF92EF920F931F93CF93DF93EC010C
:103C50006B015A01122F8091D502882369F40C3030
:103C600059F00D3049F0CB010E94BB2C992783708D
:103C70009070892B09F48BC08091D5028823A9F517
:103C8000013099F58981282F3327888199272817B2
:103C9000390759F1AC01F90183E0EE0FFF1F8A9556
:103CA000E1F7E21BF30BEC0FFD1F828193818C1572
:103CB0009D0589F4848195818A159B0561F486812F
:103CC000813049F48085882331F08E1509F45FC076
:103CD000E08617835CC02F5F3F4F2031310514F021
:103CE00020E030E024173507B1F6CE010E94F91D1F
:103CF000282F882319F080E090E04BC08881992715
:103D0000FC01B3E0EE0FFF1FBA95E1F7E81BF90BDA
:103D1000EC0FFD1FC282D38288819927FC01A3E0AA
:103D2000EE0FFF1FAA95E1F7E81BF90BEC0FFD1F43
:103D3000A482B58288819927FC0173E0EE0FFF1FF2
:103D40007A95E1F7E81BF90BEC0FFD1F17838881CB
:103D50009927FC0163E0EE0FFF1F6A95E1F7E81B6E
:103D6000F90BEC0FFD1F068388819927FC0153E0B6
:103D7000EE0FFF1F5A95E1F7E81BF90BEC0FFD1F43
:103D8000E08688818F5F8883803108F0288381E016
:103D900090E0DF91CF911F910F91EF90DF90CF9046
:103DA000BF90AF9008959F92AF92BF92CF92DF9253
:103DB000EF92FF920F931F93CF93DF93EC015B0180
:103DC0006A01922EF02E1E2D892B31F485EE96E09D
:103DD0000E94D31EC3E7D6E08091D502882321F04C
:103DE00086E0C53ED80709F10E947110282F3327BD
:103DF00028303105D0F481E001C0880F2A95EAF718
:103E00008C7999F0F894E12E0F2D292DA601B5019A
:103E1000CE010E941E1E7894882329F485E090E04C
:103E20000E942817E1CF1092D802DF91CF911F9105
:103E30000F91FF90EF90DF90CF90BF90AF909F9049
:103E40000895CF92DF92EF920F93CF93DF936C019F
:103E5000E62E0E94842BEC01892BE9F088859927B6
:103E600083709070039711F423E001C026E001E015
:103E700040E050E0B60183E796E00E94D31E8885BB
:103E8000833049F4EE2400E121E040E050E0BA0143
:103E9000CA010E94D31E81E090E0DF91CF910F9183
:103EA000EF90DF90CF900895EF920F93CF93DF9331
:103EB000EC01E62E0E94842B892B49F008E126E0D4
:103EC00040E050E0BE0183E796E00E94D31E81E00F
:103ED00090E0DF91CF910F91EF900895EF920F93C3
:103EE000CF93DF93EC010E94842BFC01892BA9F076
:103EF0008085837081509681823028F49078E92EF5
:103F000003E02BE004C09078E92E03E024E040E0D9
:103F100050E0BE01CA010E94D31E81E090E0DF9113
:103F2000CF910F91EF900895EF920F93CF93DF937E
:103F3000EC010E94842BFC01892B19F18085282F2C
:103F400033272370307021303105DCF02330310508
:103F50007CF023303105A9F40E944A2F0E9789F492
:103F6000EE2400E121E040E050E0BA01CA0107C0C0
:103F7000EE2402E027E040E050E0BE01CA010E94CA
:103F8000D31E81E090E0DF91CF910F91EF900895E3
:103F9000EF920F93CF93DF93EC010E94842BFC01EF
:103FA000892B79F08085992783709070019749F467
:103FB000EE240BE024E040E050E0BE01CA010E9484
:103FC000D31E81E090E0DF91CF910F91EF900895A3
:103FD000AF92BF92CF92DF92EF920F93CF93DF9386
:103FE0005C016B010E94842BEC01892B09F45FC0FA
:103FF00088859927837090708230910569F5D7FE86
:1040000005C06E81888199810E94211FC0FE09C070
:10401000EE8007E024E040E050E0B501CA010E94D4
:10402000D31EC1FE09C0EE8008E024E040E050E06D
:10403000B501CA010E94D31EC2FE09C0EE8009E08C
:1040400024E040E050E0B501CA010E94D31EC3FE47
:104050002EC0EE800AE024C0039749F5C6018F7098
:104060009078892B49F0EE2404E0202F40E050E0C6
:10407000B501CA010E94D31E8C2D807F49F0EE2429
:1040800005E024E040E050E0B501CA010E94D31EE3
:1040900080E09FE0C822D922CD2849F0EE2406E036
:1040A00024E040E050E0B501CA010E94D31E81E047
:1040B00090E0DF91CF910F91EF90DF90CF90BF9084
:1040C000AF900895EF920F931F93CF93DF93EC017E
:1040D000162F0E94BB2C83708150823050F4EE2446
:1040E00002E0212F40E050E0BE0183E796E00E940D
:1040F000D31E81E090E0DF91CF911F910F91EF905F
:10410000089520E030E080915B07833011F421E0D6
:1041100030E0C90108951F93CF93DF93EC01162F70
:104120000E948120882319F480E090E012C0D0938F
:104130005807C0935707112311F08DE001C08CE0A0
:104140008093590783E080935A0710925B0781E0C0
:1041500090E0DF91CF911F910895EF920F93FC01B2
:10416000242F662311F00FE001C00EE0EE2440E0A2
:1041700050E0BF01CA010E94D31E81E090E00F9180
:10418000EF900895EF920F93EE2400E1282F40E086
:1041900050E0BA01CA010E94D31E81E090E00F9165
:1041A000EF900895EF920F93FC018091D502882340
:1041B00019F480E090E013C06770862F806F44236D
:1041C00011F0862F886FE82E03E121E040E050E0F7
:1041D000BF0183E796E00E94D31E81E090E00F913B
:1041E000EF900895EF920F93FC018091D502882300
:1041F00019F480E090E013C06770862F806E44232E
:1042000011F0862F886EE82E03E121E040E050E0B7
:10421000BF0183E796E00E94D31E81E090E00F91FA
:10422000EF900895EF920F93FC01E62E8091D50256
:10423000882319F480E090E00BC004E121E040E025
:1042400050E0BF0183E796E00E94D31E81E090E03A
:104250000F91EF900895EF920F93FC01E62E80915D
:10426000D502882319F480E090E00BC005E121E03D
:1042700040E050E0BF0183E796E00E94D31E81E05A
:1042800090E00F91EF900895EF920F93FC01E62ECE
:104290008091D502882319F480E090E00BC001E101
:1042A00021E040E050E0BF0183E796E00E94D31E8A
:1042B00081E090E00F91EF900895EF920F93FC0151
:1042C000E62E8091D502882319F480E090E00BC09F
:1042D00002E121E040E050E0BF0183E796E00E9468
:1042E000D31E81E090E00F91EF900895EF920F932D
:1042F000FC01E22E662311F007E101C006E124E093
:10430000BF0180E090E00E94D31E81E090E00F9119
:10431000EF900895982F882391F010927406809161
:1043200074068093730681E08093D7028091D70250
:104330008093D502BD9A87B7846087BF089587B7F9
:104340008B7F87BF9093D502BD98C5980895089537
:10435000EF920F93E090D502EE2069F5882359F192
:10436000E0927406809174068093730689E1E3EA13
:10437000F2E011928A95E9F700E122E040E050E096
:10438000BA0183E796E00E94D31E81E08093D702B2
:104390008BE390E099BD88BD88B599B59BBD8ABD7A
:1043A00087E790E097BD86BD1DBC1CBC87B78460C5
:1043B00087BFBE9A05C0BE98C69887B78B7F87BF58
:1043C0000F91EF900895EF920F93E090D502EE20B9
:1043D00071F5882361F1E092E6068091E60680930C
:1043E000E50689E1ECEBF2E011928A95E9F700E14C
:1043F00022E040E050E0BA0185EE96E00E94D31E34
:104400008BE390E0909387008093860087E790E0AD
:104410009093810080938000109289001092880010
:1044200080917D00846080937D00139A07C013986B
:104430001B9880917D008B7F80937D000F91EF9082
:10444000089583E080935B071092600710926107E4
:104450001092620710926307809160079091610744
:10446000A0916207B091630780935C0790935D070A
:10447000A0935E07B0935F0780E00E948A2181E0ED
:104480000E94A82181E00E94E32180916200846063
:1044900080936200089580E00E948A2180916200EA
:1044A0008B7F8093620080E00E94A82180E00E94C0
:1044B000E3211092D70281E00E94C577089580E041
:1044C0000E94A82180E00E94E32181E00E94C5773C
:1044D000809162008B7F8093620089E1E3EAF2E0E1
:1044E00011928A95E9F783E08093B5028FEF80936C
:1044F000A3028BE390E099BD88BD88B599B59BBDBB
:104500008ABD87E790E097BD86BD81E00E948A2141
:1045100082E090E00E94351908950E942F61FC010D
:10452000808182FF02C0C79A0895C79808950895B0
:104530000E942F61FC01808182FF07C080E090E033
:10454000B79907C081E090E0089586B399278078F5
:104550009070089508950E947110282F33272830F5
:10456000310558F481E001C0880F2A95EAF788796F
:1045700021F08091D8029927089581E090E0089574
:1045800008958091D602992708951092D602089531
:104590009093ED028093EC0208958091EA0290914D
:1045A000EB02089580E1E9EDF2E011928A95E9F7D6
:1045B0001092E9021092EB021092EA028FEF9FE74D
:1045C0009093ED028093EC02089578941F920F92DD
:1045D0000FB60F9211242F933F934F938F939F9376
:1045E000EF93FF938091E902883010F01092E90276
:1045F0008091E902E82FFF27EE0FFF1FE752FD4FE2
:1046000024B135B1208331838F5F8093E90210920A
:10461000EB021092EA0220E030E047E0E9EDF2E040
:1046200081919191280F391F415047FFF9CF309365
:10463000EB022093EA028091EC029091ED02821746
:1046400093071CF481E08093D602FF91EF919F9134
:104650008F914F913F912F910F900FBE0F901F9010
:1046600018953F924F925F926F927F928F929F9296
:10467000AF92BF92CF92DF92EF92FF920F931F9370
:10468000CF93DF935C016B016624362C655E764028
:1046900011F461E0662EF60190818181981709F08E
:1046A00082C0662019F481E08093D8028091D502FF
:1046B000882339F0E32C0EE021E040E050E0BA011D
:1046C0006FC0662019F00E94A12C02C00E943A2CF3
:1046D000EC01009731F4EE2401E022E0AC01BC01D2
:1046E0005FC088859927837090708230910561F052
:1046F000833091051CF4019721F055C00397A9F16F
:1047000052C0EE8001E027C01E81E12E01E022E0D0
:1047100040E050E068817981C6010E941E1E0E941F
:10472000362C8370482F55274130510591F0423087
:10473000510524F44115510541F035C04230510571
:1047400071F04330510571F02EC0E12E07E022E0F8
:1047500025C0E12E08E022E040E050E01FC0E12E3D
:1047600009E0F9CFE12E0AE0F6CFEE8001E0202F3C
:1047700040E050E068817981C6010E941E1E0E94BF
:10478000362C9927AC014170507080FF04C0EE2494
:1047900004E021E0E1CFEE2405E021E068817981A9
:1047A000C6010E941E1EF60181819927FC0153E07B
:1047B000EE0FFF1F5A95E1F7E81BF90BEC0DFD1DFD
:1047C00082809380F60181819927FC0143E0EE0FFE
:1047D000FF1F4A95E1F7E81BF90BEC0DFD1D448026
:1047E0005580F60181819927FC0133E0EE0FFF1F10
:1047F0003A95E1F7E81BF90BEC0DFD1DF680F6018B
:1048000081819927FC0123E0EE0FFF1F2A95E1F734
:10481000E81BF90BEC0DFD1D7084F60181819927D1
:10482000FC0103E0EE0FFF1F0A95E1F7E81BF90B0F
:10483000EC0DFD1D878181508783882309F0E5C039
:1048400080915C0790915D07A0915E07B0915F0732
:104850000097A105B105C9F080915C0790915D07B3
:10486000A0915E07B0915F078896A11DB11DBC01A4
:10487000CD010E94ED16882341F010925C07109242
:104880005D0710925E0710925F078091600790911C
:104890006107A0916207B09163070097A105B10578
:1048A000C9F08091600790916107A0916207B09173
:1048B00063078896A11DB11DBC01CD010E94ED16B4
:1048C000882341F0109260071092610710926207EE
:1048D00010926307662039F580915B0780FD7FC0E9
:1048E00080915C0790915D07A0915E07B0915F0792
:1048F0000097A105B10509F072C080915B07816046
:1049000080935B078091410690914206A0914306F7
:10491000B091440680935C0790935D07A0935E0777
:10492000B0935F0728C080915B0781FD22C0809112
:10493000600790916107A0916207B09163070097AB
:10494000A105B105B1F480915B07826080935B079C
:104950008091410690914206A0914306B091440691
:104960008093600790936107A0936207B0936307F9
:1049700002C03320A1F1F60181819927FC0113E0E7
:10498000EE0FFF1F1A95E1F7E81BF90BEC0DFD1D6B
:10499000809157079091580782839383F601818114
:1049A0009927FC01C3E0EE0FFF1FCA95E1F7E81B52
:1049B000F90BEC0DFD1D809159078683F60181816D
:1049C0009927FC01B3E0EE0FFF1FBA95E1F7E81B52
:1049D000F90BEC0DFD1D80915A07878316C0F60177
:1049E00081819927FC01A3E0EE0FFF1FAA95E1F753
:1049F000E81BF90BEC0DFD1D3682F60181818F5FFE
:104A000081838181803108F011828F2D8C5082301A
:104A100008F05AC0662049F1809141069091420603
:104A2000A0914306B091440680936007909361077C
:104A3000A0936207B093630780916007909161072C
:104A4000A0916207B09163070097A105B105A9F590
:104A500081E090E0A0E0B0E0809360079093610770
:104A6000A0936207B093630728C08091410690919C
:104A70004206A0914306B091440680935C07909350
:104A80005D07A0935E07B0935F0780915C079091EC
:104A90005D07A0915E07B0915F070097A105B10582
:104AA00061F481E090E0A0E0B0E080935C07909337
:104AB0005D07A0935E07B0935F07C4010E94307644
:104AC000082FC0E0D0E007C0E090D502EE2029F02A
:104AD000C0E0D0E003E010E018C0C4010E94842BC5
:104AE000EC01009721F0172D088503700CC0F5012B
:104AF000E0821E2D4C01F0E1FF1611F403E003C02B
:104B0000E1E0FE2E0F2D61101078802F9927813063
:104B100091050CF420C28330910524F0039709F429
:104B2000DCC019C2C4010E943F1D982F8295869552
:104B300086958370F5018283292F220F220F21830E
:104B400071E0E72EE28A82E1808B82E0818B209700
:104B500039F18C819D8197FF02C023602183812FD1
:104B600099278F779070892BD9F088850E944A2FDA
:104B70000F97B4F01F5F88850E94322A892B31F489
:104B800010FF04C0F50181818E258183212F2078BB
:104B9000812F99278F71907095958795122F182BDB
:104BA0008F2D99278830910509F46AC089309105C5
:104BB0009CF48430910544F4823091050CF04FC090
:104BC000019709F447C0C7C18430910509F442C078
:104BD000079709F450C0BFC18B30910509F463C039
:104BE0008C30910544F48930910509F452C00A973C
:104BF00009F454C0B0C18E3091051CF0489751F1B2
:104C0000AAC1C40153E0969587955A95E1F7907033
:104C100001960E943F1D982F8295869586958370F8
:104C2000F5018283990F990F9183F7E08F229924E0
:104C300089E792E0880E991EF4018491F501808342
:104C4000FCE0FF1619F48C7FF501808382E0F5010A
:104C5000828B0EC0612F802F0E94881D3BC08E81E9
:104C600080788F60682F802F0E94881DF5018083D7
:104C700084E0818B70C18C818170482F61E004C019
:104C80008C818270482F62E0812F8F770E944B1DAC
:104C900021C08C818470482F63E0F6CF8C818870AE
:104CA000482F64E0F1CFC4010E943F1D982F8295E8
:104CB000869586958370F5018283990F990F93608D
:104CC000918382E0828BEC81FD81EF70F070E75977
:104CD000FD4F8491F50180833EC183E0F501828B15
:104CE00061E0618B88E1808B8F2D99278031910560
:104CF000ECF48E3091050CF0C1C08530910509F4BB
:104D0000A5C08630910554F48330910551F184306B
:104D100091050CF085C0019729F10DC186309105F0
:104D200009F4A1C00C970CF406C10FC0863191059F
:104D300044F4843191050CF0D1C0409709F4ACC023
:104D4000B0C048970CF0F7C0DCC0A5014F5F5F4FC3
:104D500060E0FDE0FF1609F461E0C4010E94D21D8D
:104D6000EAC01F67888599278C7090700897C9F4EE
:104D70008FE3F5018283812F99278F7790700097B9
:104D800031F08F37910511F4117801C01F5FF501E3
:104D90001183C5010396BC01C4010E94BF1D885E3A
:104DA000C8C017FF02C080E601C080E4F50181831E
:104DB00088850E944A2F212F3327A5014E5F5F4F20
:104DC0000F97BCF0C9018F779070009731F08F3743
:104DD000910511F412E001C01D5F812F86958F703F
:104DE000F5019181982B918310FF54C090619183BC
:104DF00051C0C9018F779070009731F08F379105BE
:104E000011F411E001C01F5F1F70F5012181212BFA
:104E100021838C819D8197FF3DC0206121833AC011
:104E200080E8F50181832C812F70822F8068818337
:104E30008C819D8197FF02C020692183C501029664
:104E4000BC01C4010E94BF1D805F73C080EAF501F0
:104E500081838C819D8144E0969587954A95E1F701
:104E60008F70806B09C080EAF50181838C819D8100
:104E7000892F99278F70806A8183E0CFF501118295
:104E8000A5014E5F5F4FFFE0FF1621F4C4010E94B1
:104E9000D21DDACFBA01D5CF8FEFF501828311820F
:104EA0004AC0F3E1FF1611F488E709C0F2E1FF16EA
:104EB00011F484E704C0F1E1FF1619F48CE7F50161
:104EC0008383892D9927982F9370F5018381892BEE
:104ED00083838282718280E2808B10C080E7F5013B
:104EE0008283F4E1FF1619F488E7F5018283882DA7
:104EF0008770F5019281982B928371828AE0818B71
:104F00001AC0852D992783708C6EF50183834282A8
:104F10007182A5014C5F5F4FF7E1FF1629F461E054
:104F2000C4010E94D21D04C0BA01C4010E94BF1D69
:104F3000805EF501808B20E0F5019089969596952D
:104F40009695915031F0F501E90FF11D80812827E8
:104F5000F8CFF5012083F5018289833011F010929A
:104F6000D702DF91CF911F910F91FF90EF90DF90CB
:104F7000CF90BF90AF909F908F907F906F905F90F9
:104F80004F903F900895CF93DF93DC01FC0184891B
:104F9000882319F42589222361F021E0882321F058
:104FA0008150FD01848B21C0FD0185898150858B55
:104FB0001CC0FD018289833019F487898823A9F4F4
:104FC000FD019389892F869586958695E80FF11DB9
:104FD0008081282F3327892F99278770907002C0EE
:104FE000359527958A95E2F72170FD013289832F47
:104FF00099278230910531F083309105CCF00397E9
:1050000021F016C0CBE6D0E015C0222319F0C7E787
:10501000D0E002C0CEECD0E0FD018389882351F4BA
:105020008689882339F482E0858B81E0868B2BC0CA
:10503000C7EDD0E0FD018389882329F58589882380
:1050400011F58189882399F48091D7028823D9F4B6
:105050008091D5028823B9F481E00E9450618823B1
:1050600019F0C35BDF4E0FC0CD5ED94F0CC0832F4C
:1050700099278130910529F0029729F4C857DD4F0F
:1050800002C0C05FDA4FCE01DF91CF910895DC01FD
:10509000FC018489882319F48589882311F021E093
:1050A0002BC0FD013389932F9150938B82898330DC
:1050B00069F42789222351F4892F992787709070EA
:1050C000079721F481E0878B338B16C0FD01178A87
:1050D0009389892F869586958695E80FF11D8081A5
:1050E000282F3327892F99278770907002C0359514
:1050F00027958A95E2F72170FD01828999278230F0
:10510000910549F0833091051CF4019761F01BC0B3
:10511000039789F018C0222319F08CE590E00895D8
:1051200080E190E00895222319F08EEB90E008953D
:105130008CE190E00895222319F08BE390E008952C
:1051400087E690E008958BE390E008950895FC01D0
:105150008089838B8189823010F482E0818B8289FF
:10516000992781309105B4F0833091051CF00397A5
:1051700061F010C081E00E945061882319F08DE435
:1051800090E1089583E196E0089580E1848B82E3C5
:1051900090E0089582E390E0089508951F920F92A1
:1051A0000FB60F9211241F932F933F934F935F934A
:1051B0006F937F938F939F93AF93BF93CF93DF931F
:1051C000EF93FF93C3EAD2E08091D502882331F0B8
:1051D0000E94C122882311F01092B4028091BB0278
:1051E0008823A1F08091D702882329F08BE390E0F7
:1051F00099BD88BD02C019BC18BC8BE390E09BBD73
:105200008ABD87E790E097BD86BD5CC083EA92E0E7
:105210000E94C327AC019C01255030408CB59DB540
:105220008217930718F457BD46BD0FC08CB59DB5C6
:10523000C29697BD86BD83EA92E00E94A7282CB54E
:105240003DB5280F391F37BD26BD8091B602882392
:1052500071F51091B802112351F58091B4028823A1
:1052600071F481E0888F86B7846086BF789463E7A5
:1052700076E083EA92E00E943123F894188E8091C0
:10528000B4028150898B8091B3028B8B8091B502DF
:10529000833049F48091D502882311F084E101C064
:1052A00080E18C8B01C01C8B1D8A1F8A1E8A83EAB9
:1052B00092E00E94472899279BBD8ABD8AB59BB57D
:1052C00099BD88BDFF91EF91DF91CF91BF91AF91D3
:1052D0009F918F917F916F915F914F913F912F910E
:1052E0001F910F900FBE0F901F9018951F920F9255
:1052F0000FB60F9211241F932F933F934F935F93F9
:105300006F937F938F939F93AF93BF93CF93DF93CD
:10531000EF93FF93CCEBD2E08091D4028823B1F0DD
:105320008091D702882339F08BE390E09093870037
:105330008093860004C0109287001092860087E751
:1053400090E0909381008093800060C0CE010E9425
:10535000C327AC019C01255030408091880090917A
:1053600089008217930728F45093810040938000AE
:1053700016C08091880090918900C2969093810018
:1053800080938000CE010E94A72820918800309150
:105390008900280F391F309381002093800080916D
:1053A000CF02882351F51091D102112331F580915C
:1053B000CD02882381F481E0888F80917C00846015
:1053C00080937C00789465EE76E08CEB92E00E940E
:1053D0003123F894188E8091CD028150898B809171
:1053E000CC028B8B8091CE02833019F480E18C8BC0
:1053F00001C01C8B1D8A1F8A1E8A8CEB92E00E94C2
:10540000472899279093870080938600FF91EF911A
:10541000DF91CF91BF91AF919F918F917F916F91CC
:105420005F914F913F912F911F910F900FBE0F9061
:105430001F90189580E892E0E4E6F7E0119201975A
:10544000E9F71092EF021092EE021092E40908952B
:105450008F7020E030E08950823010F421E030E09D
:10546000C90108958F7020E030E08550823010F43B
:1054700021E030E0C9010895BF92CF92DF92EF9210
:10548000FF920F931F93CF93DF93CDB7DEB7239790
:105490000FB6F894DEBF0FBECDBF7C01B62E8FEFE6
:1054A000C82ED82E00E210E0A89543E050E0B801E5
:1054B000CE0101960E945D7829813A812E153F0523
:1054C000A9F0D7FE05C088E22030380708F068014F
:1054D0000C5F1F4F8FE00C3D180730F32E153F0572
:1054E00039F0D7FE05C08FEF9FEF19C06801F6CFE6
:1054F0008B818B1519F42E153F0579F0BB82E9825B
:10550000FA82A89544E050E0B601CE0101960E94CF
:1055100079786B2DC7010E940C6E80E090E0239695
:105520000FB6F894DEBF0FBECDBFDF91CF911F91B4
:105530000F91FF90EF90DF90CF90BF900895BF92B2
:10554000CF92DF92EF92FF920F931F93CF93DF934F
:10555000CDB7DEB723970FB6F894DEBF0FBECDBF31
:105560008C01B62E009711F4FC0127C0CC24DD2459
:1055700090E2E92EF12CA89543E050E0B701CE016E
:1055800001960E945D7869817A81CB0101978F5FD6
:10559000974248F420E030E04B818B2DF8010995CB
:1055A0000894C11CD11C84E090E0E80EF91E9CED2B
:1055B000E9169FE0F906F8F2F601CF0123960FB63F
:1055C000F894DEBF0FBECDBFDF91CF911F910F9139
:1055D000FF90EF90DF90CF90BF900895EF92FF92F1
:1055E0000F931F93CF93DF93CDB7DEB723970FB6FB
:1055F000F894DEBF0FBECDBF8C010097C1F1FC0156
:105600008081918101978F5F9742E0F420E2E22E42
:10561000F12CA89543E050E0B701CE0101960E941D
:105620005D7829813A81F8018081918128173907B5
:10563000C9F084E090E0E80EF91E9CEDE9169FE0C9
:10564000F90638F3F801808191818F3F910519F0B7
:1056500010F087E00BC088E00E945061882321F0A1
:1056600087E003C08B8101C082E0F8018087239628
:105670000FB6F894DEBF0FBECDBFDF91CF911F9163
:105680000F91FF90EF9008950F931F93CF93DF93A7
:10569000CDB7DEB727970FB6F894DEBF0FBECDBFEC
:1056A0008FEF9FEFAFEFBFEF8C839D83AE83BF8300
:1056B00000E210E043E050E0B801CE0101960E9404
:1056C0005D7889819A818F5F9F4F19F48B818F3F1D
:1056D00041F044E050E0B801CE01840F951F0E94D4
:1056E00079780E9475100C5F1F4F8FE00C3D1807F2
:1056F00008F327960FB6F894DEBF0FBECDBFDF913B
:10570000CF911F910F910895CF93DF93EC010E94E9
:105710007110873019F481EF92E026C0209749F488
:10572000CE0122C08AE0689FC00111248C59984F95
:105730001BC060E07091E4096717A0F420E030E03E
:10574000A901F901E40FF51FEC59F84F808191810F
:105750008C179D0739F36F5F4F5F5F4F275F3F4F98
:10576000671778F380E090E0DF91CF910895FF9282
:105770000F931F93CF93DF938C01F62E0E9471102D
:105780008730E9F48091F1029091F202801791073D
:1057900099F01093F2020093F10281EF92E00E94DF
:1057A000EE2A8091F90299278370907001970297F1
:1057B00018F082E08093F90281EF92E04DC0C801B9
:1057C00001978F5F974290F5C8010E94842BEC01EE
:1057D000892B09F040C02091E409203450F48AE07C
:1057E000289FE0011124CC59D84F2F5F2093E40962
:1057F00020C0C4E6D7E0BE0120E030E0A901AFE35D
:10580000F901E40FF51FEC59F84F91858985891747
:1058100008F4EB01A1504F5F5F4F275F3F4F665F7A
:105820007F4FA7FFEDCF8985882319F480E090E0B2
:1058300013C008831983CE010E94EE2A80E88E836C
:105840001C821D821A821B8219861F82FF2019F07A
:10585000C8010E94D06FCE01DF91CF911F910F91AF
:10586000FF90089561E00E94B72B08958091F002A7
:1058700099270895EF92FF921F93CF93DF930E9491
:105880007110873041F4C1EFD2E08091F0028F5F58
:105890008093F0021DC09091E409992319F480E0EF
:1058A00090E049C08091EE028F5F8093EE028917ED
:1058B00038F08091F0028F5F8093F0021092EE0238
:1058C0009091EE028AE0989FE0011124CC59D84FC4
:1058D0008091F002992787709070892BA9F41E811E
:1058E000E12EFF24C7018F779070892B69F088859E
:1058F0000E94322A892B41F0E0FC06C01F5F612F15
:10590000888199810E94541F8091F00299278770A5
:105910009070049751F4888599278370907001974F
:1059200021F4888199810E94C81F89858F3F11F0D9
:105930008F5F8987CE01DF91CF911F91FF90EF900C
:1059400008959091E409992319F480E090E0089576
:105950008091EF028F5F8093EF02891710F0109211
:10596000EF029091EF028AE0989FC00111248C59B8
:10597000984F089508950E94842BFC01009709F424
:10598000089580859927089508950E94842BFC012D
:10599000009709F4089586819927089508950E9433
:1059A000842BFC01009709F4089584819581089562
:1059B00008950F931F93CF938C01C62F0E94322C12
:1059C000FC01892B49F080858C1731F0C087118646
:1059D0006C2FC8010E943C2ACF911F910F9108950E
:1059E000CF92DF92FF920F931F93CF93DF93EC013F
:1059F000F62E142F892B09F492C0442331F00E9413
:105A00007110873011F4FE828AC0112331F08F812A
:105A100081FF03C08D7F8F8382C088850E944A2FBB
:105A2000482F5885752F73708F2D99278F77907019
:105A3000242F3327281739071CF420E8F222F42AF0
:105A40006E816F1509F46BC019868F812F2D332756
:105A5000C62EDD24112311F0816001C082608F8386
:105A600020783070C601807890702817390799F136
:105A7000C6018F779070009711F020E8F222733002
:105A8000D9F4892B29F0888199810E946E1F1FC04B
:105A9000852F99278C7090700897C9F48F2D9927BE
:105AA0008F779070892B99F48F2D8160682F888172
:105AB00099810E94211F0BC0892B49F0888199810F
:105AC0000E94211F888199810E946E1F04C08881D5
:105AD00099810E94941FFE820F2D1127C8018F7794
:105AE0009070892BB9F088850E94322A892B91F019
:105AF00000FD03C08F2D8F5F08C00894C108D10836
:105B00000C151D0539F48F2D8150682F88819981DE
:105B10000E94541F6F2D888199810E94211FDF915F
:105B2000CF911F910F91FF90DF90CF900895FF923A
:105B30000F931F93CF93DF93EC01162FF42E0E9447
:105B40007110833029F00E947110873009F01078AD
:105B5000CE010E94322CEC010E814F2D612F0E944C
:105B6000F02C8A819B810097C9F060E00E94B72BDE
:105B7000EC01892B99F08E81282F33272078307003
:105B8000802F9927807890702817390711F080E8C6
:105B900018274F2D612FCE010E94F02CDF91CF915D
:105BA0001F910F91FF900895DF92EF92FF920F9354
:105BB0001F93CF93DF93EC017B01D42E892B09F443
:105BC00050C08C819D818617970709F44AC04423F1
:105BD00039F00E947110873019F4EC82FD8241C0C7
:105BE000DD2019F08F8181FD3CC019860C811D815B
:105BF0008F819885DD2011F0816001C082608F83E4
:105C0000EC82FD82892F99278370907081309105F5
:105C100031F0813091052CF104971CF51BC09801DF
:105C200020703078C701807090782817390729F0E4
:105C30006E81888199810E94211F0F7010708FE002
:105C4000E822FF240E151F0561F0888199810E94CA
:105C5000C81F07C00E251F25B801888199810E94A1
:105C6000E81FDF91CF911F910F91FF90EF90DF9090
:105C70000895FF920F931F93CF93DF938B01F42E20
:105C80000E94322CEC01892B49F18A819B81892B5E
:105C900001F1C8018F709F7B4F2DBC01CE010E9486
:105CA000D42D8A819B810E94322CEC01892BB1F08A
:105CB000C80180709074880F991F007F107034E0C5
:105CC000169507953A95E1F7802B912B4F2DBC0146
:105CD00002C04F2DB801CE010E94D42DDF91CF918B
:105CE0001F910F91FF900895EF92FF920F931F93D2
:105CF000CF93DF938C017B0160E00E94B72BEC0116
:105D0000892B81F060E0C7010E94B72BFC01892B31
:105D100049F0EA82FB821986028313831186C80147
:105D20000E944A70DF91CF911F910F91FF90EF90E9
:105D30000895CF93DF93EC010E940471209769F0DE
:105D4000CE010E94322CFC01892B39F0C281D38113
:105D5000128213821186209799F7DF91CF910895CF
:105D60001F93CF93DF93C4E6D7E01FE38A819B8123
:105D7000892B21F0888199810E94992E11502A96B1
:105D800017FFF4CFDF91CF911F910895EF92FF920B
:105D90000F931F93CF93DF93CDB7DEB726970FB640
:105DA000F894DEBF0FBECDBF7C010E94711087301A
:105DB00009F1C7010E94842B8C01892BD9F0B7010E
:105DC000CE0101960E946C63F80144815581668181
:105DD000CE0101960E944F63AE014F5F5F4F6AE0B4
:105DE0008FEF0E94EF63F801448155816681C701FE
:105DF0000E94BB2F26960FB6F894DEBF0FBECDBF14
:105E0000DF91CF911F910F91FF90EF9008951F9315
:105E1000CF93DF9310E0C4E6D7E09091E40919171F
:105E2000F0F48985899FC00111248035910534F0F3
:105E30008E8199278F779070892B59F08E81807889
:105E40008E83888199810E946E1F888199810E942A
:105E5000C62E1F5F2A969091E409191710F3DF915F
:105E6000CF911F910895FF920F931F938C01F62EEF
:105E7000C8010E94762184E00E94C22041E06F2D7B
:105E8000C8010E94AD208AE00E94C2201F910F919C
:105E9000FF900895E82FFF27EF70F070E752FC4F56
:105EA0008491992708958BEF92E0089580910F03D4
:105EB00082FF05C08091FD029091FE0208958091BD
:105EC000FB029091FC020895089580910F03826077
:105ED00080930F0308950F931F93CF93DF93CBEF1E
:105EE000D2E080910F0399278C010170107080FF20
:105EF00003C080E090E021C060910303709104032F
:105F00008091050390910603611571058105910546
:105F100031F00E94ED16882311F4C8010EC01A82D8
:105F20001B82188E198E1092FC021092FB021C8AA2
:105F30001A8E0E942C1081E090E0DF91CF911F918A
:105F40000F9108959C018091FD029091FE02892B92
:105F500011F4C90108952F703F7B77FD3064CB01A8
:105F60008F70907044E0880F991F4A95E1F7822B5B
:105F7000932B08950895FC018091FB029091FC02FF
:105F80002091FD023091FE02E817F907F9F46093C1
:105F90001103232BB1F08091010390910203F4E0EF
:105FA00096958795FA95E1F7BC016F707070892F0F
:105FB00099278695869580FD7068CA010E94A22F58
:105FC00011C0509302034093010310C0E217F3077E
:105FD00079F460931103BA01809101039091020357
:105FE0000E94A22F90930203809301030E942C1021
:105FF000089508959C01892B69F410920F03109263
:1060000003031092040310920503109206030E94EA
:106010006B2F089560931103509302034093010383
:106020008091410690914206A0914306B0914406AA
:1060300088519C4FAF4FBF4F816080930303909373
:106040000403A0930503B093060380910F0382FF1E
:1060500010C081608B7F80930F033093FE022093EA
:10606000FD02B9018091FB029091FC020E94742E06
:1060700007C08E7F80930F033093FC022093FB02B6
:106080000E942C100895089520910F032B7F21600A
:1060900020930F039093FE028093FD0280910103F1
:1060A000909102030E94A22F909302038093010318
:1060B0000E942C100895CF93DF93EB01809310037F
:1060C0000E944A2F80931203209759F045E153E034
:1060D00060E070E0CE010E94866DD0931403C093FF
:1060E00013030E942C10DF91CF910895CF93C82FF6
:1060F000882319F069EF71E002C069E172E084E081
:106100000E940F1CCC2319F061EF71E002C061E125
:1061100072E085E00E940F1CCC2319F069EE71E05B
:1061200002C069E072E086E00E940F1CCC2319F0E7
:1061300061EE71E002C061E072E087E00E940F1C36
:10614000CF910895CF93DF93C82FDD27C4FF02C0FE
:1061500083E001C085EA0E94921AC0FF02C084E079
:1061600001C085EA0E94921AC1FF02C085E001C009
:1061700085EA0E94921AC2FF02C086E001C085EA49
:106180000E94921AC3FF02C087E001C085EA0E9404
:10619000921ADF91CF910895809321030E942C10D1
:1061A0000895882319F061EC71E002C069EC71E098
:1061B00082E00E940F1C08950895882319F061ED74
:1061C00071E002C069ED71E081E00E940F1C08954A
:1061D00008950F931F93CF930BEF12E0C09121030B
:1061E000CC2399F060E081E00E94E01A8C2F81506E
:1061F0000E945260BC0182E00E94A41C1092210304
:1062000088EE93E00E94351902C0882319F00E949D
:10621000071C03C0682F0E94E01A8091FB02909136
:10622000FC02892BF9F00E942F61FC01828193818D
:106230004091FB025091FC028417950749F4218597
:10624000328580911303909114032817390751F078
:106250004283538380911303909114038187928723
:106260000E94B6602091FB023091FC02211531059D
:1062700029F4F80126833783168A158A80910F0343
:1062800082FD0DC080910B0390910C03A0910D0332
:10629000B0910E030097A105B10519F105C069EE93
:1062A00073E082E00E94A41C80910B0390910C0388
:1062B000A0910D03B0910E03BF93AF939F938F9363
:1062C0008CEE93E09F938F9382E08F930E94FA1C51
:1062D0008DB79EB707960FB6F8949EBF0FBE8DBFC1
:1062E00042C02115310531F46FEF73E082E00E9466
:1062F000A41C18C03F932F9386E094E09F938F9344
:10630000C2E0CF930E94FA1C80910F030F900F9070
:106310000F900F900F9080FF02C08C2F01C080E281
:106320000E94921AC09110030E947110863008F0EA
:106330008150833061F48C2F99278370907023E013
:10634000880F991F2A95E1F78F579C4F08C099270E
:1063500003E0880F991F0A95E1F78F559C4FBC0108
:1063600082E00E94A41C6CE080E00E94E01A809110
:10637000110399278F7790709F938F938BE094E010
:106380009F938F9382E08F930E94FA1C8091100359
:106390009927837090700F900F900F900F900F902F
:1063A000019779F487E10E94B119882331F080E0E8
:1063B0000E94921A69E871E010C080E20E94921A6D
:1063C0000FC080E00E94921A8091110387FF03C0E2
:1063D00061E672E002C069E572E080E00E940F1C95
:1063E0000E947110C82F813049F489E00E941D601D
:1063F000AC0160E08C2F0E94A21BECC040E050E09A
:1064000060E0862F0E94521BC0E08AE00E94B11912
:10641000882371F08091FD029091FE02892B39F45E
:1064200080911003992783709070039709F4C1E05D
:1064300060E081E00E94E01A80910B0390910C03D0
:10644000A0910D03B0910E030097A105B10509F4C9
:1064500042C08DE00E94B119882329F48EE00E9489
:10646000B119882381F18FE094E09F938F93C2E06C
:10647000CF930E94FA1C8DE00E94B1190F900F90EB
:106480000F90882379F061ED71E081E00E940F1C8C
:1064900069EC71E08C2F0E940F1C6CE271E08DEDB5
:1064A00090E30EC069ED71E081E00E940F1C61EC89
:1064B00071E08C2F0E940F1C6CE271E081ED90E383
:1064C0000E94191B87C087E00E941D60BC0182E00A
:1064D0000E94A41C44C08091FD029091FE0200978E
:1064E00069F19F938F938BE194E09F938F9382E068
:1064F0008F930E94FA1C809101039091020314E093
:10650000969587951A95E1F7282F2F70892F99274F
:10651000869586950F900F900F900F900F9080FDAD
:106520002061822F0E94A230CC2321F08CE30E94B4
:10653000921A15C080E20E94921A13C085E193E07E
:106540009F938F9380E294E09F938F9382E08F9349
:106550000E94FA1C0F900F900F900F900F90CC2379
:1065600061F48091070390910803A0910903B09111
:106570000A030097A105B105C9F08091FD02909131
:10658000FE02892B99F48091010390910203A4E00B
:1065900096958795AA95E1F78F7080610E94A23049
:1065A00081E00E94763061E272E011C02091010327
:1065B0002F70809101039091020397FD2061822F3B
:1065C0000E94A23080E00E94763069E272E083E0AF
:1065D0000E940F1CCF911F910F910895CF93DF93CD
:1065E000EC01288939894A895B896A817B81211577
:1065F00031054105510509F46BC061157105E1F0E4
:10660000E881F981CF01AA27BB2782179307A40746
:10661000B50741F0CB01AA27BB2782179307A40730
:10662000B50751F48C898E7F8C8BCF010E94992EF7
:106630001A821B8218821982888199819C014427C1
:10664000552788899989AA89BB896C8928173907B0
:106650004A075B0729F481E068276B7F6C8B3DC09C
:106660006C7F6C8B188E198E1A8E6A8D81E00E9459
:10667000E01A80E00E941D60BC0182E00E94A41C20
:106680008C89992796958795969587959C01217079
:10669000307080FD13C088819981009711F08C8340
:1066A0009D832A833B832E833F83288339831D8ADE
:1066B000688979898FEF0E94AA6207C04889598941
:1066C000688179818FEF0E94C6628C898B7F04C0BC
:1066D000672B19F48C8984608C8B188A198A1A8A22
:1066E0001B8ADF91CF910895609103037091040399
:1066F000809105039091060361157105810591054F
:1067000061F00E94ED16882341F01092030310926D
:106710000403109205031092060360910703709121
:1067200008038091090390910A03611571058105A1
:10673000910571F00E94ED16882351F01092070325
:10674000109208031092090310920A030E942C1061
:1067500008950895CF92DF92FF920F931F93CF93E6
:10676000DF93EC01FBEFCF2EF2E0DF2E85319105B8
:10677000CCF48F3091050CF03DC18A30910509F4BD
:10678000F7C18B30910534F4009709F48FC197FD60
:10679000FEC1B9C18C30910509F4CFC00D970CF042
:1067A000EBC0E1C18B3191057CF4893191050CF589
:1067B0008631910509F455C1863191050CF468C103
:1067C000479709F4A7C0E3C18F3891056CF48D3861
:1067D00091050CF0D1C08132910509F43AC18A3893
:1067E000910509F4D2C1D3C18739910509F4CDC10E
:1067F000CEC1FF24499711F4E1E0FE2EC0911103B0
:10680000109112030E942F61FC010781FF20B1F05B
:106810000E9471104C2F5527833041F49A012F7735
:106820003070812F99272817390714F09A016FC00B
:106830001E3711F4002371F4CF5F24C02C2F3327AF
:10684000C9018F779070892B09F461C01E37C9F494
:106850000023B9F02C2FFF2051F0023041F48C2F8F
:1068600099278F779070449714F42F5F4FC0FF20C3
:1068700061F4023051F48C2F99278F7790704597EF
:106880004CF4C1502C2F332742C0013019F42C2F67
:106890002E7F14C08C2F99278F779070459714F016
:1068A0002C2F2E7F422F5527CA018F779070CF97BC
:1068B0002CF04E5350404C7F242F225C2C1761F05B
:1068C000FF2021F10230F9F4822F99278F77907001
:1068D000CE97CCF02E5F17C0FF2049F0023039F47C
:1068E000822F99278F779070CE970CF02E5FFF2024
:1068F00051F4023051F4822F99278F779070CF97FF
:1069000024F0225002C02E5F01C022503327F6012E
:10691000268B3BC18091100399278370907001975B
:1069200029F469E871E080E00E940F1C8091110356
:10693000809580788093110328C18AE00E94B11964
:10694000882399F08091FD029091FE02892B69F0D5
:10695000809101039091020320E030E48227932785
:10696000909302038093010310C1809101039091E1
:10697000020320E030E867C080910B0390910C0384
:10698000A0910D03B0910E030097A105B10581F10F
:1069900020910B0330910C0321503040220F331F04
:1069A000CE018F7790700E9709F42160C7FF1AC04F
:1069B00041E060E0C9010E94CE7560E070E0CB016B
:1069C0000E94191B69E372E081E00E940F1C61E4E0
:1069D00072E082E00E940F1CF601108A118A128A6E
:1069E000138AD3C041E0642FC9010E94CE75CDC087
:1069F000C7FDCBC0C131D1058CF08091410690918B
:106A00004206A0914306B09144068C509E4FAF4F72
:106A1000BF4FF60184879587A687B7871C2F1D5027
:106A20008AE00E94B119882319F061970CF41C5F69
:106A300021E030E002C0220F331F1A95E2F7809167
:106A400001039091020382279327F601868397839F
:106A50009CC06CE38091FB029091FC020E9462203A
:106A600094C0F89483E00E943010882319F084E0E9
:106A70000E94C57787E10E94B119882339F06BE441
:106A80008091FB029091FC020E94622078947DC06C
:106A90008AE00E94B119811182E00E94301088239F
:106AA00009F473C084E00E94C5776FC08AE00E9439
:106AB000B1198823A9F08091FF02909100030097FB
:106AC00009F465C0AA27BB2780930B0390930C039E
:106AD000A0930D03B0930E03C6010E94EE3257C07F
:106AE00080910B0390910C03A0910D03B0910E03C4
:106AF0000097A105B10539F48FEF0E94BE5F81E0D8
:106B00000E94E93044C080910B0390910C03A09146
:106B10000D03B0910E039C01AD0163E0220F331F02
:106B2000441F551F6A95D1F7280F391F4A1F5B1F55
:106B3000280F391F4A1F5B1FCE01AA2797FDA0957A
:106B4000BA2F280F391F4A1F5B1F2030F8E23F077A
:106B5000F0E04F07F0E05F07D4F4F601208B318BB3
:106B6000428B538B12C08BEF92E00E94EE320DC02D
:106B700010920B0310920C0310920D0310920E034F
:106B800080910F038B7F80930F030E942C10DF9165
:106B9000CF911F910F91FF90DF90CF900895FC014E
:106BA000EC5BFF4F8081E454F040882319F480E0CF
:106BB00090E00895E95BFF4F8081E754F04088231F
:106BC00029F48481883511F0883719F481E090E048
:106BD000089580E090E008950895CF93DF93EC014D
:106BE0000E94CF35882319F480E090E01FC0FE0199
:106BF000E95BFF4F8081882351F4CC5BDF4F8881B4
:106C0000C454D040823018F481E090E00FC08081FD
:106C1000882311F08C8101C08D81992787FD909583
:106C2000809590958827990F881F9927DF91CF919C
:106C30000895CF93C82FCF7719F480E090E029C052
:106C4000862F0E944A2F282F33272B31310589F0B8
:106C50002C31310524F42E30310529F017C02C31A8
:106C6000310569F013C0EC2FFF27EE59FB4F8491DB
:106C70000BC0EC2FFF27EA5BFB4F849105C0EC2F84
:106C8000FF27E75DFB4F8491992703C0CF5F8C2FCF
:106C90009927CF910895CF93C82FCF7719F480E02B
:106CA00090E02EC0C150862F0E944A2F282F3327F4
:106CB0002B31310579F02C31310524F42E3031059A
:106CC00029F01CC02C31310569F018C08C2F992790
:106CD00008960DC083E0C89FC00111240B966EE09A
:106CE00070E007C08C2F9927880F991F079669E0DD
:106CF00070E00E94D57DCB01992702C08C2F992787
:106D0000CF910895019791F40E942F61FC01818138
:106D1000882311F484E608C0843011F485E604C0A9
:106D20008150843008F08150992708958FEF9FEFAC
:106D3000089508951F93CF93C82FFB01142F8181CD
:106D4000282F332782819927982F8827282B392BA2
:106D5000C90101978F5F974210F062E010C01123C4
:106D600021F0C9010E94322C03C0C9010E94842B6A
:106D7000009751F4112311F06BE001C06AE08C2FF1
:106D80000E94371C80E090E0CF911F910895EF9210
:106D9000FF920F931F93CF93DF93EB01E42E41E01B
:106DA0000E949A368C01892B19F48FEF90E066C00F
:106DB0000E940F1E882319F088E090E05FC0FB80DE
:106DC000EE2051F021E0F21639F4F82EF80180811E
:106DD00091810E946E1F08C0EE2031F0F80160859D
:106DE0008B810E944B36F82E6C81862F992785FF68
:106DF00002C0F0E8FF2AF801C481D581DF7784FD65
:106E0000D06867FF05C0C07F8F709070C82BD92BEA
:106E10002F2D332720783070F8016681862F99272F
:106E2000807890702817390731F0607840E08081D1
:106E300091810E94972D40E06F2DF8018081918112
:106E40000E94972D40E0BE01F801808191810E944F
:106E5000392EF801808191810E94C62E0E94711006
:106E6000833011F0873019F480E090E007C0823061
:106E700019F481E490E002C082E490E0DF91CF91C8
:106E80001F910F91FF90EF90089541E00E94C73647
:106E90009927089540E00E94C736992708951F93C7
:106EA000CF93DF93182F41E0812F0E949A36EC0197
:106EB000892BF1F060E0812F0E94371C68858E815C
:106EC0000E941936682F812F0E94371C6C816F70C9
:106ED0008C819D8197FD60618E8187FD6062812F2D
:106EE0000E94371C8E818F77682F812F0E94371C5C
:106EF0008FEF90E0DF91CF911F9108951F93CF9373
:106F0000DF93182F41E0812F0E949A36EC01892BE4
:106F100001F160E0812F0E94371C88858370682F03
:106F2000812F0E94371C88850E94282A892B11F006
:106F30006CE104C088850E944A2F682F812F0E942F
:106F4000371C6FEF812F0E94371C6FEF812F0E943B
:106F5000371C8FEF90E0DF91CF911F910895CF9371
:106F6000DF93EB0141E00E949A36FC01892B19F472
:106F70008FEF90E03BC08B8199278230910559F0CB
:106F8000833091051CF4019721F026C0039729F066
:106F900023C021E003C022E001C023E0822F992713
:106FA00081309105E4F0833091051CF0039749F09E
:106FB00016C06C816E3099F06B3141F06C3151F03C
:106FC0000BC06C816E3059F06C3111F4246007C035
:106FD0006E3711F4286003C082E090E007C0622F92
:106FE000808191810E94D92C80E090E0DF91CF9147
:106FF00008950F931F93CF93DF938B0141E00E947D
:107000009A36EC01892B19F48FEF90E014C08C8133
:107010009D818070F80123813327822B932B40E0E0
:10702000BC01888199810E94392E888199810E94B2
:10703000C62E80E090E0DF91CF911F910F910895CF
:107040000F931F93CF93DF938B0141E00E949A36F9
:10705000EC01892B19F48FEF90E018C02C813D8151
:10706000307CF801838199278F739070982F88273F
:10707000282B392B40E0B901888199810E94392E53
:10708000888199810E94C62E80E090E0DF91CF91A7
:107090001F910F9108951F93CF93DF93182F41E015
:1070A000812F0E949A36EC01892B41F060E0812FFC
:1070B0000E94371C6C81812F0E94371C8FEF90E05B
:1070C000DF91CF911F9108951F93CF93DF93182FD6
:1070D00041E0812F0E949A36EC01892B69F060E033
:1070E000812F0E94371C8C819D81892F99278F7356
:1070F000682F812F0E94371C8FEF90E0DF91CF9196
:107100001F910895DF92EF92FF920F931F93CF93F9
:10711000DF93982F8B01823008F059C088E4989F44
:107120007001112483E293E0E80EF91EFB018181D6
:10713000C82FDD278281992787709070982F882724
:10714000C82BD92B2197F7E0C83FDF0718F082E062
:1071500090E03FC00E947110982F8250823028F03A
:10716000973019F086E090E034C0CC0FDD1FF801B5
:10717000628167FFC160862F9927E6E09695879523
:10718000EA95E1F771E0D72ED82287010B5B1F4FFC
:10719000F80180819181FFEF8F3F9F0749F040E028
:1071A000642F0E94CE758FEF9FEFF801808391834B
:1071B00040E06D2DCE010E94CE75882319F489E040
:1071C00090E007C0DD2019F0F801C083D18380E092
:1071D00090E0DF91CF911F910F91FF90EF90DF90A2
:1071E0000895FF920F931F93CF93F82EFB01818197
:1071F000082F11278281992787709070982F8827F0
:10720000082B192B87E0083F180718F082E090E060
:107210001CC0C8010E942474873611F0873411F411
:10722000C4E001C0C0E0C801880F991F0E943076F9
:10723000039709F4C16060E08F2D0E94371C6C2F0A
:107240008F2D0E94371C8FEF90E0CF911F910F91EF
:10725000FF9008951F93CF93182FFB01C181CC237A
:1072600019F482E090E00FC060E00E94371CEC2F20
:10727000FF27EA55F54F80818095682F812F0E9466
:10728000371C8FEF90E0CF911F9108951F93CF93FC
:10729000182FFB01C181C150C03218F082E090E08C
:1072A00015C060E00E94371C60E08C2F0E94D16AFC
:1072B000682F812F0E94371C61E08C2F0E94D16AB9
:1072C000682F812F0E94371C8FEF90E0CF911F9184
:1072D00008950E94EC6A80E090E008951F93CF9398
:1072E000182FFB0181819927009719F0039729F046
:1072F00008C0C091E509CC0F07C0C091E609C17074
:1073000003C082E090E00AC060E0812F0E94371C39
:107310006C2F812F0E94371C8FEF90E0CF911F912F
:107320000895FB0181819281282F33272115310592
:1073300021F02330310559F014C0913490F4892F95
:1073400099270196959587958093E5090DC08091C1
:10735000E609992311F0816001C08E7F8093E609D0
:1073600003C082E090E0089580E090E008950895E1
:10737000EF92FF920F931F93CF93DF93CDB7DEB7BA
:1073800060970FB6F894DEBF0FBECDBFF82E63E056
:107390000E94371C61E08F2D0E94371C64E08F2D06
:1073A0000E94371C64E08F2D0E94371C64E08F2DF3
:1073B0000E94371C0E946C61DC01CB01BF93AF932C
:1073C0009F938F9381E794E09F938F938E010F5F3C
:1073D0001F4F1F930F930E949D788DB79EB70896FD
:1073E0000FB6F8949EBF0FBE8DBF33E0E32EF801B9
:1073F00091919295907F81918F018053982B692F65
:107400008F2D0E94371CEA94E7FEF1CF80E090E0D8
:1074100060960FB6F894DEBF0FBECDBFDF91CF915F
:107420001F910F91FF90EF9008951F93CF93182F06
:10743000C0E00E947110833021F0873011F082305B
:1074400009F4C8E0823009F4C0616C2F812F0E94DA
:10745000371C8FEF90E0CF911F9108951F93CF932A
:10746000DF93182FFB018181282F332782819927F1
:10747000982F8827822B932B0E948236EC0197FF4E
:1074800003C082E090E00AC060E0812F0E94371CB8
:107490006C2F812F0E94371C8FEF90E0DF91CF91EE
:1074A0001F91089560E00E94371C82E00E94301016
:1074B0008FEF90E0089580E00E94301080E090E02F
:1074C000089583E00E94301080E090E0089580E00D
:1074D00090E008951F93CF93DF93182F0E94607759
:1074E000EC0160E084E0989F812D9927112480FDB4
:1074F00061E0CE01892F992782958695877080FD5E
:107500006460C0FD6860D7FD6062CE7FDF71209748
:1075100009F06068812F0E94371C209791F060E08D
:10752000C1FD61E0C2FD6064C97F209709F0606819
:10753000812F0E94371CCD2B21F060E0812F0E940B
:10754000371C8FEF90E0DF91CF911F9108950F933B
:107550001F93CF93DF93182FC4E6D7E000E080910C
:10756000E409081778F58F8180FF29C068858E812E
:107570000E941936682F812F0E94371C6C81812F41
:107580000E94371C6881812F0E94371C8881998155
:10759000892F9927682F6F738C819D8197FD606477
:1075A0008E8187FD6068812F0E94371C8E818F77C6
:1075B000682F812F0E94371C8F818E7F8F830F5FF2
:1075C0002A96CDCF80E890E0DF91CF911F910F9167
:1075D00008956F927F928F929F92AF92BF92CF92B7
:1075E000DF92EF92FF920F931F93CF93DF93CDB76C
:1075F000DEB7C254D0400FB6F894DEBF0FBECDBF89
:10760000882E01E010E0AA249A2CB1E0BB2E7E0166
:10761000E00EF11E3701C92CDD24F601E955F44FC7
:10762000E081EE2319F4095F1F4F2CC0EB2141F1DB
:10763000F70101937F01812F992787708083C8010B
:1076400001970E942474982F873411F0873621F413
:10765000F701808180688083973411F0923521F49E
:10766000F7018081806480830894E11CF11CA3945D
:10767000F601E955F44F9B2D9095808189238083F5
:10768000BB0C19F49394F1E0BF2E0F5F1F4FF7E08E
:10769000093F1F0720F48FE18A1508F0BCCF6A2D3F
:1076A000882D0E94371CDD2473010A2D1127011536
:1076B000110581F0F70181917F01682F882D0E94CB
:1076C000371CD3942D2D3327C801800F911F281705
:1076D000390784F38FEF90E0CE5BDF4F0FB6F8945D
:1076E000DEBF0FBECDBFDF91CF911F910F91FF90F5
:1076F000EF90DF90CF90BF90AF909F908F907F9052
:107700006F900895CF92DF92EF92FF920F931F93A5
:10771000CF93DF93D82ECC248091E509882309F4F8
:1077200054C0F8948C2D992787FD9095880F991F48
:107730009C012959354F8C01095D154FEC01C95148
:10774000D64F4881942F9095D8018C918923F901C7
:10775000E080E82A5981952F9095F801818189234D
:10776000F901F180F82A2E2D332727FD3095842F3B
:1077700099272817390749F42F2D332727FD3095EE
:10778000852F99272817390799F08C2D8F5F682F3F
:107790008D2D0E94371C6E2D8D2D0E94371C6F2D54
:1077A0008D2D0E94371CE882F982F8011182108227
:1077B0007894C3942C2D332727FD30958091E509CB
:1077C0009927281739070CF4ACCF60E08D2D0E9463
:1077D000371C8FEF90E0DF91CF911F910F91FF90B9
:1077E000EF90DF90CF9008951F93CF93C82F162F5F
:1077F000603418F067E774E002C061E874E08C2F31
:107800000E94A41C812F99278A30910589F18B3021
:1078100091057CF48630910511F1873091051CF4B7
:107820000297D1F039C088309105F9F00997D1F06D
:1078300033C08E30910529F18F30910534F48B30AF
:107840009105C9F00D97D1F027C081349105E1F081
:1078500082349105E1F020C069E874E01AC06DE956
:1078600074E017C06AEA74E014C06DEB74E011C0F4
:1078700060ED74E00EC068ED74E00BC06AEE74E079
:1078800008C063EF74E005C06AE075E002C065E11E
:1078900075E08C2F0E94A41C103420F06DE08C2F1A
:1078A0000E94371C81E090E0CF911F910895282F0E
:1078B000862F992785309105A9F1863091058CF4A2
:1078C0008230910531F1833091052CF40097D9F085
:1078D0000197E1F03BC083309105F1F00497F9F096
:1078E00035C08830910539F18930910534F48630FE
:1078F0009105D9F00797E1F029C089309105F1F0A1
:107900004097F9F023C060E275E01DC063E275E0C6
:107910001AC069E275E017C06DE275E014C060E35B
:1079200075E011C066E375E00EC06DE375E00BC055
:1079300068E475E008C06FE475E005C067E575E0D0
:1079400002C066E675E0822F0E94A41C81E090E0F0
:1079500008953F924F925F926F927F928F929F9283
:10796000AF92BF92CF92DF92EF92FF920F931F934D
:10797000CF93DF93CDB7DEB722970FB6F894DEBF73
:107980000FBECDBF89839A83332486E9E3EBF3E00E
:1079900011928A95E9F705C00894411C511C49824F
:1079A0005A8249805A80F2019081992391F09C3249
:1079B00081F0943271F0953261F0892F80538A30D2
:1079C00040F0892F992787FD90950E94067E892B8C
:1079D00019F3F2018081882309F4BDC004C00F5F50
:1079E0001F4F09831A8309811A81F801D0808D2DD8
:1079F000992787FD90950E94067E892B81F7DD20CF
:107A000009F4ABC0FCE2DF1609F497C08FE0389EA2
:107A10007001112483EB93E0E80EF91E82E0682EDA
:107A2000712C6E0C7F1CCC2497E2D91619F0E2E27F
:107A3000DE1629F40F5F1F4F09831A83CD2CA9800E
:107A4000BA80450183010E191F090250104008C079
:107A50000894811C911CF301D1923F010F5F1F4FCD
:107A60000B301105ACF4F401D080DD2089F0CC207E
:107A700011F0DC1469F7CC2059F4FCE2DF1641F078
:107A80008D2D992787FD90950E94067E892B01F305
:107A9000F3011082F5018081843239F4C501019629
:107AA00089839A8340E150E008C0853251F4C501D2
:107AB000019689839A8342E050E0BE016F5F7F4F59
:107AC00006C04AE050E0BE016F5F7F4FC5010E94D3
:107AD0000879DC01CB01F7018083918381E0F70114
:107AE000868704C00F5F1F4F09831A8309811A819B
:107AF000F801F080FF2081F08F2D992787FD909568
:107B00000E94067E892B41F4FCE2FF1659F704C05F
:107B10000F5F1F4F09831A8309811A81F801F080D2
:107B2000FF2041F08F2D992787FD90950E94067EBA
:107B3000892B71F7FCE2FF1621F40F5F1F4F0983B9
:107B40001A833394E981FA818081882321F089E0C6
:107B5000831508F048CFF2011082832D99272296D1
:107B60000FB6F894DEBF0FBECDBFDF91CF911F914E
:107B70000F91FF90EF90DF90CF90BF90AF909F90CC
:107B80008F907F906F905F904F903F9008950F93EC
:107B90001F93D8018A30C0F48617B0F49927FC01EE
:107BA00064E0EE0FFF1F6A95E1F7E81BF90BED5457
:107BB000FC4F8685882341F0008111810417150749
:107BC00018F02017310708F48D01C8011F910F919B
:107BD0000895CF93DF93EC01009719F48FEF90E0B5
:107BE0001CC06EE675E00E94DB78892B11F481E001
:107BF00013C062E775E0CE010E94DB78892B11F497
:107C000082E00AC066E775E0CE010E94DB78892B2E
:107C100011F483E001C08FEF9927DF91CF91089590
:107C20000F931F93CF93C82F8B016115710549F1F5
:107C30008F3F39F1C370CB010E9428788F3708F04D
:107C40008EE72C2F332721303105F4F02330310516
:107C500024F02330310559F017C08B3181F462E4F0
:107C600070E0C8010E94CE78892B39F402C08C31B3
:107C700011F4C46009C08E3711F4C86005C08E309D
:107C800019F08FEF90E002C08C2F9927CF911F91B0
:107C90000F9108956AE775E00E94A41C81E090E0CE
:107CA000089561EB75E00E94A41C81E090E00895C6
:107CB0006EEC75E00E94A41C81E090E008951F9393
:107CC000182F67E076E00E94A41C61E276E0812F25
:107CD0000E94A41C60E476E0812F0E94A41C81E035
:107CE00090E01F910895CF93C82F0E94711099279B
:107CF00084309105D9F0853091054CF4823091059E
:107D000079F0833091057CF4892B39F01AC08730E3
:107D1000910594F0079769F014C06DE576E00EC008
:107D200065E676E00BC06DE676E008C064E776E0D5
:107D300005C060E876E002C06CE876E08C2F0E9417
:107D4000A41C81E090E0CF910895EF92FF920F93F1
:107D50001F93182F7B01042F80E00E943010402FCA
:107D6000B701812F0E94733E99271F910F91FF90B9
:107D7000EF900895EF92FF920F931F93182F7B01BE
:107D8000042F83E00E943010402FB701812F0E9402
:107D9000733E99271F910F91FF90EF90089562E92C
:107DA00076E00E94A41C82E00E94301080E090E007
:107DB00008950F931F93CF93C82F762F642F00E061
:107DC00010E0A801872F0E94C73D8C01892B21F468
:107DD00062E08C2F0E94F43BC801CF911F910F915C
:107DE0000895EF92FF920F931F93CF93DF93082F85
:107DF0007B01EA012223A9F0122F60E2802F0E946A
:107E0000371CC7018C239D23892B11F061E301C02E
:107E100060E3802F0E94371C1150CC0FDD1F11230F
:107E200061F7DF91CF911F910F91FF90EF9008952F
:107E30008F929F92AF92BF92CF92DF92EF92FF927A
:107E40000F931F93CF93DF93882E5B017A01922EBD
:107E5000C02EEB01DD24DC14F8F4C7018095909569
:107E6000C823D92300E010E0C5018E219F21892B72
:107E700011F001E010E021E030E040E050E0682D3A
:107E80008D2D890D0E94C73D892B11F0CE29DF2948
:107E9000D394EE0CFF1CDFCFCE01DF91CF911F9169
:107EA0000F91FF90EF90DF90CF90BF90AF909F9099
:107EB0008F9008959F92AF92BF92CF92DF92EF92F0
:107EC000FF920F931F93CF93DF93982EB42E2FEF33
:107ED00037E260E00E94D93E6C01009719F481E01E
:107EE00090E0EAC00E94842B7C01892B69F421E098
:107EF0002B1510F06AE012C0C6010E94322C7C01E2
:107F0000892B11F46BE00AC031E03B1508F085C005
:107F10000E940F1EA82E882331F068E0892D0E9450
:107F2000F43B9927C9C0F70184819581EC01DF7783
:107F3000892F992787FD90958827990F881F992762
:107F40008C0121E030E040E050E06B2D82E00E94A7
:107F5000C73D892B09F0D06804E0202F41E050E0B4
:107F6000BE018B2D0E94183F4A2DBC01C6010E9404
:107F7000392EF701608586810E94193699278C0178
:107F80002FE730E040E050E06B2D81E00E94C73DDC
:107F9000C82F8091E203863411F411E015C08235B8
:107FA00011F41A2D11C000E010E0F701868187FF5F
:107FB00002C001E010E021E030E040E050E06B2D35
:107FC00083E00E94C73D182FC13029F4C0E0C601EC
:107FD0000E946E1F06C0F70160858C2F0E944B36F1
:107FE000C82F1111C0682C2F332720783070F7016B
:107FF0006681862F9927807890702817390729F095
:10800000607840E0C6010E94972D40E06C2FC601C9
:108010000E94972DC6010E94C62E0E9471108230C8
:1080200011F461E405C00E947110833021F062E414
:10803000892D0E94F43BF701868187FF03C086E605
:1080400090E002C082E790E09F938F93F7018581D3
:10805000282F332727FD3095209530952227330F81
:10806000221F332781E390E0821B930B9F938F9312
:10807000608586810E94193699279F938F93DF929E
:10808000CF928CE996E09F938F939F920E94FA1C67
:1080900024E041E050E0F70164817581892D0E9460
:1080A000F13E81E090E02DB73EB7255F3F4F0FB620
:1080B000F8943EBF0FBE2DBFDF91CF911F910F915E
:1080C000FF90EF90DF90CF90BF90AF909F9008957A
:1080D000CF93C82F2FEF37E260E08C2F0E94D93E5C
:1080E000009719F10E94842BFC01892B19F46AEA8C
:1080F00076E018C080859927837090708230910552
:1081000061F0833091051CF4019721F00EC00397B4
:1081100039F00BC061EB76E005C06EEB76E002C093
:108120006BEC76E08C2F0E94A41C81E090E0CF9154
:108130000895CF92DF92EF92FF920F931F93CF9308
:10814000DF93182FD42E2FEF37E260E00E94D93E44
:10815000EC01009719F481E090E053C00E94842B59
:108160007C01892B69F481E08D1510F06AE011C063
:10817000CE010E94322C7C01892B11F46BE009C0E6
:10818000E1E0ED15E8F40E940F1EC82E882331F0BF
:1081900068E0812F0E94F43B992733C008E021E07A
:1081A00041E050E0F701648175818D2D0E94183FF8
:1081B0004C2DBC01CE010E94392ECE010E94C62E4C
:1081C0000E947110882321F462E4812F0E94F43B05
:1081D000DF93CF938FEC96E09F938F931F930E9432
:1081E000FA1C28E041E050E0F70164817581812F9D
:1081F0000E94F13E81E090E00F900F900F900F9061
:108200000F90DF91CF911F910F91FF90EF90DF9032
:10821000CF900895CF92DF92EF92FF920F931F932A
:10822000CF93DF93182FD42E2FEF37E260E00E9418
:10823000D93EEC01009719F481E090E053C00E9410
:10824000842B7C01892B69F481E08D1510F06AE0A4
:1082500011C0CE010E94322C7C01892B11F46BE0FD
:1082600009C0E1E0ED15E8F40E940F1EC82E882336
:1082700031F068E0812F0E94F43B992733C006E07B
:1082800021E040E051E0F701648175818D2D0E946D
:10829000183F4C2DBC01CE010E94392ECE010E9408
:1082A000C62E0E947110882321F462E4812F0E945F
:1082B000F43BDF93CF9384ED96E09F938F931F93CE
:1082C0000E94FA1C26E040E051E0F70164817581CC
:1082D000812F0E94F13E81E090E00F900F900F906F
:1082E0000F900F90DF91CF911F910F91FF90EF9022
:1082F000DF90CF900895AF92BF92CF92DF92EF922E
:10830000FF920F931F93CF93DF93A82EC42F0E9449
:108310007110882311F466E05DC028EF37E04C2F20
:1083200060E08A2D0E94D93E6C01892B19F021E072
:108330002A1518F481E090E083C088E4A89EC0016B
:1083400011248D5D9C4FC23008F44EC025E4E22E0E
:10835000F12CE80EF91EF70180819181FFEF8F3F2C
:108360009F0749F040E0642F0E94CE758FEF9FEF8A
:10837000F701808391838091C403873411F4BB2477
:1083800010C0823519F491E0B92E0BC002E010E064
:1083900021E030E040E050E06C2F81E00E94C73DDA
:1083A000B82E00E010E021E030E0A8016C2F82E060
:1083B0000E94C73DEC01860101501040000F111FC3
:1083C0000B0D111D40E06C2FC8010E94CE75882353
:1083D00031F469E08A2D0E94F43B992731C0CC2307
:1083E00019F0F70100831183C60101970E942474DC
:1083F000C0E0D0E0082F112707FD1095C8010E94AA
:10840000FC7D892B11F0C1E0D0E0DF93CF93C80150
:108410000E940F7E9F938F93DF92CF928AED96E01A
:108420009F938F93AF920E94FA1C81E090E02DB74A
:108430003EB7275F3F4F0FB6F8943EBF0FBE2DBF2C
:10844000DF91CF911F910F91FF90EF90DF90CF9030
:10845000BF90AF9008951F93182F65EE76E00E94AD
:10846000A41C62EF76E0812F0E94A41C0E946C6124
:10847000DC01CB01BF93AF939F938F9388EF96E07E
:108480009F938F931F930E94FA1C8DB79EB70796F8
:108490000FB6F8949EBF0FBE8DBF81E090E01F9194
:1084A0000895EF92FF920F931F93CF93DF93E82EDF
:1084B000F42E0E942F61EC01FF20E1F08B859927BB
:1084C0008C0124E130E040E050E06F2D80E00E941C
:1084D000C73D8B878C859927880F991F8C012EEFBC
:1084E00031E042E050E06F2D81E00E94C73D96955B
:1084F00087958C878C859927880F991F9F938F93D9
:108500008B8599279F938F9385E097E09F938F9317
:10851000EF920E94FA1C8DB79EB707960FB6F8949B
:108520009EBF0FBE8DBF81E090E0DF91CF911F9184
:108530000F91FF90EF9008950F931F93CF93C82F43
:10854000642F442379F08091E60999278170907017
:108550008C0121E030E040E050E080E00E94C73D27
:108560000E94E16A8091E6099927817090709F933B
:108570008F938EE097E09F938F93CF930E94FA1C86
:108580000F900F900F900F900F9081E090E0CF919F
:108590001F910F910895DF92EF92FF920F931F9317
:1085A000CF93E82E842F00E010E020E230E041E09D
:1085B00050E0682F80E00E94C73DC82F882309F44F
:1085C00047C099279F938F9384E197E09F938F9360
:1085D000EF920E94FA1CDC2EDA9460E08D2D0E944E
:1085E000D16A082F112751E0F52E0F900F900F90B0
:1085F0000F900F90C7E08F2D992780239123892B0F
:1086000011F061E301C060E38E2D0E94371CC15060
:10861000FF0CC7FFF0CF60E28E2D0E94371C61E097
:108620008D2D0E94D16A082F112741E0F42EC7E05A
:108630008F2D992780239123892B11F061E301C0AD
:1086400060E38E2D0E94371CC150FF0CC7FFF0CF96
:1086500081E090E0CF911F910F91FF90EF90DF901C
:108660000895FF920F931F93F82E642F8091E509D0
:108670009927880F991F8C0120E430E040E050E0FA
:1086800080E00E94C73D8F5F86958093E50999271A
:10869000880F991F9F938F9387E397E09F938F9302
:1086A000FF920E94FA1C0F900F900F900F900F9066
:1086B00081E090E01F910F91FF900895CF93C82F14
:1086C0004423C9F4C13031F46DE377E08C2F0E946C
:1086D000A41C13C00E942D139F938F9383E497E0F3
:1086E0009F938F93CF930E94FA1C0F900F900F903F
:1086F0000F900F9002C0C13019F481E090E00DC0DE
:1087000066E477E08C2F0E94A41C8091B3039091C3
:10871000B4030E94B51280E090E0CF9108950F93CA
:108720001F93CF93C82F842F0FEF1FEF27EE33E057
:1087300040E050E0682F80E00E94C73D0E948236F2
:1087400097FF06C062E08C2F0E94F43B992711C06E
:1087500090709F938F9389E497E09F938F93CF932B
:108760000E94FA1C81E090E00F900F900F900F9004
:108770000F90CF911F910F910895EF92FF920F9359
:108780001F93982F642F4423C9F088E4989F7001A9
:10879000112483E293E0E80EF91E00E010E021E0EE
:1087A00030E0A80180E00E94C73DF701E95BFF4F80
:1087B000892B19F081E0808301C0108281E090E074
:1087C0001F910F91FF90EF900895FF920F931F93C9
:1087D000CF93C82F842F00E010E02FEF37E241E065
:1087E00050E0682F80E00E94C73D8C01009701F1A6
:1087F0000E94322CFC01892B11F46BE01AC0908589
:10880000F92E8091D003882339F084EC93E00E9404
:10881000E93D982F8F3F61F08091DF03882371F04D
:1088200063ED73E0892F0E94103E982F8F3F31F443
:1088300062E08C2F0E94F43B992708C09F1521F01D
:10884000692FC8010E94D92C81E090E0CF911F913F
:108850000F91FF900895CF92DF92EF92FF920F93C6
:108860001F93CF93DF93E82E8B01F42E6901842FA1
:108870000E944A2F9F938F931F930F938CE497E04E
:108880009F938F93EF920E94FA1C0F2D1127C8011E
:108890008370907001972DB73EB7295F3F4F0FB699
:1088A000F8943EBF0FBE2DBF029780F4E801CC7054
:1088B000D070C430D10521F461E68E2D0E94371CA2
:1088C000289721F462E68E2D0E94371C63E577E03D
:1088D0008E2D0E94A41CC801837090708230910577
:1088E00061F0833091051CF4019721F00EC00397CD
:1088F00039F00BC066E577E005C06AE577E002C0B5
:108900006EE577E08E2D0E94A41CC114D10491F075
:10891000F6018081882371F0DF92CF9282E697E0A2
:108920009F938F93EF920E94FA1C0F900F900F90DD
:108930000F900F906DE08E2D0E94371CDF91CF912C
:108940001F910F91FF90EF90DF90CF900895DF92ED
:10895000EF92FF920F931F93CF93DF93CDB7DEB7C4
:108960002D970FB6F894DEBF0FBECDBFD82E80E096
:1089700090E00E94466E8C017C01892BE1F0AE01F3
:108980004F5F5F4FBE01635F7F4FC8010E94866DDE
:10899000BC01892B81F09E012F5F3F4F4D858D2DAE
:1089A0000E942B44C8010E94466E8C018E159F05C3
:1089B00011F0892B21F72D960FB6F894DEBF0FBE6C
:1089C000CDBFDF91CF911F910F91FF90EF90DF907E
:1089D00008951F93182F0E94A74467E677E0812F20
:1089E0000E94A41C81E090E01F910895FF920F93D4
:1089F0001F93CF93DF93F82E842F00E010E02FEF2A
:108A000037E241E050E0682F80E00E94C73DEC0172
:108A1000892BA9F08091D003882389F08091DF030E
:108A2000882369F083ED93E00E94E93D8F3F39F0A0
:108A300064EC73E00E94103E182F8F3F31F462E027
:108A40008F2D0E94F43B992722C0CE010E94842BD7
:108A5000892B21F0612FCE010E94D92C612FCE01EC
:108A60000E943C2ACE010E94C66DFC018091EE035B
:108A7000882341F022EE33E0412FBE01CF010E9456
:108A8000E66C03C0CF010E94E36C81E090E0DF91CF
:108A9000CF911F910F91FF9008950E94442B02C027
:108AA0000E94E36C80E090E00E94466E0097C1F760
:108AB00081E090E00895EF92FF920F931F93CF9380
:108AC000DF93CDB7DEB766970FB6F894DEBF0FBE63
:108AD000CDBFE82ECE0101960E94F06B8D819E8164
:108AE000009709F442C020E0AE01495F5F4F60E1AA
:108AF000E4E0880F991FEA95E1F70E94CC6BFF2410
:108B000000E010E0F801EC0FFD1F21853285C9015E
:108B100001978F5F974200F53F932F93FF2019F045
:108B200088E791E002C08BE791E09F938F938DE6F9
:108B300097E09F938F93EF920E94FA1C8DB79EB798
:108B400007960FB6F8949EBF0FBE8DBFF3940E5FCD
:108B50001F4F96E09F15B0F66DE08E2D0E94371CDA
:108B60008F819885009709F0BECF66960FB6F8946E
:108B7000DEBF0FBECDBFDF91CF911F910F91FF9050
:108B8000EF9008951F93182F0E945B4562E777E0EE
:108B9000812F0E94A41C81E090E01F910895CF9244
:108BA000DF92FF920F931F93CF93C42F00E010E04A
:108BB0002FEF37E241E050E06C2F80E00E94C73D8C
:108BC0006C01892BA1F0F1E0FF2EFC1680F400E08F
:108BD00010E02FEF37E241E050E06C2F8F2D0E9424
:108BE000C73DBC01C6010E94742EF394EECF81E014
:108BF00090E0CF911F910F91FF90DF90CF9008955B
:108C00000E94B02E81E090E008951F93CF93C82F6B
:108C1000142F8C2F0E94A41C60E28C2F0E94371C02
:108C2000112319F068E777E002C06CE777E08C2F3A
:108C30000E94A41C6DE08C2F0E94371CCF911F91C5
:108C40000895AF92BF92CF92DF92EF92FF921F935F
:108C5000CF93C82F0E942F616C016FE777E08C2FB4
:108C60000E94A41C67E877E08C2F0E94A41C60E996
:108C700077E08C2F0E94A41C6DE08C2F0E94371C83
:108C80008DE090E09F938F9386E997E09F938F9379
:108C9000CF930E94FA1C0F900F900F900F900F909F
:108CA00065EA77E08C2F0E94A41C0E946C61DC01B5
:108CB000CB01BF93AF939F938F9384EB97E09F93E8
:108CC0008F93CF930E94FA1C8DB79EB707960FB66D
:108CD000F8949EBF0FBE8DBF60EC77E08C2F0E9492
:108CE000A41C6C2F8BE294E40E949F2A8C2F0E947C
:108CF000A74468EC77E08C2F0E94A41C8C2F0E9464
:108D00005B4565ED77E08C2F0E94A41CEE24FF24C8
:108D10005701C5010E943076182FFF92EF928FED18
:108D200097E09F938F93CF930E94FA1C0F900F9020
:108D30000F900F900F90113019F464EE77E002C09D
:108D400067EE77E08C2F0E94A41C6DE08C2F0E94B0
:108D5000371C0894E11CF11CE8E0F0E0AE0EBF1EE9
:108D6000FFEFEF16F104ACF26BEE77E08C2F0E9470
:108D7000A41CF60180818170482F65EF77E08C2F6D
:108D80000E940546F60180818470482F6FEF77E0DE
:108D90008C2F0E940546F60180818870482F6DE077
:108DA00078E08C2F0E940546F601868199279F93D3
:108DB0008F9388E198E09F938F93CF930E94FA1C42
:108DC0000F900F900F900F900F90F60180859927CC
:108DD0009F938F9386E298E09F938F93CF930E9407
:108DE000FA1C0F900F900F900F900F90F601938543
:108DF00082E3989FC00111249F938F9385E398E0AD
:108E00009F938F93CF930E94FA1C0F900F900F9017
:108E10000F900F90F601948584E6989FC00111246D
:108E20009F938F9384E498E09F938F93CF930E94B6
:108E3000FA1C0F900F900F900F900F90F601818108
:108E40000E94F5129F938F9383E598E09F938F93F1
:108E5000CF930E94FA1C0F900F900F900F900F90DD
:108E600060E678E08C2F0E94A41C81E090E0CF9116
:108E70001F91FF90EF90DF90CF90BF90AF9008953B
:108E8000EF92FF920F931F93CF93DF93E82EF42E70
:108E900066E678E084EC93E00E94DB78892B19F495
:108EA000C1E0D0E002C0C3E0D0E08091C1038823DC
:108EB00041F48091D003882321F0CE010E94607696
:108EC0002EC00FEF1FEF2FEF30E040E050E06F2D8E
:108ED00080E00E94C73D9C0197FF06C062E08E2D96
:108EE0000E94F43B99271DC08091D003A3E0220F7C
:108EF000331FAA95E1F7882371F4C9010E943076E7
:108F0000019719F469E678E002C06CE678E08E2DEE
:108F10000E94A41C04C0BE01C9010E94787681E0B1
:108F200090E0DF91CF911F910F91FF90EF90089506
:108F3000EF92FF920F931F93CF93DF93E82EF42EBF
:108F40000E942F61EC018091C103882369F060E7E2
:108F500078E085EB93E00E94DB782881892B11F47F
:108F60002B7F01C0246028838091D003882371F077
:108F70000FEF1FEF28EC30E040E050E06F2D81E074
:108F80000E94C73D99230CF443C08E838091DF0378
:108F9000882369F063E778E083ED93E00E94DB7853
:108FA0002881892B11F4277F01C0286028838091B4
:108FB000EE03882349F08091E2032881893511F47A
:108FC000216001C02E7F28838091FD03882369F0F2
:108FD0000FEF1FEF20E230E040E050E06F2D84E023
:108FE0000E94C73D9923A4F0888780910C048823B0
:108FF000F9F000E010E020E031EE40EB54E06F2D9E
:1090000085E00E94C73D8C0184E0003B180730F4E6
:1090100062E08E2D0E94F43B99270EC0FF2401C010
:10902000F3948F2D0E94F51280179107C8F3F982EF
:109030000E94B66081E090E0DF91CF911F910F9187
:10904000FF90EF900895FF920F931F93F42E80E00E
:109050000E94301088EE93E00E9435190EE410E073
:109060002FEF30E041E050E06F2D80E00E94C73DDF
:109070008C01F89487E00E943010C8010E94322CC5
:1090800066E9C8010E946220789481E090E01F9117
:109090000F91FF900895EF92FF920F931F93CF933C
:1090A000E82EF42E00E010E027EE30E040EC50E037
:1090B0006F2D80E00E94C73DC82F2FEF30E0A80140
:1090C0006F2D81E00E94C73D282F8C2F805C883255
:1090D00030F061E08E2D0E94573C992718C08C2FEC
:1090E00099278F739070982F8827820F911D9F93D7
:1090F0008F9386E798E09F938F93EF920E94FA1CDC
:1091000081E090E00F900F900F900F900F90CF9113
:109110001F910F91FF90EF9008950F931F93CF939E
:10912000C82F842F0FEF1FEF2FEF37E241E050E001
:10913000682F80E00E94C73D9C0188E220303807FC
:1091400030F061E08C2F0E94573C992723C0C90161
:1091500090709F938F939F938F93832F9927806C09
:109160009F938F939F938F933F932F933F932F932F
:1091700085E898E09F938F93CF930E94FA1C81E03B
:1091800090E02DB73EB7215F3F4F0FB6F8943EBF3A
:109190000FBE2DBFCF911F910F910895AF92BF9237
:1091A000CF92DF92EF92FF920F931F93CF93DF93B3
:1091B000E82E5B01F42E8091DF03882309F447C079
:1091C00000E010E020E034E041E050E06F2D81E06D
:1091D0000E94C73DEC01892BD1F100E010E02FEF98
:1091E00030E0A8016F2D82E00E94C73D6C0160EC69
:1091F00078E0C5010E94DB78AC01892BC9F40FEF40
:109200001FEF2EEF31E06F2D80E00E94C73DFC0183
:1092100088E2E030F807D8F4CE0101972C2DAC019C
:1092200061E0CF0103E0880F991F0A95E1F717C0AD
:109230000FEF1FEF2FEF37E241E050E06F2D80E09E
:109240000E94C73DFC0188E2E030F80710F061E0C1
:1092500009C0CE0101972C2DAC0160E0CF010E9426
:10926000332F60E08E2D0E94573C9927DF91CF91DC
:109270001F910F91FF90EF90DF90CF90BF90AF9034
:109280000895FF920F931F93CF93DF93F82EEB0176
:10929000842F00E010E020E034E041E050E0682F4F
:1092A00080E00E94C73D9C01892B29F18B81682FAA
:1092B000772764347105D1F06534710524F4623484
:1092C0007105A1F018C06035710559F0623571055E
:1092D00091F42930310578F4822F81500E94A16ADF
:1092E0000CC0C90101970E94B66A07C0C901019765
:1092F0000E94816A02C061E004C08C0197FF06C031
:1093000067E08F2D0E94573C992726C09F938F932B
:109310009F938F9383EC98E09F938F93FF920E948B
:10932000FA1C8DB79EB707960FB6F8949EBF0FBE76
:109330008DBFC02F65E28F2D0E94371C10E88C2F47
:10934000812311F061E301C060E38F2D0E94371C7F
:109350001695A9F781E090E0DF91CF911F910F91D1
:10936000FF900895CF92DF92EF92FF920F931F9399
:10937000CF93DF93D82E7B01C42E8091D003882316
:1093800009F461C000E010E020E034E041E050E08A
:109390006C2D80E00E94C73DEC01892B09F453C07D
:1093A00000E010E02FEF30E0A8016C2D81E00E947A
:1093B000C73D9C01F7018381682F772764347105CD
:1093C000E1F06534710524F462347105E1F03BC0CD
:1093D0006035710561F062357105A9F5C930D105B7
:1093E00090F5622F8C2F81500E94966A2EC0622FBA
:1093F000CE0101970E94AC6A28C0622FCE0101976E
:109400000E94776A22C00FEF10E027E030E040E0D2
:1094100050E06C2D81E00E94C73D7C018F3F99F0A8
:109420000FEF10E021E030E040E050E06C2D82E0F2
:109430000E94C73DAC018F3F31F06E2DCE010197E8
:109440000E94636A02C061E005C0892B11F067E0E9
:1094500001C060E08D2D0E94573C9927DF91CF918C
:109460001F910F91FF90EF90DF90CF9008951F9381
:10947000CF93DF93182F80E190E00E94816A9923B7
:1094800054F0C82F805C8832C8F481E190E00E94DB
:10949000816A97FF02C067E012C0282F8C2F99279E
:1094A0008F739070D82FCC27C20FD11D41E065E09B
:1094B0008CE190E00E94636A97FF06C061E0812F13
:1094C0000E94573C992710C0DF93CF9381ED98E01D
:1094D0009F938F931F930E94FA1C81E090E00F905E
:1094E0000F900F900F900F90DF91CF911F910895E3
:1094F0000F931F93CF93C82F842F0FEF1FEF2FEFE2
:1095000037E240E850E0682F80E00E94C73D8C01C0
:1095100088E200301807D8F4812F9927806C682FD3
:1095200080E190E00E94776A99233CF0602F81E10E
:1095300090E00E94776A97FF02C067E00BC041E0AD
:1095400065E08CE190E00E94636A97FF02C061E0F1
:1095500001C060E08C2F0E94573C9927CF911F914A
:109560000F910895DF92EF92FF920F931F93CF9385
:10957000DF93082FEB01D42E823008F00EC188E46F
:10958000089F900111242D5D3C4F4881142F1F71BD
:10959000642F7727CB01807E90708034910509F489
:1095A000A3C08134910534F40097A9F0809709F4A1
:1095B00063C0F3C08038910509F4BFC081389105BC
:1095C0002CF48036910509F4B0C0E7C0803C9105C9
:1095D00009F4CCC0E2C021E02D1508F0E0C089817B
:1095E000C82FDD27CE010E94322CFC01892B09F403
:1095F000D4C0E480F58014FF05C080E090E8E82A3C
:10960000F92A04C08FEF9FE7E822F9221F70068134
:1096100000781F3019F460E8602729C080851F702A
:1096200011F01F3019F460E070E020C00E944A2F52
:10963000282F33272C31310571F02D31310524F4D9
:109640002B31310529F010C02E37310531F00CC017
:10965000110F115009C0110F07C089E0189F802D0C
:109660001124682F772702C0612F7727602B40E0F5
:10967000CE010E94972D50C0437F4883E5E4EE2E33
:10968000F12CE20EF31EF70180819181FFEF8F3FF5
:109690009F0749F040E0642F0E94CE758FEF9FEF47
:1096A000F701808391832881203209F476C0233228
:1096B00009F473C0F1E0FD15D0F46981213231F471
:1096C000C62FDD272197CC0FDD1F05C0C62FDD2754
:1096D000CC0FDD1F219740E061E0CE010E94CE75E6
:1096E000F701C083D18359C0F1E0FD1518F080E087
:1096F00090E055C08981C82FDD27CE010E94CF2C74
:1097000050EFE52E5FEFF52EE822F922812F992701
:109710008F709070E82AF92A40E0B701CE010E94CC
:10972000392ECE010E94C62E38C060FF02C080E0F4
:1097300001C083E00E94301030C0112311F4812F4A
:1097400018C0C0E0C11748F560E08C2F0E94C06AC5
:10975000682F802F0E94371C61E08C2F0E94C06A06
:10976000682F802F0E94371CCF5FECCF112321F48C
:1097700081E00E94E16A11C0115060E0812F0E94D7
:10978000C06A682F802F0E94371C61E0812F0E94E1
:10979000C06A682F802F0E94371C81E090E0DF9123
:1097A000CF911F910F91FF90EF90DF9008959B0153
:1097B0002F5F3F4F42E0B9010E94B24A8FEF90E025
:1097C00008959B012F5F3F4F41E0B9010E94B24ACB
:1097D0008FEF90E008958230C0F4282F332788E47B
:1097E00090E0289FF001299FF00D389FF00D112483
:1097F000ED5DFC4FEC5BFF4F1082339610828FEFD4
:109800009FEF929382930E94F47708950895CF92E8
:10981000DF92EF92FF920F931F93CF93DF93C82EA7
:10982000062F81E08C1508F4ACC288E4C89EE001E4
:109830001124CD5DDC4FF4E4EF2EF12CEC0EFD1E77
:10984000F70180818823A9F088819981AA81BB8151
:1098500088539F4FAF4FBF4FBC01CD010E94ED1603
:10986000882339F0CE010E94CF35882311F4F70107
:1098700080838091410690914206A0914306B09169
:10988000440688839983AA83BB83F701808180344F
:1098900008F01082CE010E94ED35882381F0083057
:1098A00041F4F7018081882309F46BC281508083E1
:1098B00068C2002309F465C20D3009F400E0F70125
:1098C0001081FE01E10FF11D04831F5FF70110837A
:1098D000CE010E94CF35D82E882309F448C2CE018C
:1098E0000E94ED35882309F412C2002309F049C211
:1098F000F70100838E010C5F1F4FC95BDF4F88812A
:10990000C754D040882319F48E010B5F1F4FF80114
:109910008081882309F4F5C143E050E064ED78E0EC
:10992000C8010E94FA78892B59F4CDEBD3E4C80121
:1099300003960E94587AC8010E94A93CF82ED9C10A
:10994000C8010E94587AC8010E94A93CF82E68ED0F
:1099500078E0C8010E94DB78892B39F06AED78E065
:10996000C8010E94DB78892B19F4CFE5DEE3C1C181
:109970006CED78E0C8010E94DB78892B19F4CAE409
:10998000DEE3B7C16FED78E0C8010E94DB78892B78
:1099900019F4C1E5DEE3ADC162EE78E0C8010E94D2
:1099A000DB78892B19F4C8E5DEE3A3C165EE78E026
:1099B000C8010E94DB78892B39F067EE78E0C80196
:1099C0000E94DB78892B19F4C5EADEE392C16CEEC4
:1099D00078E0C8010E94DB78892B39F06EEE78E0E0
:1099E000C8010E94DB78892B19F4CAEBDEE381C140
:1099F00061EF78E0C8010E94DB78892B19F4CFEC85
:109A0000DEE377C166EF78E0C8010E94DB78892B3E
:109A100019F4CAE5DFE36DC168EF78E0C8010E9480
:109A2000DB78892B19F4C8E6D0E463C16BEF78E0EA
:109A3000C8010E94DB78892B19F4C9E9D0E459C127
:109A40006DEF78E0C8010E94DB78892B19F4CAE039
:109A5000D1E44FC160E079E0C8010E94DB78892B36
:109A600019F4CBE7D1E445C162E079E0C8010E9476
:109A7000DB78892B19F4C3E7DEE33BC164E079E0CE
:109A8000C8010E94DB78892B19F4CBE2D2E431C102
:109A900066E079E0C8010E94DB78892B19F4C1E502
:109AA000D2E427C169E079E0C8010E94DB78892B04
:109AB00019F4CCE9D2E41DC16CE079E0C8010E9440
:109AC000DB78892B19F4CBECD2E413C16FE079E099
:109AD000C8010E94DB78892B19F4C1E3D3E409C1E2
:109AE00062E179E0C8010E94DB78892B19F4CAE3AE
:109AF000D3E6FFC065E179E0C8010E94DB78892BDD
:109B000019F4CEE5D3E4F5C067E179E0C8010E941D
:109B1000DB78892B19F4CFE8D3E4EBC06AE179E074
:109B2000C8010E94DB78892B19F4CBE4D8E4E1C0AA
:109B30006DE179E0C8010E94DB78892B19F4CDE84A
:109B4000D8E4D7C060E279E0C8010E94DB78892BB5
:109B500039F063E279E0C8010E94DB78892B19F4BF
:109B6000CEECD8E4C6C066E279E0C8010E94DB789A
:109B7000892B51F16BE279E0C8010E94DB78892BD7
:109B800069F160E379E0C8010E94DB78892BE1F09C
:109B900065E379E0C8010E94DB78892BF9F06AE37C
:109BA00079E0C8010E94DB78892B71F06FE379E0DE
:109BB000C8010E94DB78892B89F064E479E0C80150
:109BC0000E94DB78892B19F4C1E4D9E492C069E4DE
:109BD00079E0C8010E94DB78892B19F4C2EBD9E443
:109BE00088C06EE479E0C8010E94DB78892B19F403
:109BF000C7E3DAE47EC063E579E0C8010E94DB7860
:109C0000892B19F4C8E7DAE474C068E579E0C80183
:109C10000E94DB78892B19F4C5EED3E46AC06BE5AA
:109C200079E0C8010E94DB78892B19F4C9EED4E4ED
:109C300060C063E679E0C8010E94DB78892B19F4E3
:109C4000C6EFD4E456C06AE679E0C8010E94DB782A
:109C5000892B19F4CDE4D5E44CC063E779E0C80161
:109C60000E94DB78892B19F4C2ECD5E442C06BE783
:109C700079E0C8010E94DB78892B19F4CFECD5E498
:109C800038C062E879E0C8010E94DB78892B19F4BA
:109C9000C0E0D6E42EC06BE879E0C8010E94DB7812
:109CA000892B19F4C1E2D6E424C063E979E0C80144
:109CB0000E94DB78892B19F4C0E4D7E41AC06AE962
:109CC00079E0C8010E94DB78892B19F4C8E9D7E450
:109CD00010C061EA79E0C8010E94DB78892B19F491
:109CE000C3E2D8E406C065EA79E08C2D0E94A41C8A
:109CF00008C04F2DB8018C2DFE010995882309F469
:109D000040C065EB79E08C2D0E94A41C3AC0E0E0D5
:109D1000F1E0DE011496212FC95BDF4F8881C75423
:109D2000D040882319F4DE0115962150809100015E
:109D3000882339F190818C919817A1F4818128179B
:109D400000F10280F381E02D309749F0BD018C2DA8
:109D50000995682F8F3F19F08C2D0E94371CF70151
:109D600010820FC034968081882321F70AC0249680
:109D7000412FBE018C2D0E94B24A882311F0F701B9
:109D8000D082DF91CF911F910F91FF90EF90DF90E4
:109D9000CF900895FB0121E057FF04C020E05095CB
:109DA00041955F4F8330910549F18430910534F43A
:109DB0008130910591F0029729F12AC084309105F4
:109DC00019F0059761F024C081818F5F8183992705
:109DD00084179507ECF0222359F0118219C0818174
:109DE0008150818399278417950794F0222321F0CD
:109DF000842F815081830CC021830AC01282138278
:109E0000168A06C090E08281882309F491E092834B
:109E100080E090E008950F931F93CF93DF938C0120
:109E20000E94562FEC01009731F463E273E182E067
:109E30000E94A41C0FC09F938F9389E293E19F938C
:109E40008F9382E08F930E94FA1C0F900F900F90D7
:109E50000F900F900115110521F0B80182E00E94CA
:109E6000A41CCE01DF91CF911F910F9108950F9304
:109E70001F93CF93DF93EC018B01009731F097FD97
:109E800035C00297029790F52BC060E081E00E94F8
:109E9000E01AF8018281882359F46DE273E182E0CF
:109EA0000E94A41C66E373E182E00E94A41C18C017
:109EB0000E946C61DC01CB01BF93AF939F938F93A2
:109EC0008CE393E19F938F9382E08F930E94FA1C1F
:109ED0008DB79EB707960FB6F8949EBF0FBE8DBF85
:109EE00040E050E0B801CE010E94CA4E80E090E010
:109EF000DF91CF911F910F9108958230910541F02C
:109F00008330910541F440E050E00E94CA4E03C006
:109F10008FEF9FEF089580E090E008950895AF924D
:109F2000BF92CF92DF92EF92FF920F931F93CF9346
:109F3000DF93EC017B010E94532F8C01C230D105CD
:109F400009F453C0C330D1052CF42097D1F02197E8
:109F500031F092C0C630D1050CF08EC02AC0FC0191
:109F60006589262F269526952370637009F461E094
:109F700083E0689FC0011124280F2350F70121833B
:109F80007BC060E081E00E94E01A88E493E10E94D7
:109F90000B4F892B09F470C0F70191818AE0989FDB
:109FA000C0011124875F954FBC0182E00E94A41C70
:109FB00063C049E050E0B701CE010E94CA4EF801EB
:109FC000808191818F3F910509F008F455C0F70118
:109FD0008181882311F486E08183F70181818630B5
:109FE00008F04AC088E0818347C0FC01A280B380AA
:109FF000A114B10409F040C0F70182818823A1F1C6
:10A00000F801C081D1812097B9F1F7013181832F07
:10A0100063E00E94C97D282F2F5F832F0E94C97D96
:10A02000892F9927880F991F880F991F282BF801CE
:10A03000C08CD18C622FCE010E94D92CCE010E94FF
:10A04000BB2CB5010E945B30C114D10469F0C8017A
:10A050004A969C01F801458960817181C6010E9480
:10A06000E66CF801808F918F90E0F7018281882360
:10A0700009F491E0F701928380E090E0DF91CF91C5
:10A080001F910F91FF90EF90DF90CF90BF90AF9016
:10A090000895482F30E0832F992787FD9095FC0184
:10A0A000E852F64F2491241729F03F5F222399F7B5
:10A0B0008FEF9FEF08950895EF92FF920F931F93F4
:10A0C000CF93DF93EB018230910509F486C0833092
:10A0D000910534F4009709F43EC0019769F0BAC0C5
:10A0E0008430910509F443C0843091050CF470C0AC
:10A0F000059709F456C0AEC00E94532F8C01FC0195
:10A1000080819181892B09F4A5C04AE1E42EF12CCC
:10A11000E00EF11E8E01065F1F4F65960C171D079E
:10A12000B8F4F7018081882339F00E94495087FDF7
:10A1300003C0F701808101C080E2F80181938F01A3
:10A14000F7018081882351F30894E11CF11CE6CFCC
:10A15000F80110827FC00E940B4F60E081E00E94F6
:10A16000E01A2A96BE0182E00E94BA1C73C089815F
:10A17000FB01E80FF11DEF012A9682850E944950EC
:10A180008F5FE82FFF27E7FDF095E852F64F8491A7
:10A19000882319F4E8EDF9E08491992787FD9095DB
:10A1A00015C08981FB01E80FF11DEF012A96828518
:10A1B0000E944950181614F08FE201C08150E82F18
:10A1C000FF27E7FDF095E852F64F8491888342C05F
:10A1D00049E050E00E94CA4E3DC00E94532F8C01BE
:10A1E000FC0182819381892BA9F59A81992349F4F5
:10A1F00089E08B8381E0888F99839F8B8A838E8B04
:10A2000029C089818F5F89838F8B8B3018F11B82E6
:10A210001A821E8A8CE09801265E3F4FD901FE010A
:10A220003A9601900D928A95E1F7F801808D918D13
:10A23000009731F04589608171810E94E66C07C00A
:10A24000A901F8016589808191810E947E6DF801E4
:10A25000808F918F80E090E0DF91CF911F910F91DF
:10A26000FF90EF900895AF92BF92CF92DF92EF925E
:10A27000FF920F931F93CF93DF93CDB7DEB7219754
:10A280000FB6F894DEBF0FBECDBF9C018B018230AC
:10A29000910509F455C0833091052CF40097C1F065
:10A2A000019759F0A5C084309105D9F1843091050A
:10A2B0000CF441C00597C9F19BC04BE050E060E24F
:10A2C00070E0C8010A960E948E78F801158A90C045
:10A2D000FB018281882309F48BC08181882309F4E2
:10A2E00087C0065F1F4FA801B90199270E94866D9C
:10A2F0009F938F938BE493E19F938F9362E0F62E6D
:10A30000FF920E94FA1C60E081E00E94E01AB8010E
:10A310008F2D0E94BA1C0F900F900F900F900F90EE
:10A3200067C0FB018181992721C0FB0181819927A9
:10A330000E947B6E1DC049E050E00E94CA4E58C08A
:10A3400090E0FB018281882309F491E0F801928377
:10A350000E94532F7C01F8018281882361F0F7016C
:10A36000808D918D009711F0808D02C00E94466E05
:10A37000F80181833DC05AE0A52EB12CA00EB11E7C
:10A38000F8018181A501BE016F5F7F4F99270E946F
:10A39000866D6C01F7011282138210821182BC015A
:10A3A0008FEF0E94AA62F70180819181892B69F069
:10A3B0006981C6010E94D92CC6010E94BB2C60E0B5
:10A3C00070E00E945B300E94652FF70180819181CF
:10A3D000892B59F0B501C7014A960E94E578F8012A
:10A3E00081819927F701808F918F8FEF9FEF02C0B6
:10A3F00080E090E021960FB6F894DEBF0FBECDBF8F
:10A40000DF91CF911F910F91FF90EF90DF90CF9050
:10A41000BF90AF9008950F931F93CF93DF93EC01FC
:10A420000E94532F8C01209719F02297C9F03DC04C
:10A43000CE010E940B4F892BC1F160E081E00E94A8
:10A44000E01AF801808D918D892B11F081E001C017
:10A4500082E00E941D60BC0182E00E94A41C25C015
:10A46000FC01C281D381209701F580819181892BE4
:10A47000E1F0808D918D892BC1F060E081E00E9438
:10A48000E01A83E00E941D60BC0182E00E94A41CCF
:10A4900084EF91E00E943519F801808D918D0E9422
:10A4A000E36CF801C08FD18F128E80E090E0DF91D5
:10A4B000CF911F910F910895CF93DF93EB018230DD
:10A4C000910561F1833091052CF4009781F001979B
:10A4D00029F034C0863091058CF51BC00E942F6195
:10A4E000FC0187818983833048F1198227C060E0AD
:10A4F00081E00E94E01A8981865F0E941D609F931F
:10A500008F9382E08F930E94FA1C0F900F900F9010
:10A5100015C043E050E00E94CA4E10C08A818823D3
:10A5200039F00E942F612981FC0127830E94B660C7
:10A5300090E08A81882309F491E09A8380E090E09A
:10A54000DF91CF9108951F93CF93DF93EB0182307A
:10A55000910509F440C0833091052CF4009789F0EF
:10A56000019731F04CC0863091050CF048C02EC0E8
:10A570000E942F61FC01848163E00E94C97D898370
:10A580003EC060E081E00E94E01A898113E0819F73
:10A59000802D11240E94321C82E090E00E94351927
:10A5A00081B7612F0E94C97D898399279F938F93DB
:10A5B0008FE493E19F938F9382E08F930E94FA1C24
:10A5C0000F900F900F900F900F9019C04FEE5FEF0C
:10A5D0000E94CA4E14C08A81882359F00E942F61BC
:10A5E000398123E0329F90011124FC0124830E94D1
:10A5F000B66090E08A81882309F491E09A8380E034
:10A6000090E0DF91CF911F9108951F93CF93DF9337
:10A61000EC018A81882309F45CC060E081E00E943B
:10A62000E01A8C819D819F938F9383E593E19F93A3
:10A630008F9312E01F930E94FA1C8B810F900F9052
:10A640000F900F900F90843059F489E593E19F9318
:10A650008F931F930E94FA1C0F900F900F9010C0C1
:10A66000888599279F938F938DE593E19F938F938F
:10A670001F930E94FA1C0F900F900F900F900F9055
:10A68000898D9A8D97FD03C061E673E10AC08E5FE4
:10A690009F4F19F469E673E104C084E00E941D60D5
:10A6A000BC0182E00E94A41C81E0888F8E8B8B818C
:10A6B00099278130910564F08330910524F0049747
:10A6C000029730F402C083E001C088E08F8B01C0A4
:10A6D0001E8ADF91CF911F9108950F931F93CF93FF
:10A6E000DF938C01FC018281882311F581E0838353
:10A6F000643019F488E090E003C080E094E0F80151
:10A7000086839783F801248135818681978182171A
:10A71000930724F481E090E08483958381E0F8013D
:10A720008283683009F410C180E00E9430100CC1AF
:10A73000F801848195819093530480935204C62F2D
:10A74000DD27C430D10561F1C530D10594F4C130A5
:10A75000D10509F4C2C0C230D1051CF4209701F123
:10A76000F3C0C230D10509F4BAC0239709F4E9C097
:10A77000EBC0C730D10509F4B0C0C830D10544F4EE
:10A78000C530D10509F4A9C0C630D10549F0DCC0F7
:10A79000C830D10509F47EC0299709F49EC0D4C001
:10A7A000F801838181508230E0F58EEF9FEF818F39
:10A7B000928FC8010E9405536AE081E00E94E01A6E
:10A7C0008DE00E941D60BC0182E00E94A41CC43088
:10A7D000D10581F0C530D1051CF4CD2B21F019C075
:10A7E000269771F016C0F8018481958101970E9427
:10A7F000816A0CC0F801848181500E94A16A06C060
:10A80000F8018481958101970E94B66AF801818FD1
:10A81000928FF801818D928D97FD5DC0818D80872B
:10A820005AC06AE081E00E94E01A8EE00E941D603A
:10A83000BC0182E00E94A41CC430D10589F0C5305F
:10A84000D1051CF4CD2B21F046C02697C1F043C0A2
:10A85000F80184819581608501970E94776A16C00E
:10A86000F8018481958109971CF08FEF9FEF0FC04D
:10A87000F8018481608581500E94966A07C0F801C2
:10A8800084819581608501970E94AC6AF801818F6F
:10A89000928F21C00E94532FFC01A081B18110979B
:10A8A000D1F085899927837090700397A1F4F801FE
:10A8B000448155814115510571F083818150823069
:10A8C00050F041505040208560E0CD010E94332F70
:10A8D000F801138239C081E035C084E033C0F8014B
:10A8E00083818150823010F481E02DC06AE081E0E4
:10A8F0000E94E01AF8018381863079F48DE00E948D
:10A900001D60BC0182E00E94A41CF8018481958135
:10A91000618501970E946D6A0FC08EE00E941D60E4
:10A92000BC0182E00E94A41CF80184819581418DC4
:10A93000618501970E94636AF801818F928F86E09A
:10A9400001C087E0F8018383DF91CF911F910F91C0
:10A9500008959C01FB018130910561F082309105E1
:10A960001CF4892BD1F024C083309105E9F00597C0
:10A97000C1F01EC08EEF9FEF818F928F40915204E5
:10A9800050915304CA0101978050944018F44483B5
:10A9900055830EC0248335830BC0CB010E94055321
:10A9A00007C081E0838304C040E050E00E94CA4EAB
:10A9B00080E090E008950F931F93CF93DF938C0175
:10A9C000EB010E94532FFC0180819181892B31F092
:10A9D0008589992783709070039731F060E081E05A
:10A9E0000E94E01A85E00DC00E947110833081F052
:10A9F0000E947110823061F060E081E00E94E01AF4
:10AA000086E00E941D60BC0182E00E94A41C1BC065
:10AA10000230110541F00430110589F469E0CE01DE
:10AA20000E946D5310C068E0CE010E946D538B816F
:10AA3000882349F40E94EF1A8FEF9FEF06C0BE01F2
:10AA4000C8010E94A95480E090E0DF91CF911F914E
:10AA50000F910895CF93DF93EB018230910509F4B4
:10AA600081C08330910534F40097A1F081309105C5
:10AA700069F07CC08430910509F462C0843091058E
:10AA80000CF46BC0059709F460C070C00E94A95413
:10AA900019866CC08A81882309F468C060E081E06F
:10AAA0000E94E01A8B81882331F461E773E182E030
:10AAB0000E94A41C18C0898599279F938F938C812D
:10AAC0009D819F938F9381E893E19F938F9382E081
:10AAD0008F930E94FA1C8DB79EB707960FB6F89415
:10AAE0009EBF0FBE8DBF898D9A8D97FD0BC08230A2
:10AAF00091051CF0029721F005C0898D805D03C08F
:10AB00008FE301C085E40E94921A81E0888F8E8BCA
:10AB10008B8199278630910561F08730910524F467
:10AB20000197029758F403C0079729F007C086E001
:10AB300003C08CE001C08EE08F8B18C01E8A16C047
:10AB40008B81863039F463E00EC08B81863011F43E
:10AB500081E001C086E08B8309C040E050E00E94A4
:10AB6000CA4E04C062E0CE010E946D5380E090E0C6
:10AB7000DF91CF9108959B018230910529F08430B7
:10AB8000910539F461E001C060E0C9010E946D5394
:10AB900002C00E94A95480E090E008959B01823099
:10ABA000910529F08430910539F465E001C064E035
:10ABB000C9010E946D5302C00E94A95480E090E038
:10ABC00008959B018230910529F08430910539F474
:10ABD00067E001C066E0C9010E946D5302C00E9497
:10ABE000A95480E090E008951F93182F60E081E061
:10ABF0000E94E01A812F99278130910571F08230EF
:10AC000091051CF4892B39F013C08230910539F07D
:10AC1000039739F00DC08FE005C080E103C081E1EA
:10AC200001C082E10E941D60BC0182E00E94A41C60
:10AC30001F910895CF93C82F1816B4F480E00E9496
:10AC4000F4556C2F80E090E00E94776A892B39F4EC
:10AC500040E065E08CE190E00E94636A07C08C2FC1
:10AC60000E948B6A892B11F082E001C083E00E9470
:10AC7000F45584EF91E00E943519CF910895CF9358
:10AC8000DF93EB0182309105E1F1833091051CF4F3
:10AC9000892B29F04EC08330910571F14AC08A8119
:10ACA000882309F446C060E081E00E94E01A8C81AC
:10ACB0009D8197FF0CC080E993E19F938F9382E081
:10ACC0008F930E94FA1C0F900F900F900FC09F93CC
:10ACD0008F9385E993E19F938F9382E08F930E94F6
:10ACE000FA1C0F900F900F900F900F9083E08F8BB6
:10ACF00081E0888F8E8B1DC040E050E00E94CA4EDC
:10AD000018C08A81882321F08C810E941A5605C0C0
:10AD100081E00E94F45581E08A8380E090E00E9407
:10AD2000816A8C839D8381E08B838FE790E08E83A3
:10AD30009F8380E090E0DF91CF9108950F931F9360
:10AD4000CF93DF938B018130910571F082309105B3
:10AD50001CF4892B79F0B4C08230910509F43FC00E
:10AD600083309105B9F1ACC08FEF9FEFFB01848375
:10AD70009583A6C0FB018281882309F4A1C060E00D
:10AD800081E00E94E01AF8018481958197FF0CC050
:10AD900089E993E19F938F9382E08F930E94FA1C3D
:10ADA0000F900F900F900FC09F938F9380EA93E1C5
:10ADB0009F938F9382E08F930E94FA1C0F900F90C5
:10ADC0000F900F900F9085E0F801878B81E0808FC6
:10ADD000868B76C040E050E00E94CA4E71C0FB01F5
:10ADE0008281882389F1C481D581C038D10520F4BE
:10ADF0008C2F0E941A562EC0F8E2C030DF07A0F454
:10AE000080E00E94F4558D2F9927806C682F80E197
:10AE100090E00E94776A009729F46C2F81E190E01E
:10AE20000E94776A892B11F082E007C041E065E05B
:10AE30008CE190E00E94636A83E00E94F45584EF05
:10AE400091E00E94351906C081E00E94F45581E02E
:10AE5000F8018283F8018481958101978F379105EC
:10AE600040F480E090E00E94816AF8018483958339
:10AE700015C080E190E00E94816A982F8827F80130
:10AE80008483958381E190E00E94816AF8012481A6
:10AE90003581282B392B3F7324833583F801848136
:10AEA0009581805098422CF08FEF9FEFF8018483BA
:10AEB000958381E0F80183838FEF97E28683978300
:10AEC00080E090E0DF91CF911F910F9108951F9343
:10AED000CF93DF93EB01122F8230910519F183306C
:10AEE00091052CF4009761F0019729F02EC086306F
:10AEF00091055CF512C0842F0E945061898325C0A2
:10AF000060E081E00E94E01A8981810F0E947560F3
:10AF1000BC0182E00E94A41C18C042E050E00E94E4
:10AF2000CA4E13C08A81882351F08981882321F079
:10AF3000842F0E945A6103C0842F0E94626190E0B6
:10AF40008A81882309F491E09A8380E090E0DF9180
:10AF5000CF911F91089522E048E00E94675708951D
:10AF600020E041E00E94675708950F931F93CF930D
:10AF7000DF938C01EB0126E044E00E94675702302A
:10AF8000110529F48A81882311F40E948D2280E022
:10AF900090E0DF91CF911F910F9108951F93CF9370
:10AFA000DF93EB018230910541F1833091052CF460
:10AFB000009789F0019729F03CC086309105CCF5C7
:10AFC00017C010E080E090E00E943076039709F40B
:10AFD00011E019832EC060E081E00E94E01A8981AF
:10AFE0008E5F0E947560BC0182E00E94A41C21C09B
:10AFF00042E050E00E94CA4E1CC08A81882399F02A
:10B0000060E081E00E94E01A64EA73E182E00E945D
:10B01000A41C8981882319F083E090E002C081E0BC
:10B0200090E00E94607690E08A81882309F491E0A4
:10B030009A8380E090E0DF91CF911F9108950F9364
:10B040001F93CF93DF939C01EB018230910509F4AC
:10B050006BC0833091052CF4009739F1019731F0E2
:10B0600097C0863091050CF093C059C08C819D81AA
:10B0700001978C5F934010F02C833D838CEF93E01D
:10B080008E839F8311E01B831E8B83E08F8B188F31
:10B0900000E08C819D81880F991F02970E94307675
:10B0A000039709F4012F098373C060E081E00E94D7
:10B0B000E01A8B812C813D81813009F52D5F3F4F56
:10B0C0003F932F938C819D819F938F938BE292E08E
:10B0D0009F938F9312E01F930E94CE1C89818C5FF7
:10B0E0000E947560BC01812F0E94A41C8DB79EB781
:10B0F00007960FB6F8949EBF0FBE8DBF49C03F9311
:10B100002F9385E392E09F938F9382E08F930E9429
:10B11000CE1C0F900F900F900F900F9039C042E00F
:10B1200050E00E94CA4E34C02A812223A1F08981B6
:10B130002C813D81882329F0220F331F63E070E0CA
:10B1400004C0220F331F61E070E0C90102970E9422
:10B1500078761A821DC08B81813019F48A832E8BF8
:10B1600017C08C819D8101978C7F01968C839D8374
:10B17000122F880F991F02970E943076039709F4C7
:10B1800011E0198391E09B839E8B83E08F8B988FD6
:10B1900080E090E0DF91CF911F910F910895FF9291
:10B1A0000F931F93CF93DF93EC018B01F42E0E943A
:10B1B0002F61FC01C230D10509F471C0C330D10543
:10B1C0002CF42097C9F0219771F07DC0C430D105CF
:10B1D00009F44DC0C430D1050CF44DC0C530D105C3
:10B1E00009F449C070C0FF2019F08485E80155C0FA
:10B1F0008385F801818367C060E081E00E94E01AE6
:10B20000E8019981FF20F9F0892F6AE00E94C97D49
:10B21000892F99279F938F9389810E94C97D9927B0
:10B220009F938F9383EB93E19F938F9382E08F9310
:10B230000E94FA1CEDB7FEB737960FB6F894FEBF22
:10B240000FBEEDBF40C082E3989FC00111249F93C1
:10B250008F938BEB93E19F938F9382E08F930E9468
:10B26000FA1C0F900F900F900F900F902CC0F801C8
:10B2700081818F3F41F1FF2019F040E05FEF02C074
:10B280004BEE5FEFB801CE010E94CA4EFF20D9F00D
:10B29000E80189818823B9F481E0898314C0E80139
:10B2A0008A81882341F09981FF2011F0948701C0A1
:10B2B00093870E94B66090E0F8018281882309F4A8
:10B2C00091E0E8019A8380E090E0DF91CF911F91B7
:10B2D0000F91FF90089540E00E94CF58089541E0FB
:10B2E0000E94CF580895CF93DF93EB0182309105F0
:10B2F00059F1833091052CF4009759F0019729F00A
:10B300002FC08630910564F51AC00E943761898389
:10B3100027C060E081E00E94E01A89819927880FA8
:10B32000991F880F991F8854964FBC0182E00E9494
:10B33000A41C61EC73E182E00E94A41C11C048E0EF
:10B3400050E00E94CA4E0CC08A81882319F089817E
:10B350000E943B6190E08A81882309F491E09A83FE
:10B3600080E090E0DF91CF910895CF93DF93EB01E0
:10B3700082309105C1F18330910534F4009749F092
:10B380008130910551F157C0863091050CF053C0C2
:10B3900024C08A81882309F44EC061E080E00E94C5
:10B3A000E01A8981885F0E947560BC0182E00E947A
:10B3B000A41C60E081E00E94E01A6981623020F004
:10B3C00086E10E941D6004C0862F845F0E94756024
:10B3D000BC0182E00E94A41C2EC042E050E0BE01ED
:10B3E0000E94CA4E28C08A81882319F1898182303F
:10B3F00018F48E5F89831FC060E081E00E94E01A2C
:10B400008981833051F483E10E941D60BC0182E098
:10B410000E94A41C0E94D97109C084E10E941D6091
:10B42000BC0182E00E94A41C0E94A1728FEF9FEFDA
:10B4300004C081E08A8380E090E0DF91CF9108959D
:10B44000CF9380914904803178F010924904109292
:10B450004A0461E0862F0E94E01ACEE085EA0E944D
:10B46000921AC150C7FFFACF6091490481E00E944F
:10B47000E01A80914A0499278130910559F0823071
:10B4800091051CF4892B21F014C0029739F011C0EA
:10B4900085E001C084E00E94921A0BC080E20E9405
:10B4A000921A85E00E94921A809149048F5F8093DE
:10B4B000490480914A048F5F80934A04833010F0DE
:10B4C00010924A04CF910895CF93DF93EB0182301D
:10B4D000910559F1833091051CF4892B31F053C04B
:10B4E000863091050CF04FC01BC08A81882309F477
:10B4F0004AC061E080E00E94E01A8DE10E941D6078
:10B50000BC0182E00E94A41C60E081E00E94E01A7D
:10B5100085E10E941D60BC0182E00E94A41C33C032
:10B5200040E050E00E94CA4E2EC08A81882329F153
:10B530000E944B2269EB71E084E00E940F1C61EBDA
:10B5400071E085E00E940F1C68EC70E080E29AE5F3
:10B550000E94191B60E0862F0E94E01A83E00E947F
:10B560001D60BC0182E00E94A41C0E94442B0E942A
:10B57000A46E0E94D8600E943A6390E08A8188237A
:10B5800009F491E09A8380E090E0DF91CF910895F3
:10B59000CF92DF92EF92FF920F931F93CF93DF939F
:10B5A000029709F0CEC060E0862F0E94E01A80E288
:10B5B0000E94921A60E081E00E94E01A80E00E94FE
:10B5C000301069EC73E182E00E94A41C21E04EE49B
:10B5D00068E086E00E94A7116D9880E00E94A913A0
:10B5E00080E00E943815CC24DD248EEF0E94AC153B
:10B5F00080E00E94261D8F5F9F4FD1F781E00E945F
:10B60000261D8F5F9F4FD1F7A8950E94771A87312B
:10B61000910509F488C08B30910509F484C00A971C
:10B6200001F581C0CF3FD10551F0209741F06C2F3B
:10B6300080E00E94371C6C2F81E00E94371CCF33C2
:10B64000D10519F0CB32D10519F4B4E8CB2ED12CA9
:10B65000C332D10511F0AA9721F4A6E0CA2EA1E0C9
:10B66000DA2E0E94D915EC018F5F9F4FD9F6C114D5
:10B67000D10409F4BACFE0904106F090420600915F
:10B6800043061091440688EC90E0A0E0B0E0E80E9C
:10B69000F91E0A1F1B1F3BC0A8950E94261DEC0126
:10B6A0009FEFCF3FD90721F481E00E94261DEC01D6
:10B6B000AFEFCF3FDA0721F18C2F0E94AC15089431
:10B6C000C108D108E0904106F0904206009143067F
:10B6D0001091440688EC90E0A0E0B0E0E80EF91E7E
:10B6E0000A1F1B1F0DC0CF3FD10551F0209741F01D
:10B6F0006C2F80E00E94371C6C2F81E00E94371C69
:10B700000E94D915EC019FEFCF3FD90761F7C11413
:10B71000D10409F468CFC801B7010E94ED1688234F
:10B7200009F4BACF60CF81E00E94A91381E00E94A2
:10B7300038156D9A0E94376121E04EE468E00E945E
:10B74000A71180E090E0DF91CF911F910F91FF90C2
:10B75000EF90DF90CF900895CF93DF93EB0182308D
:10B76000910509F440C0833091052CF4009771F0E5
:10B77000019731F048C0863091050CF044C02EC0CE
:10B780000E942F61FC01868189833DC060E081E0D9
:10B790000E94E01A6981662369F488E10E941D60B5
:10B7A0009F938F9382E08F930E94FA1C0F900F90CB
:10B7B0000F9029C085E0689FC00111249F938F934B
:10B7C00086ED93E19F938F9382E08F930E94FA1C02
:10B7D0000F900F900F900F900F9015C049EC50E014
:10B7E0000E94CA4E10C08A81882339F00E942F61BE
:10B7F0002981FC0126830E94B66090E08A8188231B
:10B8000009F491E09A8380E090E0DF91CF91089570
:10B81000CF93DF93EB018130910569F08230910580
:10B820001CF4892B81F049C08230910539F18330B5
:10B830009105F9F042C00E942F61FC018085992793
:10B840008C839D833AC060E081E00E94E01A8C8185
:10B850009D819F938F938CED93E19F938F9382E0D3
:10B860008F930E94FA1C0F900F900F900F900F90E3
:10B8700024C040E050E00E94CA4E1FC08A81882345
:10B8800061F483E08B8380E290E08E839F8391E07C
:10B89000988F82E08F8B9E8B0AC01E8A0E942F6138
:10B8A0002C81FC0120872093E5090E94B66090E07E
:10B8B0008A81882309F491E09A8380E090E0DF9107
:10B8C000CF910895EF92FF920F931F93CF93DF9341
:10B8D0008C01EB010E942F617C010230110509F4FB
:10B8E00063C00330110544F40115110571F00130F6
:10B8F000110509F446C072C00330110509F43DC0BA
:10B90000063011050CF06AC03CC08A81882309F416
:10B9100065C0F7018085882309F460C060E081E09C
:10B920000E94E01A8C819D819F938F9381EE93E119
:10B930009F938F9382E08F930E94FA1C60E089812D
:10B940000E94C06A082F61E089810E94C06A182F96
:10B95000C0E80F900F900F900F900F9094E0802F01
:10B960008C2309F096E0812F8C2309F09F5F892FAB
:10B970000E94921AC69591F731C01E8A81E00E94FA
:10B98000E16AF70180859927AC01BE01C8010E94D8
:10B99000CA4E8981992701968C839D838B81823041
:10B9A000E9F488E08B831AC02A81222391F481E094
:10B9B00090E08C839D83F701808599278E839F83F8
:10B9C00011E01A83822F0E94E16A188F85E08F8B25
:10B9D0001E8B88E08B838C818150898380E090E08E
:10B9E000DF91CF911F910F91FF90EF900895CF922B
:10B9F000DF92EF92FF920F931F93CF93DF937C011F
:10BA0000C62F0E94071C0E942F616C01C43208F0EF
:10BA10006FC085E0C89F8001112404581E4FF701B4
:10BA20008281882311F080E001C082E00E94921A96
:10BA3000F6018581992781309105B1F08230910519
:10BA40001CF4892B39F031C082309105B9F003978D
:10BA5000F9F02BC08C2F992744E0880F991F4A9545
:10BA6000E1F78D509F4E1DC08C2F992734E0880F31
:10BA7000991F3A95E1F78D53914F13C08C2F992759
:10BA800024E0880F991F2A95E1F78D56934F09C03E
:10BA90008C2F9927C4E0880F991FCA95E1F78D591B
:10BAA000954FBC0182E00E94A41CE8018C8187FDB7
:10BAB0000BC060E081E00E94E01A8C810E941D6052
:10BAC000BC0182E00E94A41CE801EA81FB8130975E
:10BAD00021F0B70180E090E00995F701868988237D
:10BAE00029F06789808D0E94E91A02C00E94EF1A2E
:10BAF000DF91CF911F910F91FF90EF90DF90CF904A
:10BB0000089560E0ECE7F1E0482F552747FD509598
:10BB100020E030E0808199278417950711F4C9014E
:10BB200008956F5F2F5F3F4F3596633298F38FEF25
:10BB30009FEF08950895BF92CF92DF92EF92FF9208
:10BB40000F931F93CF93DF93CDB7DEB76B970FB6ED
:10BB5000F894DEBF0FBECDBFB82E22E2281718F42E
:10BB600080E090E0FBC16E010894C11CD11C8BE108
:10BB7000F60111928A95E9F7A89585E0B89EF00143
:10BB80001124E458FE4F0280F381E02D309721F01C
:10BB9000B60181E090E009956B2DC6010E94F75C2B
:10BBA0000E94751085E0B89E700111248CE791E029
:10BBB000E80EF91E0E94771AAC018A30910509F44B
:10BBC000E9C08B30910564F4009709F40AC1181696
:10BBD00019060CF41EC14F5F5F4F09F4AEC1E0CFF0
:10BBE0008731910509F48EC08831910544F48B307A
:10BBF000910509F487C0459709F49BC1D1CF8931DC
:10BC0000910519F04A9751F1CBCFF6018281882333
:10BC100081F0F701228133812115310531F0BE0118
:10BC20006F5F7F4F84E090E081C1F60181818F5F7B
:10BC300028C0F601868BF7019081F1E2FB1534F004
:10BC4000F7018581891711F4B39431C0892F0E94BF
:10BC5000815D682F772767FD709540C0F60182816E
:10BC6000882389F0F701228133812115310531F0D4
:10BC7000BE016F5F7F4F85E090E058C1F601818182
:10BC80008150818367C1F601868B6B2DF70190810E
:10BC9000BB2091F02BEF3FEFE20EF31EF701808106
:10BCA00025E030E0E20EF31E891731F4BA946B2DD3
:10BCB000772767FD709512C031E23B1564F0D7011C
:10BCC0001596F7018581891731F46F5F62321CF494
:10BCD00015968C91F8CF772767FD7095B62E85E085
:10BCE000689FF0011124E458FE4F0280F381E02D9B
:10BCF000309709F42FC1BE016F5F7F4F81E090E064
:10BD0000099528C1F7019181992361F1092F112724
:10BD1000055B1B4FF801808118162CF0892F0E94BB
:10BD2000815DF8018083F7018181E82FFF27E55BC2
:10BD3000FB4F80810E949B5D282F332727FD309584
:10BD4000F7018181E82FFF27E55BFB4FC90137FF32
:10BD500004C088279927821B930B808337FFFAC082
:10BD6000B1943AC0F701228133812115310551F098
:10BD7000BE016F5F7F4F82E090E0F9010995992342
:10BD80007CF319C0F6018281882309F491E0F60161
:10BD90009283E0C0F60182818823F1F0F7012281CD
:10BDA000338121153105A9F0BE016F5F7F4F83E01C
:10BDB00090E0F9010995F6018281882309F0CAC053
:10BDC000F70122813381BE016F5F7F4F81E090E0F8
:10BDD000ADC0F6011282BEC08B2D992787FD9095CC
:10BDE000BDC0F6018381813009F4DACE883089F450
:10BDF00081E00E94E16A60E0F60181810E94C06AF0
:10BE000061E0F60181810E94C06A80E00E94E16ADF
:10BE1000A1C0F601838199278530910509F454C0AA
:10BE20008630910584F48230910581F1833091054B
:10BE30001CF40197B9F08EC08330910599F00497F6
:10BE400009F43EC087C08730910509F456C0873099
:10BE500091050CF44CC08830910521F0099709F444
:10BE600053C078C0F60186819781892B21F48FEF2A
:10BE70009FE786839783F6018681978184179507CC
:10BE80000CF468C01482158282E08383F6018481F9
:10BE900095819C0163E0220F331F6A95E1F7280F1B
:10BEA000391F280F391F240F351F37FD53C08681D6
:10BEB0009781821793070CF44DC0248335834AC0C1
:10BEC000F601108685E08383F60190858AE0989FCD
:10BED00090011124240F351F2F3F310509F008F47C
:10BEE00020878EEF9FEFF601818F928F33C048300D
:10BEF000510584F5F60141872DC04230510554F5B6
:10BF0000F601418F528F26C0F6018181E80FF11DA5
:10BF1000842F805D8287F7012281338121153105CD
:10BF2000C9F0BE016F5F7F4F82E090E0F901099593
:10BF300011C080E00E9430100DC0F601838188306E
:10BF400009F02ECEBE016F5F7F4F80E090E00E942F
:10BF5000625C26CE6B2DCE01019620CE6B960FB67D
:10BF6000F894DEBF0FBECDBFDF91CF911F910F912F
:10BF7000FF90EF90DF90CF90BF900895CF93C82FA0
:10BF80000E947A61803809F456C061E871E080E06F
:10BF90000E940F1C69E871E082E00E940F1C69EAB0
:10BFA00071E084E00E940F1C61EA71E085E00E946C
:10BFB0000F1C69E971E086E00E940F1C61E971E0E5
:10BFC00087E00E940F1C80914B04833210F0109286
:10BFD0004B04C7FD04C08C2F0E949B5D0EC0809156
:10BFE0004B040E949B5D992787FD909597FF03C0A6
:10BFF000909581959F4F80934B0461E672E080E0BD
:10C000000E940F1C61E472E082E00E940F1C69E153
:10C0100072E084E00E940F1C61E172E085E00E9402
:10C020000F1C69E072E086E00E940F1C61E072E084
:10C0300087E00E940F1CCF910895CF93C82F8F31B6
:10C0400018F08BEE9FE12CC00E942F61FC018581CE
:10C0500099278230910581F0833091051CF4019776
:10C0600021F018C0039779F015C081E1C89FC00185
:10C0700011248452924E14C081E1C89FC001112442
:10C080008353944E0DC081E1C89FC0011124825496
:10C09000964E06C081E1C89FC00111248155984E7B
:10C0A000CF910895882319F088EF9FE108950E94A9
:10C0B0002F61FC01858199278230910561F08330E1
:10C0C00091051CF4019721F00CC0039739F009C0C9
:10C0D0008EE997E108958DE897E108958CE797E15F
:10C0E00008958BE697E108950895CF93C82F8E3079
:10C0F00018F088E090E238C00E942F61FC01858131
:10C1000099278230910599F0833091051CF40197AD
:10C1100021F021C00397A9F01EC08C2F992754E06D
:10C12000880F991F5A95E1F78557994E1DC08C2F9E
:10C13000992744E0880F991F4A95E1F785559A4E53
:10C1400013C08C2F992734E0880F991F3A95E1F797
:10C1500085539B4E09C08C2F992724E0880F991F87
:10C160002A95E1F785519C4ECF910895EF92FF9269
:10C170001F93CF93DF9384E5E82E84E0F82EC0E090
:10C18000D0E01FE1CE010E945578F70161917F0157
:10C19000861719F0CE010E946E78A895115021964D
:10C1A00017FFF0CFDF91CF911F91FF90EF9008958F
:10C1B00090915904943008F091E08FE0E4E5F4E0C8
:10C1C00011928A95E9F788E1809358049093590475
:10C1D00081E08093550484E180935A0482E0809347
:10C1E0005F0482E3809360040E94B660089540E299
:10C1F00050E060E070E084E594E00E945D7880911A
:10C200005604909157048F5F9F4F11F40E94D8609D
:10C2100080915504883018F081E080935504809116
:10C22000610490916204885F974020F0109262044C
:10C230001092610480915904843010F010925904D6
:10C240008AEF9FEFA1E0B0E0ABBFFC0187918F3F89
:10C2500021F0882311F080936F000895089584E5FC
:10C2600094E00895809359040E94B66008958091E7
:10C27000550499270895CF93C82F883008F0C7E058
:10C2800080915504C81751F0C09355040E94B660C0
:10C2900021E04EE468E08C2F0E94A711CF91089511
:10C2A00020E030E090915404982311F021E030E038
:10C2B000C901089590915404982B909354040E94BE
:10C2C000B6600895982F90958091540489238093A7
:10C2D00054040E94B66008958CEF9FEFA1E0B0E097
:10C2E000ABBFFC0187919791A791B691B070BC014B
:10C2F000CD0108958FEF9FEFA1E0B0E0ABBFFC014F
:10C300008791823011F4079B80E8992708950E9455
:10C31000842BFC01892BB9F0A4E7B4E043E02D9114
:10C320003C911197808191812817390729F08281EA
:10C3300093812817390719F41D921C9211974150C7
:10C34000139647FFECCF089508959F92AF92BF9246
:10C35000CF92DF92EF92FF920F931F93CF93DF93D1
:10C36000CDB7DEB726970FB6F894DEBF0FBECDBFB0
:10C37000C82E7B01942ECE0101960E946C63DD24B1
:10C3800094E7A92E94E0B92EF501808191818E1554
:10C390009F0509F096C082818F5F8283843008F404
:10C3A000C5C0C7010E94322C8C01009709F4C0C09F
:10C3B000FFEFCF1639F5992029F0FC0164817581D2
:10C3C000C7011BC0FC01448155816681C7010E94E1
:10C3D000FA2FC7010E94C66DBC01F80180850E943A
:10C3E0005B30F80182819381009749F00E94322CE2
:10C3F000FC0164817581808191810E9444300E949A
:10C40000652F59C0992049F0FC014481558160E0B5
:10C41000CE0101960E944F6341C0FC0144815581C9
:10C420006681CE0101960E944F63AE014F5F5F4F60
:10C4300067E08C2D0E94EF63F80180858F778B83F6
:10C44000C7010E94C66DBC01CE0104960E946C63B8
:10C450000E9405648823E1F3AE014F5F5F4F69E0FE
:10C460008C2D0E94EF63F801828193810E94842BBE
:10C470008C010097D1F0FC0160817181CE010196A1
:10C480000E946C63F8014481558160E0CE01019601
:10C490000E944F630E9405648823E1F3AE014F5F61
:10C4A0005F4F68E08C2D0E94EF6340E050E06DE04C
:10C4B0008C2D0E94EF63F5011082118281E090E0E3
:10C4C00037C0D39483E090E0A80EB91E93E09D1589
:10C4D00008F05ACFDD2404E714E0F801808191814F
:10C4E000892BA1F40E94562F8E159F0519F40E94E6
:10C4F0006B2F07C0AE014F5F5F4F65E08FEF0E946B
:10C50000EF63F801E082F182128206C0D3940D5FDE
:10C510001F4FF3E0FD1508F783E08D1538F4AE01E9
:10C520004F5F5F4F66E08FEF0E94EF6380E090E027
:10C5300026960FB6F894DEBF0FBECDBFDF91CF9128
:10C540001F910F91FF90EF90DF90CF90BF90AF9031
:10C550009F9008950F931F93CF93DF93082FEB01C4
:10C56000672B79F010E040E0BE01802F0E94A561AA
:10C57000882339F40E9405648823E1F31F5F143196
:10C5800090F3DF91CF911F910F9108958F929F9219
:10C59000BF92CF92DF92EF92FF920F931F93CF93B0
:10C5A000DF93CDB7DEB726970FB6F894DEBF0FBE88
:10C5B000CDBFB82E4B016A01CB010E94322C8C01F9
:10C5C000892B09F445C0C6010E94322C7C01892BBD
:10C5D00009F43EC0F80180850E944A2F8C01F701C2
:10C5E00080850E944A2F081B190BC80117FF03C042
:10C5F000909581959F4F0297E4F0FFEFBF1621F4CD
:10C6000081E00E94CC3024C086E0FE013196119278
:10C610008A95E9F781E08983AE014F5F5F4F61E260
:10C620008B2D0E94EF6314C0B601C4010E94742ECA
:10C630000FC010E041E0B6018B2D0E94A561882358
:10C6400099F70E9405648823E1F31F5F143190F38A
:10C6500026960FB6F894DEBF0FBECDBFDF91CF9107
:10C660001F910F91FF90EF90DF90CF90BF909F9020
:10C670008F9008950E944B22F894FFCF682790E096
:10C6800027E0862F86959F5F60FF03C0682F622793
:10C6900001C0682F9830A8F3862F99270895FC01D0
:10C6A000262F862F8F77828326952074CA01892FA3
:10C6B0009927869586958F73822B8383CA0123E001
:10C6C000969587952A95E1F78F778483842F8295B5
:10C6D000807F8F7785830895FC01CB01262F2F77EC
:10C6E0002083880F892F881F990B91958F778183DD
:10C6F0000895803480F4E82FFF27662329F0E95459
:10C70000FB4F8AE080830895E954FB4F80818823A2
:10C7100011F08150808308950895EF92FF920F9356
:10C720001F93CF93DF93782FC62F7A01A89580911E
:10C73000A404282F33278091A5049927019728174F
:10C74000390741F08091A404833039F48091A50425
:10C75000882319F480E090E03BC09091A40489E024
:10C76000989F8001112400581B4F872F8068F80183
:10C770008083682F80E00E943E63F801C1836C2FA4
:10C780000E943E63982FE801229605E0E114F1042F
:10C7900031F0F70181917F018F77888301C0188282
:10C7A0006991892F0E943E63982F015007FFEECFB9
:10C7B00087FD909598838091A4048F5F8093A40453
:10C7C0008091A404843010F01092A40481E090E0E1
:10C7D000DF91CF911F910F91FF90EF9008950F93EC
:10C7E0001F93CF93DF93082F162FEA0102C00E94F8
:10C7F0007510AE01612F802F0E948D638823B9F3DD
:10C80000DF91CF911F910F9108959F92AF92BF92A8
:10C81000CF92DF92EF92FF920F931F93CF93DF930C
:10C82000CDB7DEB76C970FB6F894DEBF0FBECDBFA5
:10C83000992459C227FF05C01092AD048FEF809351
:10C84000AF048091AD04893040F4E82FFF27E25512
:10C85000FB4F20838F5F8093AD048091AD048930BE
:10C8600009F041C28091AE0487FF3DC28EEAE82EF6
:10C8700084E0F82E90E017E0F70181917F01682FA6
:10C88000892F0E943E63982F115017FFF5CF87FD27
:10C8900090958091B604981709F020C2FF248091EA
:10C8A000AE0488230CF01AC20FE7B02EB8223091E4
:10C8B000B004C32EDD244091B104842F99279695AE
:10C8C000982F882797958795C82AD92A2091AF0451
:10C8D000822F9927AA27BB27FC013197E334F10562
:10C8E00008F0FCC1EA5BFF4FEE0FFF1F0590F491CB
:10C8F000E02D09941091B2048091B304282F3327BE
:10C9000026FD1068322F2227330F330F8091B40495
:10C9100099278F779070A3E0880F991FAA95E1F768
:10C92000282B392B8091B504992780779070F4E0FB
:10C9300095958795FA95E1F7282B392B41E0B901B8
:10C94000C6010E94392E41E0612FC6010E94972D39
:10C95000C6010E948761BEC18091B204992790E40C
:10C96000899F902D88271124C82AD92A6091B30461
:10C97000662319F041E0642F01C041E0C6010E9426
:10C98000CE75A8C18091B204482F55278091B30479
:10C99000282F3327C901877090709695982F882784
:10C9A00097958795482B592B20743070220F331F91
:10C9B0008091B404822B282F60E0C6010E94332F9F
:10C9C00089C18091B204E82EFF24002711278091AD
:10C9D000B30499279695982F882797958795AA2726
:10C9E00097FDA095BA2FE82AF92A0A2B1B2B8091D4
:10C9F000B404992790E4899F902D88271124AA27B1
:10CA000097FDA095BA2FE82AF92A0A2B1B2B209113
:10CA1000B504822F9927AA27BB2787709070A07032
:10CA2000B07035E1880F991FAA1FBB1F3A95D1F747
:10CA3000E82AF92A0A2B1B2B269526952695D8013C
:10CA4000C7010197A109B1098F5F9F4FAF4FB04058
:10CA500008F040C1A601C801B7010E9483713AC124
:10CA60000E947110843009F435C18091B0040E9495
:10CA70003010882309F42EC184E00E94C5772AC1B2
:10CA8000C114D10409F426C1B6018B2D0E94AA62FB
:10CA900021C16091B204C6010E94D92C8091B004DA
:10CAA0008A878091B1048B87C6010E94BB2C8C873A
:10CAB000AE01465F5F4F69E0A7C01AE0E12EF12C9E
:10CAC000EC0EFD1EAE01405F5F4FBE01645F7F4F05
:10CAD000C6010E94866D6C018F778A87CC0CCD2CA5
:10CAE000CC1CDD08D1948C2D8F778B8788898D871E
:10CAF00089898E871F86A70161E18B2D0E94EF63D4
:10CB00008E010F5F1F4FF80194E08189818791505A
:10CB1000319697FFFACFA70162E18B2D0E94EF6358
:10CB2000F80193E0868981879150319697FFFACF7B
:10CB3000A70163E169C0A3E0FA2E33E0F30E83E0BE
:10CB4000F80E8601243199F48091B204C82EDD24B8
:10CB50008091B30499279695982F88279795879564
:10CB6000C82AD92A8091B4048C8F188A23C0AE01B8
:10CB7000405F5F4FBE01645E7F4FC6010E94866DBD
:10CB80006C0194E0EAE0EF1588F0DE01AF0DB11D15
:10CB90005096E92FFF27E255FB4F80818D939F5FD1
:10CBA000F394973018F4FAE0FF1598F7FE01EF0DB3
:10CBB000F11D108A9E01205F3F4F4C8DB601C801C8
:10CBC0000E94E66C8C018F778A87000F012F001F6F
:10CBD000110B1195802F12C0213121F4C6010E9442
:10CBE000466E03C0C6010E947B6E6C018F778A87F8
:10CBF000CC0CCD2CCC1CDD08D1948C2D8F778B8761
:10CC0000AE01465F5F4F60E18B2D0E94EF6362C013
:10CC1000C6010E94E36C5EC08091B204282F3327C6
:10CC20008091B30499279695982F88279795879593
:10CC3000282B392BA901B6018B2D0E94C6624AC050
:10CC4000C6010E94992E46C0BB24E7EBF4E0819117
:10CC5000882369F440EB54E064E08B2D0E94EF637D
:10CC60008091A7048B1538F4B092A70404C0B39444
:10CC70003FE33B1560F782E08093A8042BC08091CE
:10CC8000A804833038F583E08093A8043093A90486
:10CC90004093AA048091B2048093AB041092AC0438
:10CCA00019C08091A8048230A8F482E08093A8047F
:10CCB0003093A9044093AA041092AB040BC0909146
:10CCC000A804992339F481E08093A8043093A9043F
:10CCD0009093AA0461E08B2D0E9479631092AD04B9
:10CCE0008FEF8093AF040E94D9159C018FEF2F3FE7
:10CCF000380709F09FCD0E949B150A970CF421C1BB
:10CD00009091A4048091A504981711F19091A50425
:10CD100089E0989F70011124E0E8F4E0EE0EFF1E18
:10CD200008E010E0F70181917F010E94AC150150ED
:10CD3000104017FFF7CF8091A5048F5F8093A50463
:10CD40008091A504843008F4FCC01092A504F9C0B9
:10CD50007E010894E11CF11C57018091A6048034E7
:10CD600029F06091A804662309F475C08FEF8983C8
:10CD70000894E11CF11C8091A80499278130910549
:10CD8000C9F0823091051CF4892B39F059C08230EA
:10CD9000910519F10397C1F153C080E4F701819324
:10CDA0008091A904982F97708F5F8093A904919325
:10CDB0007F0148C081E4F70181938091A9048770C5
:10CDC00081938091AA04982F9F778F5F8093AA0404
:10CDD00091937F018091AA0431C082E4F70181938D
:10CDE0008091A904877081938091AA048F778193A1
:10CDF0008091AB04982F9F778F5F8093AB049193C2
:10CE00007F018091AB041AC083E4F7018193809184
:10CE1000A904877081938091AA048F778193809170
:10CE2000AB048F7781938091AC04982F9F778F5FAD
:10CE30008093AC0491937F018091AC0487FF02C082
:10CE40001092A8048091A804882309F059C0809109
:10CE5000A6048F5F53C08134A1F58FEF89830894B6
:10CE6000E11CF11C83E0F70181937F018F0108949D
:10CE7000E11CF11C0E9471108F77F8018083809172
:10CE8000A6048F5F8093A6040E94532F8C01FC019F
:10CE9000848981FF13C0808191810E94876141E074
:10CEA000F8016689808191810E94972D41E0F80107
:10CEB00066817781808191810E94392E51E0952E83
:10CEC0001FC0803410F06093A6048091A60480688F
:10CED00089830894E11CF11C82E0F70181937F01B2
:10CEE0008091A6040E9479638091A6048F5F80934D
:10CEF000A6049091A704981718F480E48093A604E0
:10CF0000CE010996E816F90620F4F70111927F0187
:10CF1000F9CFDD24750107E010E0F70160818D2D68
:10CF20000E943E63D82EF70181917F010E94AC15CB
:10CF30000150104017FFF1CFD7FCD0948D2D0E94E7
:10CF4000AC15A895892D99276C960FB6F894DEBF7D
:10CF50000FBECDBFDF91CF911F910F91FF90EF904A
:10CF6000DF90CF90BF90AF909F900895CF93DF93C5
:10CF7000CDB7DEB726970FB6F894DEBF0FBECDBF94
:10CF800036E0FE01319611923A95E9F74983AE01F8
:10CF90004F5F5F4F0E94EF6326960FB6F894DEBF97
:10CFA0000FBECDBFDF91CF9108951F93CF93DF9335
:10CFB000EC0110E001C0A8950E94AB228823D9F3B0
:10CFC00011C0A89504C081E090E00E9435190E942C
:10CFD000AB228823C1F341E060E080E090E00E9452
:10CFE000AD2021970E94C122882311F4209749F790
:10CFF0000E94C122811111E0C5E00FC043E060E052
:10D0000080E090E00E94AD200E94C52201C0A8955A
:10D010000E94AB228823D9F3C1500E94C1228823E9
:10D0200011F0CC2359F7CC2309F41C2F812F992719
:10D03000DF91CF911F910895EF92FF921F93CF93AD
:10D04000DF937C01CFEFDFEF10E0612FC7010E947B
:10D050002B2180E090E00E94D567882311F0C12F3A
:10D06000DD271F3F49F483E090E00E94D5678823C5
:10D0700031F0CFEFD0E005C01F5FD7FDE6CFD7FD81
:10D0800014C01C2FCFEFDFEF612FC7010E942B21AF
:10D0900083E090E00E94D567882311F0C12FDD273F
:10D0A000112319F01150D7FDEFCFCE01DF91CF91B1
:10D0B0001F91FF90EF9008954F925F926F927F9231
:10D0C0008F929F92AF92BF92CF92DF92EF92FF9298
:10D0D0000F931F93CF93DF93CDB7DEB726970FB68D
:10D0E000F894DEBF0FBECDBF782E5B01C42E522E4A
:10D0F000402E8091620082608093620080E00E94F6
:10D10000321C86E0FE01319611928A95E9F7AE0154
:10D110004F5F5F4F62E28FEF0E94EF630E94D22267
:10D1200083EC87B98FEE86B96FEF862E962E662434
:10D1300080E00E94301082E390E00E94351984E084
:10D140000E94301084E690E00E943519E09041067C
:10D15000F0904206009143061091440680ED97E05E
:10D16000A0E0B0E0E80EF91E0A1F1B1FDD2410929C
:10D17000F8041092F7042BC00E94CD22AC0120913C
:10D18000F7043091F804C901885A9D4F8417950718
:10D1900034F0C901885592404817590744F4509318
:10D1A000F8044093F704DD2059F0DA9409C0240F05
:10D1B000351F359527953093F8042093F704D394C1
:10D1C00094E09D1550F08AE090E00E943519C80166
:10D1D000B7010E94ED16882379F28091F7049091AF
:10D1E000F80444975CF584E393E00E94C82283E04E
:10D1F00090E00E94D56710E0412F612F80E090E021
:10D200000E94F22083E090E00E94D567811111E036
:10D2100041E060E080E090E00E94F22083E090E056
:10D220000E94D56781111F5F113041F484E190E0C5
:10D230009093F8048093F70445E0D42E8091F7048E
:10D240009091F8044497855A9B4028F4B4E0BD15AA
:10D2500010F1442001F560E081E00E94E01A809125
:10D26000F7049091F8048431910514F489E106C023
:10D27000895B9B4014F08AE101C08BE10E941D6034
:10D28000BC0182E00E94A41C80E00E94301088EE65
:10D2900093E00E9435198091F7049091F804805E24
:10D2A0009C4F0E94C82286E990E00E9435190E9496
:10D2B0007110843009F0D8C0072D112703301105F3
:10D2C00009F447C0043011054CF40130110539F15F
:10D2D00002301105FCF4012B71F0ACC005301105D2
:10D2E0000CF4A8C0073011050CF453C00930110527
:10D2F0000CF0A0C06FC0452D6C2DC5010E94D2203E
:10D300008FE090E00E94D567882309F497C0852CB0
:10D31000992494C06C2DC5010E9444214CC040E06A
:10D320006C2DC5010E94F22083E090E00E94D56739
:10D33000882309F046C041E06C2DC5010E94F2200F
:10D3400083E090E00E94D567882309F477C0480104
:10D3500077C010E0012F169540E0602FC5010E94B4
:10D36000F22083E090E00E94D567882309F41068DA
:10D370000F5F083080F3612FC5010E945D2183E0BB
:10D3800090E00E94D567882309F458C0812E992423
:10D3900055C061E085E090E00E9412218FE090E0AE
:10D3A0000E94D567C50187709070F5E07F1661F423
:10D3B0006C2D0E9412218FE090E00E94D567882397
:10D3C000E9F1882499243CC00E941C684C0133E098
:10D3D000632E34C0C5019695879596958795682FDD
:10D3E0006F5F85E090E00E9412218FE090E00E9444
:10D3F000D567C5018370907027E0721661F46C2DBB
:10D400000E9412218FE090E00E94D567882341F0AE
:10D410008824992405C00E941C684C0193E0692E61
:10D4200061E085E090E00E9412218FE090E00E9490
:10D43000D56704C08FEF882E982E08C097FC06C0D1
:10D44000442021F08CE291E00E94351980E00E9496
:10D45000301097FE09C08CE291E00E943519639468
:10D4600082E0861508F064CE16B886B187B90E94AE
:10D470002F61FC0184810E94321C81E08983AE010E
:10D480004F5F5F4F62E28FEF0E94EF638091620017
:10D490008D7F80936200C40126960FB6F894DEBF9C
:10D4A0000FBECDBFDF91CF911F910F91FF90EF90F5
:10D4B000DF90CF90BF90AF909F908F907F906F90B4
:10D4C0005F904F9008950F93242F01E0462FBC01E9
:10D4D00080E00E945C680F9108950F9300E0202F78
:10D4E000462FBC0181E00E945C680F9108950F9364
:10D4F00001E020E0462FBC0182E00E945C680F91B1
:10D5000008950F9300E0202F402FBC0183E00E947C
:10D510005C680F9108950F9301E020E0482F60E0D0
:10D5200070E085E00E945C680F9108950F93992741
:10D5300001E020E0462FBC0185E00E945C680F916D
:10D5400008950F93992700E0202F402FBC0186E01B
:10D550000E945C680F9108950F9301E020E0462F30
:10D56000BC0187E00E945C680F9108950F9300E072
:10D57000202F402FBC0188E00E945C680F91089525
:10D58000880F61118F5FF894E82FFF27E95DF54F51
:10D5900090818091E60980FD10827894892F9927E7
:10D5A0000895880F61118F5FF894E82FFF27DF013E
:10D5B000A959B54F8C91E951F64F808378949927FA
:10D5C00008959091E609882311F0916001C09E7F33
:10D5D0009093E6090895089580E4E7EEF9E011924A
:10D5E0008A95E9F7089584E08093740010927100A1
:10D5F00082E28093700008951F920F920FB60F92EF
:10D6000011248F939F93EF93FF938091710099273B
:10D61000887F90708032910509F487C0813291052E
:10D620006CF480319105D9F0813191051CF4089793
:10D63000D1F07DC0489709F43FC079C0803491058E
:10D64000A9F18134910524F4889709F441C06FC091
:10D6500080359105D9F08835910561F068C08091D9
:10D66000F90487FF02C080EA01C081EA8093730059
:10D6700085E861C0E091FF04F0910005809173009E
:10D680008193F0930005E093FF0448C0E091FF040C
:10D69000F0910005809173008193F0930005E09371
:10D6A000FF048091FA0481508093FA048091FA0477
:10D6B0008230F4F285EC3FC08091FD049091FE042D
:10D6C000892F9927809373008FEF8093F904D0CF2F
:10D6D0008091F90487FF09C08091FD049091FE04B8
:10D6E000809373001092F904C3CF8091FB048823C8
:10D6F000E1F08091FA04882389F0E091FF04F09131
:10D7000000058191F0930005E093FF04809373007E
:10D710008091FA0481508093FA04AACF84E980931F
:10D72000740081E08093FC0408C085EA04C08FEF98
:10D730008093FC0484E980937400FF91EF919F91A2
:10D740008F910F900FBE0F901F90189580917400CD
:10D75000992787709070009711F081E090E008950C
:10D7600008956093FA049093FE048093FD0420933F
:10D77000FB04509300054093FF048EEF8093F9045F
:10D780001092FC0485EA8093740008958091FC0453
:10D79000992787FD909508950E94B16B01C0A895C7
:10D7A0000E94C66B892BD9F38091FC04992787FDD1
:10D7B00090950895AB0120E060E134E0880F991F57
:10D7C0003A95E1F70E94CC6B0895AB0121E060E14E
:10D7D00074E0880F991F7A95E1F70E94CC6B089549
:10D7E00020E0AC0166E080E090E00E94CC6B089500
:10D7F00021E0AC0166E080E090E00E94CC6B0895EF
:10D80000EF92FF920F931F93CF93DF93CDB7DEB7C5
:10D8100022970FB6F894DEBF0FBECDBF7C011982F0
:10D820001A8209811A8120E0AE014F5F5F4F62E0EA
:10D83000C801E4E0880F991FEA95E1F70E94CC6BDC
:10D84000A89589819A81009719F08E159F0549F74F
:10D85000C80122960FB6F894DEBF0FBECDBFDF9190
:10D86000CF911F910F91FF90EF9008950F931F9309
:10D87000CF93DF93CDB7DEB722970FB6F894DEBF14
:10D880000FBECDBF8C0101978F5F934000F520E064
:10D89000AE014F5F5F4F62E0C801A4E0880F991F9F
:10D8A000AA95E1F70E94CC6BC8010E94006C24E0AD
:10D8B0008030920760F421E0AE014F5F5F4F62E07D
:10D8C000F4E0880F991FFA95E1F70E94CC6B22963D
:10D8D0000FB6F894DEBF0FBECDBFDF91CF911F9181
:10D8E0000F910895EF92FF920F931F93CF93DF93C1
:10D8F000CDB7DEB766970FB6F894DEBF0FBECDBFCB
:10D900007C0101978F5F9340F8F4C7010E94366C49
:10D91000CE0101960E94F06B8E01095F1F4F40E11E
:10D9200050E06FEF70E0C8010E948E788B819C817F
:10D930008F839887B801C7010E94E56BEB82FC8258
:10D94000CE0101960E94F86B66960FB6F894DEBF82
:10D950000FBECDBFDF91CF911F910F91FF90EF9040
:10D9600008950F931F93CF93DF93CDB7DEB726971C
:10D970000FB6F894DEBF0FBECDBFCE0101960E9458
:10D98000F06B0B811C810115110589F020E0AE01BF
:10D990004D5F5F4F62E0C801B4E0880F991FBA95F0
:10D9A000E1F70E94CC6BCE0101960E94F86BC80192
:10D9B00026960FB6F894DEBF0FBECDBFDF91CF9194
:10D9C0001F910F9108950E94726C08959F92AF92DB
:10D9D000BF92CF92DF92EF92FF920F931F93CF935C
:10D9E000DF93CDB7DEB7A8970FB6F894DEBF0FBEB2
:10D9F000CDBF8C016B01942E7901232B99F0672BFD
:10DA000089F084E00030180768F40115110521F051
:10DA1000C8010E94366C03C00E94B16C8C010115D4
:10DA2000110511F4C80158C05E010894A11CB11C75
:10DA3000F701CB82DC829D82DE01169620812223B3
:10DA400051F0CE014196A817B90728F431962D93CD
:10DA500020812223C1F7C5014096A817B90708F411
:10DA60001C920FA318A7CE0141960E94F06BEE24E2
:10DA7000FF2409891A8901151105B1F0A895BE0185
:10DA8000695E7F4FC8010E94DA6BC50105964BE0C5
:10DA900050E0BC01CE014C960E94EC78992324F40E
:10DAA00078010F89188DE7CFF50100831183A895C0
:10DAB000B5018FA198A50E94E56B21E0AE01495DFB
:10DAC0005F4F62E0C70114E0880F991F1A95E1F7D4
:10DAD0000E94CC6B8FA198A5A8960FB6F894DEBFD4
:10DAE0000FBECDBFDF91CF911F910F91FF90EF90AF
:10DAF000DF90CF90BF90AF909F9008959A01462FEE
:10DB0000BC0180E090E00E94E66C0895EF92FF92E5
:10DB10000F931F93CF93DF93CDB7DEB760970FB608
:10DB2000F894DEBF0FBECDBF9C017B018A01019737
:10DB30008F5F934018F080E090E01BC0BE016F5FE4
:10DB40007F4FC9010E94DA6BE114F10419F08D8155
:10DB5000F70180830115110551F08BE0F801DE011A
:10DB600016960D9001928A95E1F7F80113868B8144
:10DB70009C8160960FB6F894DEBF0FBECDBFDF91DB
:10DB8000CF911F910F91FF90EF900895EF92FF9228
:10DB90000F931F93CF93DF93CDB7DEB766970FB682
:10DBA000F894DEBF0FBECDBF7C01009719F427C0EB
:10DBB000C80125C0CE0101960E94F06B09811A812F
:10DBC00019C08FEF0F3F1807C1F020E0AE01495F89
:10DBD0005F4F64E0C801062E02C0880F991F0A94A7
:10DBE000E2F70E94CC6B89859A858E159F0501F31B
:10DBF0000F8118850115110521F780E090E06696E8
:10DC00000FB6F894DEBF0FBECDBFDF91CF911F914D
:10DC10000F91FF90EF900895DF92EF92FF920F9394
:10DC20001F93CF93DF93CDB7DEB72D970FB6F89440
:10DC3000DEBF0FBECDBF7C01D62E0E94C66D8C010B
:10DC40000097B1F0AE014F5F5F4FBE01635F7F4F42
:10DC50000E94866DBC018E159F0551F48D858D1532
:10DC600039F09E012F5F3F4F4D2DC8010E94E66C99
:10DC70002D960FB6F894DEBF0FBECDBFDF91CF91CA
:10DC80001F910F91FF90EF90DF9008950F931F93D6
:10DC9000CF93DF93CDB7DEB766970FB6F894DEBFAC
:10DCA0000FBECDBF8C018150944018F080E090E011
:10DCB00017C0CE0101960E94F06B0115110571F09D
:10DCC000BE01695F7F4FC8010E94DA6B8F81988522
:10DCD000009721F02FEF8F3F920711F489819A81ED
:10DCE00066960FB6F894DEBF0FBECDBFDF91CF9121
:10DCF0001F910F910895CF93DF93CDB7DEB726978D
:10DD00000FB6F894DEBF0FBECDBF24E0813092077E
:10DD100018F080E090E00FC0009739F4CE01019632
:10DD20000E94F06B89819A8106C00E94006C009766
:10DD300011F40E94006C26960FB6F894DEBF0FBE59
:10DD4000CDBFDF91CF910895CF92DF92EF92FF92F6
:10DD50000F931F93CF93DF93CDB7DEB766970FB6C0
:10DD6000F894DEBF0FBECDBF1D821E8219821A82BB
:10DD700001E010E00B831C83A895CE01800F911F5A
:10DD80000E94F86B97E0C92ED12CCC0EDD1E40E12D
:10DD900050E06FEF70E0C6010E948E7880E1E82EBF
:10DDA000F12C83E00F3F18073CF40F5F1F4F0F83E8
:10DDB00018870150104002C01F8218860E947510FB
:10DDC00021E0A60160E1C7010E94CC6B0F5F1F4FED
:10DDD00080E190E0E80EF91E94E0003019070CF3A2
:10DDE00066960FB6F894DEBF0FBECDBFDF91CF9120
:10DDF0001F910F91FF90EF90DF90CF900895EF92D9
:10DE0000FF920F931F93CF93DF93CDB7DEB7669743
:10DE10000FB6F894DEBF0FBECDBFCE0101960E94B3
:10DE2000F06B89E00E94B119882329F08EE00E94EE
:10DE3000B119882351F48B819C818F5F9F4F21F50D
:10DE400089819A818F5F9F4FF9F469EB71E084E0DB
:10DE50000E940F1C61EB71E085E00E940F1C68ECD2
:10DE600070E080E29AE50E94191B60E0862F0E9414
:10DE7000E01A83E00E941D60BC0182E00E94A41CA5
:10DE80000E94A46E0E943A6309811A81C801019719
:10DE90008F5F9340A0F4BE01695F7F4FC8010E946D
:10DEA000DA6BEF80F88489859A8501978F5F9742B6
:10DEB00018F0C8010E94726C8701A895E7CF8D8188
:10DEC0009E818F5F9F4F51F4CE0101960E94F06BAF
:10DED0001D821E82CE0101960E94F86B66960FB6D7
:10DEE000F894DEBF0FBECDBFDF91CF911F910F9190
:10DEF000FF90EF900895CF92DF92EF92FF920F93F1
:10DF00001F93CF93DF93CDB7DEB726970FB6F89464
:10DF1000DEBF0FBECDBF6C017B01CE0101960E941A
:10DF2000F06B0D811E8124E00030120718F027C02D
:10DF3000C80127C0C80101978F5F934000F5A895DD
:10DF400020E0A70160E1C80134E0880F991F3A95ED
:10DF5000E1F70E94CC6B20E0F7013296819191911C
:10DF60009F778C159D0521F32F5F2730B8F3F701BC
:10DF700000811181C80101978F5F934000F380E019
:10DF800090E026960FB6F894DEBF0FBECDBFDF91AE
:10DF9000CF911F910F91FF90EF90DF90CF90089558
:10DFA0009F92AF92BF92CF92DF92EF92FF920F9328
:10DFB0001F93CF93DF93CDB7DEB760970FB6F8947A
:10DFC000DEBF0FBECDBF00910105002319F080E038
:10DFD00090E04EC0BE016F5F7F4F0E947B6F009745
:10DFE00009F446C011E010930105AB80BC8045E008
:10DFF000C42ED12CCC0EDD1EC5010E94322CFC019A
:10E00000892B91F1902E868187FD912EE12EF601CC
:10E01000808191818C011F77F92EFF1CFF24FF1C4A
:10E02000C80101978E5F9742B8F4C8010E94322C54
:10E03000FC01892BC9F0FF2021F08681992031F461
:10E0400003C08681992011F0806801C08F77868394
:10E05000B801C5010E94742EE39482E090E0C80EDE
:10E06000D91E96E09E1598F61092010581E090E089
:10E0700060960FB6F894DEBF0FBECDBFDF91CF9193
:10E080001F910F91FF90EF90DF90CF90BF90AF90D6
:10E090009F9008956F927F928F929F92AF92BF92BE
:10E0A000CF92DF92EF92FF920F931F93CF93DF9364
:10E0B000CDB7DEB766970FB6F894DEBF0FBECDBF03
:10E0C0006C01F0900105FF2019F080E090E087C01E
:10E0D0000E94842B8C01009709F481C0FC0182818D
:10E0E0009381009709F47BC08F2CF801868187FF0C
:10E0F00002C0B1E08B2EA7E06A2E712C6C0E7D1E43
:10E10000B301C6010E947B6F7C015C01892BC9F4BD
:10E110000E94B16C7C01892B09F460C0CE0101968C
:10E120000E94F06B8D819E818F83988780509440F0
:10E1300010F0AF82B886ED82FE82CE0101960E9479
:10E14000F86B8EE0FE01399611928A95E9F7C9863F
:10E15000DA86F1E09F2EF801828193818C159D056E
:10E1600091F1E2E0AE2EB12C0E94842B8C0100973D
:10E1700051F1BE016F5F7F4F6A0D7B1DDC012D9158
:10E180003C91FB012087318740E050E0FC01868113
:10E1900087FF02C041E050E0882D992748175907B2
:10E1A00021F03068FB0120873187939482E090E072
:10E1B000A80EB91EF801828193818C159D0519F076
:10E1C000F6E0F91588F621E0A30160E1C70174E0EB
:10E1D000880F991F7A95E1F70E94CC6BC70166966C
:10E1E0000FB6F894DEBF0FBECDBFDF91CF911F9168
:10E1F0000F91FF90EF90DF90CF90BF90AF909F90E6
:10E200008F907F906F900895EF92FF920F931F93DE
:10E21000CF93DF93CDB7DEB7A0970FB6F894DEBFEC
:10E220000FBECDBFBE01695F7F4F0E947B6F7C0137
:10E23000892B09F45BC0CE0147960E94F06B0B8DD1
:10E240001C8D0E151F0519F400E010E01AC0011511
:10E250001105A9F0A89520E0AE01435E5F4F62E092
:10E26000C80134E0880F991F3A95E1F70E94CC6B02
:10E270008D8D9E8D8E159F0521F08C01E8CF0FEFBF
:10E280001FEF84E00030180788F58F8198858F8F05
:10E2900098A3CE0101960E94F06B0115110529F497
:10E2A0008F8D98A18D839E830DC021E0AE01415ECC
:10E2B0005F4F62E0C80104E0880F991F0A95E1F7FB
:10E2C0000E94CC6BA89521E0AE014D5F5F4F62E0EC
:10E2D000C70114E0880F991F1A95E1F70E94CC6BD3
:10E2E000EB82FC82CE0101960E94F86BA0960FB6DD
:10E2F000F894DEBF0FBECDBFDF91CF911F910F917C
:10E30000FF90EF900895EF92FF920F931F93CF939A
:10E31000DF93CDB7DEB728970FB6F894DEBF0FBEF8
:10E32000CDBF7B018C01FA0180910205909103051C
:10E33000892B91F1E982FA820B831C831F82188654
:10E34000022F112700FF09C04F83588740E050E09B
:10E35000BA01CF010E94866DFC0101FF05C08F81CB
:10E36000988590688F839887ED83FE83EF2BA1F0CB
:10E3700021E0AE014F5F5F4F68E080910205909110
:10E3800003050E94CC6B80910205909103050896CD
:10E39000909303058093020528960FB6F894DEBF8C
:10E3A0000FBECDBFDF91CF911F910F91FF90EF90E6
:10E3B0000895CF92DF92EF92FF921F93CF93DF9356
:10E3C000CDB7DEB728970FB6F894DEBF0FBECDBF2E
:10E3D00010E0C12C30E4D32E8091E409181798F591
:10E3E000812F9927FC0123E0EE0FFF1F2A95E1F70B
:10E3F000E80FF91FE80FF91FEC59F84F8081918160
:10E4000089839A83828193818B839C838481958184
:10E410008D839E838085282F33272F83388786819D
:10E4200087FD03C031602F83388721E0AE014F5F45
:10E430005F4F68E0C6010E94CC6B1F5F88E090E0F0
:10E44000C80ED91EC9CF0E942F612FEF3FEF29833D
:10E450003A83FC01858596858B839C8321E0AE0100
:10E460004F5F5F4F68E0C6010E94CC6B88E090E090
:10E47000C80ED91E0E94532FFC01D0920305C092F2
:10E480000205808D918D2489892B41F020FF02C0E7
:10E4900023E001C021E0408D518D07C020FF02C064
:10E4A00022E001C020E04081518160E070E080E026
:10E4B00090E00E94837110E040E050E06BE0812F1B
:10E4C0000E94EF631F5F1034B8F310E00E940564F0
:10E4D0008823E1F31F5F1630C8F310E0212F4FEFC0
:10E4E0005FEF6FEF7FEF8FEF9FEF0E948371C09020
:10E4F0000205D0900305109203051092020587EAE9
:10E50000E82E8AE0F82E1FE121E0A70168E0C601AD
:10E510000E94CC6B1150E8E0F0E0EE0EFF1ECE0E34
:10E52000DF1E17FFF1CF28960FB6F894DEBF0FBE9F
:10E53000CDBFDF91CF911F91FF90EF90DF90CF90F3
:10E5400008957F928F929F92AF92BF92CF92DF9267
:10E55000EF92FF920F931F93CF93DF93CDB7DEB768
:10E560006C970FB6F894DEBF0FBECDBF0E9471103E
:10E57000782E80E00E94301040E050E060E0CA0158
:10E580000E94FA2F86E08E010F5E1F4FF801119254
:10E590008A95E9F7FF24A80167E08F2D0E94EF63B9
:10E5A00084E190E00E943519F3942FE32F1598F73A
:10E5B0000E941A2A19821A82A12C00E4B02E20E0AF
:10E5C000AE014F5F5F4F68E0C5010E94CC6B89814F
:10E5D0009A81EFEF8F3F9E07E1F00E94322C8C0171
:10E5E000892BB9F08F818F70682FF801808191811C
:10E5F0000E94D92C8B819C81F801828393838D8129
:10E600009E81848395838F819885892F992780FDAA
:10E61000168288E090E0A80EB91E89819A818F5FEA
:10E620009F4F69F619861A861B861C86B9E08B2EC9
:10E63000912C8C0E9D1E20E0A40168E0C5010E9473
:10E64000CC6B89859A85AB85BC8580509040A04075
:10E65000B14008F0AAC08D859E85009709F4A5C039
:10E6600028E28030920708F0A0C0FF242F85388967
:10E6700037FF02C0A2E0FA2E8C012115310589F086
:10E6800089011F7740E050E0BA01C8010E94866D01
:10E690002D853E852817390719F481E0F82A01C035
:10E6A0008901F4012081318142815381CF2CDD2405
:10E6B0002115310541055105D1F50E94532F7C01EB
:10E6C000C0FE08C04A96AC0160E070E0C8010E943C
:10E6D000866D8C01C8010E94842B8C010097E1F0AB
:10E6E000FC01448155816681808191810E94FA2FCD
:10E6F00060E070E0F80180850E945B30F801828163
:10E7000093810E94842B009739F0FC01648175810C
:10E71000808191810E944430C1FE04C0F701848948
:10E720008160848BF70184898260848B3EC0802F56
:10E730008F778F8B000F012F001F110B1195802FEA
:10E740008F77888FF40180818F77898FE7E05695E6
:10E75000479537952795EA95D1F7822F8F778A8F3E
:10E7600077E056954795379527957A95D1F7822F7B
:10E770008F778B8F67E056954795379527956A95E4
:10E78000D1F7822F877053E0CC0CDD1C5A95E1F74E
:10E790008C298C8FAE01495E5F4F6CE08FEF0E9439
:10E7A000EF630E9405648823E1F388E090E0A80EFF
:10E7B000B91E89859A85AB85BC8580509040A04064
:10E7C000B14008F433CF07EA1AE04FE1F42E20E01D
:10E7D000A80168E0C5010E94CC6BFA94085F1F4F46
:10E7E00088E090E0A80EB91EF7FEF1CF83E00E940A
:10E7F000301084E690E00E9435198B819C810E9444
:10E80000C576872D0E9430106C960FB6F894DEBF47
:10E810000FBECDBFDF91CF911F910F91FF90EF9071
:10E82000DF90CF90BF90AF909F908F907F90089592
:10E830002FEF3FEFE4E0F5E08FE12083318337965F
:10E84000815087FFFACF0895AC01FC0123E0F695D3
:10E85000E7952A95E1F7E955F54F808199279A01C7
:10E860002770307002C0959587952A95E2F7440F7E
:10E87000551F382F317080FF02C04F5F5F4F20E07F
:10E88000E4E0F5E0808191818417950759F4868151
:10E8900080FF0CC0332319F082E590E0089587E4EF
:10E8A00090E008952F5F3796203260F3332319F0FC
:10E8B00082E790E0089587E690E008950895DF925A
:10E8C000EF92FF920F931F93CF93DF93CDB7DEB7F5
:10E8D00026970FB6F894DEBF0FBECDBF7C01D62EB3
:10E8E000009709F476C0FC01008111816623D9F1FB
:10E8F00061E0C8010E948B208823D1F180914106FC
:10E9000090914206A0914306B0914406F70182839C
:10E910009383A483B583868181608683C80174E074
:10E92000969587957A95E1F7482F98013695279522
:10E930002770307081E090E002C0880F991F2A95FF
:10E94000E2F7982F552700FF06C0FA01E955F54F69
:10E950008081892B06C0FA01E955F54F9095808199
:10E96000892380830DC0C8010E948B20882319F45D
:10E9700080E090E02EC08FEF9FEFF70180839183BE
:10E98000F701868183FF05C0C801969587950E948F
:10E99000CB77802F8F778983000F012F001F110BFA
:10E9A0001195802F8F778A83000F012F001F110B85
:10E9B0001195802F8F778B8380E0D11081E08C833D
:10E9C000AE014F5F5F4F63E28FEF0E94EF6381E024
:10E9D00090E026960FB6F894DEBF0FBECDBFDF9154
:10E9E000CF911F910F91FF90EF90DF9008955F926C
:10E9F0006F927F928F929F92AF92BF92CF92DF924F
:10EA0000EF92FF920F931F93CF93DF930E94812089
:10EA1000882309F4B3C00E942F618C01FC01838517
:10EA20009927AA27BB27BC01CD0122E330E040E0B3
:10EA300050E00E94AA7D3B014C01F8018485992792
:10EA4000AA27BB27BC01CD0124E630E040E050E01E
:10EA50000E94AA7D5B016C0100E010E07801552462
:10EA6000C4E0D5E048815981FFEF4F3F5F0709F4CB
:10EA700072C08E81992780FF3BC082FD11C08A81C0
:10EA80009B81AC81BD81860D971DA81DB91DBC0160
:10EA9000CD010E94ED16882319F08E8184608E834B
:10EAA0008E81992781FF02C082FD0FC08A819B81E0
:10EAB000AC81BD818A0D9B1DAC1DBD1DBC01CD016E
:10EAC0000E94ED16882309F446C0E114F10471F0A8
:10EAD000F70122813381448155818A819B81AC81F8
:10EAE000BD8182179307A407B507A8F57E0133C03F
:10EAF00090E0E4E0F5E0BA01B3E076956795BA9569
:10EB0000E1F7208131818FEF2F3F380771F0241713
:10EB1000350759F0868180FF08C0A3E03695279518
:10EB2000AA95E1F726173707B1F09F5F3796903225
:10EB300040F30115110571F0F80122813381448100
:10EB400055818A819B81AC81BD8182179307A4077F
:10EB5000B50708F48E0153942796FFE1F51508F0E8
:10EB600081CFE114F10419F060E0C70105C001157F
:10EB7000110521F061E0C8010E945F74DF91CF911F
:10EB80001F910F91FF90EF90DF90CF90BF90AF90CB
:10EB90009F908F907F906F905F9008951F93CF9379
:10EBA000DF93EC01162F805F9F4018F080E090E02B
:10EBB00053C020E0E4E0F5E0808191818C179D074F
:10EBC00031F12F5F37962032B8F3112389F41CC03E
:10EBD000C083D1838091410690914206A091430663
:10EBE000B091440682839383A483B58316820FC0B9
:10EBF00020E0E4E0F5E0808191818F5F9F4F41F359
:10EC00002F5F37962032B8F3E0E0F0E002C0309793
:10EC100021F4CF01112301F51DC0112319F48681C0
:10EC200082608683442319F08681886086830E94EF
:10EC30002F61FC01112361F09E0136952795858592
:10EC400096858217930720F4258736870E94B66041
:10EC50000E94F77481E090E0DF91CF911F910895B9
:10EC6000CF93DF93EC018FE0C03FD80718F08FEF10
:10EC70009FEF23C0D695C79583E0CD3FD807C0F45A
:10EC8000D695C795D695C795CE0123E096958795DD
:10EC90002A95E1F78452904F0E9455789927C770C2
:10ECA000D07002C095958795CA95E2F780FF03C0A2
:10ECB00083E090E002C081E090E0DF91CF91089581
:10ECC0001F93CF93DF93039711F41FEF01C010E060
:10ECD000CCEDDFE0A895612FCE010E946E782196E1
:10ECE0008FE0CC3FD807B4F3DF91CF911F91089507
:10ECF000EF92FF920F931F93CF93DF93EC018B0161
:10ED00008FE0C03FD807D0F56330710519F061304E
:10ED10007105A1F5D695C79583E0CD3FD80770F56D
:10ED2000D695C795D695C7957E0153E0F694E7949E
:10ED30005A95E1F7C7018452904F0E945578682F89
:10ED40009E01277030700330110549F481E090E096
:10ED500002C0880F991F2A95E2F7682B09C081E04D
:10ED600090E002C0880F991F2A95E2F780956823EA
:10ED7000A895C7018452904F0E946E78DF91CF9181
:10ED80001F910F91FF90EF9008959F92AF92BF92C5
:10ED9000CF92DF92EF92FF920F931F93CF93DF9367
:10EDA0007C0188EFE81687E0F80608F07DC00E9435
:10EDB0002F615C01FC01E586F6860E94B660CC24DA
:10EDC000DD249924092D1127E016F10608F457C017
:10EDD000C801F3E096958795FA95E1F7482F9801D9
:10EDE0002770307081E090E002C0880F991F2A954B
:10EDF000E2F7982FE801CC0FDD1FE42FFF27E9553C
:10EE0000F54F8081892331F0219604C08AE090E09B
:10EE10000E94351940E061E0CE010E94CE75882342
:10EE2000A9F340E0642FCE010E94CE7560E081E03E
:10EE30000E94E01A0894E11CF11CFF92EF920894E2
:10EE4000E108F1080894C11CD11CDF92CF928CE13B
:10EE50000E941D609F938F9382E08F930E94FA1C03
:10EE600084E690E00E9435198DB79EB707960FB6DD
:10EE7000F8949EBF0FBE8DBF0C5F1F4FA5CFF5014D
:10EE8000838599270E9435199394F3E0F91508F0CA
:10EE900099CF84E690E00E94351902C00E94751057
:10EEA0000E94AB228823D1F3DF91CF911F910F9164
:10EEB000FF90EF90DF90CF90BF90AF909F9008951C
:10EEC000EF92FF920F931F93CF93DF938091E4050E
:10EED000682F77271092E405E7EAFBE08191882309
:10EEE00011F0706805C08CE0E63AF807B9F3B4F3A6
:10EEF00040E050E08091E4099927481759079CF4B5
:10EF0000DC019A01F901E40FF51FEC59F84F8781F4
:10EF100080FF02C0706407C04F5F5F4F275F3F4FA5
:10EF20004A175B077CF340E050E08091E5099927A0
:10EF3000880F991F4817590704F57C01E7E2FAE0AA
:10EF400007EE19E0C7E6DAE09991D8018D918D01BD
:10EF5000981759F48081282F3327892F9927809576
:10EF6000909528233923232B11F0706206C04F5F40
:10EF70005F4F31964E155F053CF3CB01DF91CF918A
:10EF80001F910F91FF90EF9008959091E405982BB9
:10EF90009093E40508959C0187E0283F3807A0F48A
:10EFA000F90183E0F695E7958A95E1F7E955F44F85
:10EFB0002770307081E090E002C0880F991F2A9579
:10EFC000E2F72081282B20830895089528E28030DD
:10EFD000920740F40E94842BFC01892B19F0878151
:10EFE0008160878308950895CF93DF931092E4059D
:10EFF00080E091E0E7EAFBE011920197E9F7C7EEC4
:10F00000D9E0A7E6BAE0E7E2FAE08091E5099927BE
:10F01000880F991F009741F09C018D919191892B48
:10F02000899321503040C9F7E4E6F7E08091E40984
:10F030009927009751F09C0187818E7F878321500B
:10F0400030403A9621153105B9F7DF91CF910895F7
:10F05000FC0188279927E89421912223F1F020329E
:10F06000D9F32930C9F32A30B9F32C30A9F32D3064
:10F0700099F3263789F32B3219F02D3221F4689455
:10F080002191222351F0203344F02A3334F42053C9
:10F090000E949578820F911DF3CF8115910521F083
:10F0A0001EF48095909501960895E199FECF9FBB3F
:10F0B0008EBBE09A99278DB308954115510569F0EB
:10F0C000DC01E199FECF7FBB6EBBE09A6F5F7F4FA3
:10F0D0000DB20D9241505040B1F70895E199FECF25
:10F0E0009FBB8EBB6DBB0FB6F894E29AE19A0FBE40
:10F0F00008954115510589F0DC018FB7E199FECFE4
:10F100007FBB6EBB0D900DBAF894E29AE19A8FBF67
:10F110006F5F7F4F4150504089F70895DC0101C077
:10F120006D9341505040E0F708957AE0979F902DFD
:10F13000879F802D910D112408950F931F93CF93D6
:10F14000DF93CDB7DEB72C970FB6F894DEBF0FBEB6
:10F15000CDBF0B891C89ED89FE893EE03C83098384
:10F160001A834FEF5FE74D835E83AE01495E5F4FC9
:10F17000BF01CE0101960E94657A2F813885020F6A
:10F18000131FD8011C922C960FB6F894DEBF0FBE49
:10F19000CDBFDF91CF911F910F910895FC01019098
:10F1A000061629F00020D9F7882799270895319766
:10F1B0008E2F9F2F0895FB01DC018D910590801902
:10F1C00011F40020D1F7990B0895FB01DC010190A7
:10F1D0000D920020E1F70895FB01DC014150504001
:10F1E00030F08D910190801919F40020B9F7881B37
:10F1F000990B0895FB01DC014150504030F08D9196
:10F200000590801919F40020B9F7881B990B08950F
:10F210002F923F924F925F926F927F929F92AF9206
:10F22000BF92CF92DF92EF92FF920F931F93CF93F3
:10F23000DF93CDB7DEB76E970FB6F894DEBF0FBE83
:10F24000CDBF898B9A8B6B8B7C8B4D8B5E8B3C01FE
:10F250001F8A188EF30191903F01892D99270E94F2
:10F26000247E892BB9F70DE2901609F4FFC01BE24A
:10F27000911609F4F7C02D893E892115310509F44D
:10F28000DAC02031310509F4D6C0ED89FE89EF2BB3
:10F2900041F430E3931609F4C9C04AE050E04D8BC5
:10F2A0005E8B8D899E89AA2797FDA095BA2F898F9D
:10F2B0009A8FAB8FBC8F8F89988D892B09F4B1C041
:10F2C00060E070E080E090E8298D3A8D4B8D5C8D98
:10F2D0000E94557E29873A874B875C876D877E879A
:10F2E0008F87988B58E0DE011196FE0139960190C8
:10F2F0000D925A95E1F7CC24DD247601AA24BB2493
:10F3000029803A804B805C802D813E812D8F3E8FFD
:10F31000092D1127C8010E94187E892BC9F1C80147
:10F320000E941D7E892B09F46BC070ED970E892D0C
:10F3300099276D897E898617970754F5B7FC24C0F5
:10F340002C143D044E045F04F8F0C214D304E4040A
:10F35000F504A9F021E0A22EB12CC701B601298D38
:10F360003A8D4B8D5C8D0E94AA7D6B017C01C90C8E
:10F37000D11CE11CF11CD3019D903D01C9CFAD8C86
:10F38000BE8CA816B90634F73FEFA32EB32EF3CFE9
:10F39000B7FE29C0EF89F88DEF2BE1F0C12CD12CFD
:10F3A000E12C90E8F92E02E210E01093A80C0093F3
:10F3B000A70C8B899C89892B09F460C0AB2839F094
:10F3C000C3010197AB89BC898D939C9357C08989F0
:10F3D0009A89F8CF8FEFC82E8FEFD82E8FEFE82EB7
:10F3E0008FE7F82EE0CFAF89B88DAB2B11F3F094F7
:10F3F000E094D094C094C11CD11CE11CF11CD9CF65
:10F40000C8010E94FE7D892B19F2C8010E94FC7D73
:10F41000892B21F0802F8753982E89CF802F8755F5
:10F42000FBCF6FEF7FEF8FEF9FE74ECF08E010E04D
:10F430000D8B1E8B36CF40E3941609F026CFF301D7
:10F440008081883719F0883509F01FCFD3011196D4
:10F450009C9082E090E0680E791E60E170E06D8B18
:10F460007E8B13CFD3019D903D0105CF21E030E08D
:10F470002F8B388FF30191903F01FDCEC701B6016C
:10F480006E960FB6F894DEBF0FBECDBFDF91CF9161
:10F490001F910F91FF90EF90DF90CF90BF90AF90B2
:10F4A0009F907F906F905F904F903F902F90089526
:10F4B000DC015C91552341F05F7D51341CF05B35DC
:10F4C0000CF45C931196F5CF08952F923F924F92D2
:10F4D0005F926F927F928F929F92AF92BF92CF92E4
:10F4E000DF92EF92FF920F931F93CF93DF93CDB7ED
:10F4F000DEB762970FB6F894DEBF0FBECDBFAA2469
:10F50000BB2465014C016D877E874F87588B44244F
:10F510005524FC0146825782838181FD5BC28FEFB7
:10F520009FEF6FC240FE44C2862D80538A30E0F4C4
:10F53000F0E36F1641F42A89222329F4772019F485
:10F5400080E091E08BC08AE09A89989F902D1124E9
:10F55000892F860D80538A8B882314F4EFE7EA8B7A
:10F5600043FC38C27A8836C243FE05C0FA89FF23BD
:10F5700011F421E02A8B862D992787FD90958836F6
:10F58000910554F5853691050CF06BC088359105D1
:10F5900009F4D3C089359105B4F48B32910509F48F
:10F5A00042C08C32910544F48032910509F43FC089
:10F5B000839709F442C0F2C18D329105D9F18E973B
:10F5C00009F440C0EBC18336910509F454C0843678
:10F5D000910509F478C0E2C18037910509F4A5C00E
:10F5E0008137910584F48C369105B1F18D36910502
:10F5F0002CF48936910509F466C0D0C18F36910587
:10F6000009F490C0CBC18537910509F498C08637BD
:10F61000910524F483379105B9F1C0C1883791056C
:10F6200009F48BC0BBC180E190E0482A592AE0E28E
:10F63000F0E005C080E890E011C0E0E4F0E04E2A80
:10F640005F2AC8C188E090E0482A592AEFEFFEEF10
:10F650004E225F221A8ABEC184E090E0482A592ACD
:10F66000B9C10F2EFFE3AF2EF02D7A940F2EF3E6E3
:10F670006F2EF02D3AC1EF85F889CF0102968F8762
:10F68000988BA0807A9431C1EF85F889CF010296DA
:10F690008F87988BA080B18043FE0BC0EA898E2FA4
:10F6A000992787FD9095BC01C5010E949F7D898B9C
:10F6B00007C0F50101900020E9F73197EA19E98BBD
:10F6C000F9897F1A12C142FE0BC0EF85F889CF017C
:10F6D00004968F87988B20813181428153810DC0A0
:10F6E000EF85F889CF0102968F87988B8081918171
:10F6F0009C01442737FD4095542F59016A01552339
:10F7000064F4E2E0F0E04E2A5F2AD094C094B09412
:10F71000A094A11CB11CC11CD11C8FEB9FEF4822EF
:10F7200059222BC098E0998B0AC0E0E4F0E04E2A01
:10F730005F2A0F2EF8E76F2EF02DF0E1F98B42FED5
:10F740000BC0EF85F889CF0104968F87988B2081B5
:10F750003181428153810BC0EF85F889CF01029638
:10F760008F87988B808191819C014427552759016F
:10F770006A01EFECFFEF4E225F221E010894211C6C
:10F78000311CF989EF2EFF2400271127C601B5018E
:10F79000A80197010E94337EDC01CB01F101808337
:10F7A0008A301CF0860D815203C0F1018081805D9A
:10F7B000F10181931F01C601B501A80197010E94C3
:10F7C000337E59016A012115310541055105F1F6D4
:10F7D000CE010196A22CA81AC20182739070892BC7
:10F7E00009F07A9446FE0FC0872D992787FD9095E2
:10F7F000F989F03131F40F2EFEEF7F2EF02D780EC7
:10F8000002C0782E7A9443FE12C08A89282F3327AB
:10F8100027FD30958A2D9927821793072CF0E7EF63
:10F82000FFEF4E225F2203C0FA89FA19FA8B43FEDA
:10F8300003C02A89721A01C07A18C20180789170B7
:10F84000892B69F4872D7A9418164CF4B40180E260
:10F8500090E00E946C7D872D7A941816BCF341FECF
:10F8600004C0B4018DE290E00BC044FE04C0B401BA
:10F870008BE290E005C045FE05C0B40180E290E057
:10F880000E946C7D46FE0FC0B40180E390E00E94B0
:10F890006C7D8989803139F4862D992787FD909573
:10F8A000B4010E946C7D50FE0DC0872D7A9418160D
:10F8B0004CF4B40180E390E00E946C7D872D7A9433
:10F8C0001816BCF343FE11C08A89982F91509A8B69
:10F8D00018165CF4B40180E390E00E946C7D8A8984
:10F8E000E82FE150EA8B1816ACF3842D807869F488
:10F8F000872D7A9418164CF4B40180E290E00E94AF
:10F900006C7D872D7A941816BCF3F3E66F1641F4DC
:10F910008A2D992787FD9095B4010E946C7D2DC09A
:10F9200023E76216B1F489898150898B8F3F29F1D1
:10F93000F5018081992787FD90950894A11CB11C41
:10F94000B4010E946C7D99899150998B9F3F81F7FA
:10F9500014C0CE0101962816390679F08E010F5F8A
:10F960001F4FF10182911F01992787FD9095B401E6
:10F970000E946C7D20163106A1F7842D8078A9F0B5
:10F98000872D7A9418168CF4B40180E290E00E94DE
:10F990006C7D872D7A941816BCF307C0862D9927A5
:10F9A00087FD9095B4010E946C7D4424552412C0BB
:10F9B000F5E26F1641F44424552443941A8A7A8858
:10F9C0002AE0298B07C0862D992787FD9095B401E1
:10F9D0000E946C7DF401838183FF08C0ED85FE8564
:10F9E000CF0101968D879E87649005C0ED85FE85C9
:10F9F0006190ED87FE87662009F094CDF401868141
:10FA0000978162960FB6F894DEBF0FBECDBFDF912F
:10FA1000CF911F910F91FF90EF90DF90CF90BF900B
:10FA2000AF909F908F907F906F905F904F903F909E
:10FA30002F9008950F931F93CF93DF93CDB7DEB729
:10FA40002C970FB6F894DEBF0FBECDBF8C0136E009
:10FA50003C8389839A832FEF3FE72D833E83CE013A
:10FA600001960E94657AAF81B885A00FB11F1C92E4
:10FA70002C960FB6F894DEBF0FBECDBFDF91CF91AD
:10FA80001F910F9108950F931F93CF93DF93CDB7DD
:10FA9000DEB72C970FB6F894DEBF0FBECDBF8C013A
:10FAA0003EE03C8389839A832FEF3FE72D833E839B
:10FAB000CE0101960E94657AAF81B885A00FB11F73
:10FAC0001C922C960FB6F894DEBF0FBECDBFDF910F
:10FAD000CF911F910F9108950F931F93CF93DF93B1
:10FAE0008C01EB018B81992781FF22C082FF14C01A
:10FAF0002E813F814C815D81241735073CF4A8811C
:10FB0000B9810D93A883B9832E813F812F5F3F4F29
:10FB10002E833F83C8010EC0E885F985802F0995A3
:10FB2000892B31F4EE81FF813196EE83FF83F2CF92
:10FB30008FEF9FEFDF91CF911F910F910895FC01FF
:10FB40006150704001900110D8F7809590958E0F0C
:10FB50009F1F0895629FD001739FF001829FE00D67
:10FB6000F11D649FE00DF11D929FF00D839FF00D3C
:10FB7000749FF00D659FF00D9927729FB00DE11DE8
:10FB8000F91F639FB00DE11DF91FBD01CF011124C5
:10FB90000895991B79E004C0991F961708F0961BE9
:10FBA000881F7A95C9F78095089597FB092E072637
:10FBB0000AD077FD04D00CD006D000201AF470953E
:10FBC00061957F4F0895F6F7909581959F4F089521
:10FBD000AA1BBB1B51E107C0AA1FBB1FA617B70773
:10FBE00010F0A61BB70B881F991F5A95A9F780958F
:10FBF0009095BC01CD01089585FD17C080629923C1
:10FC0000A1F4813694F08B3784F40895992369F434
:10FC1000803269F0893059F08B3039F408958F9330
:10FC2000EDDF8F9109F08062089599278827089564
:10FC30009923D9F78095807808959923B1F7803377
:10FC4000A4F38A3394F70895992379F7803279F3EE
:10FC50008A3069F38C3059F38D3049F3893039F3A8
:10FC60008B3019F70895A1E21A2EAA1BBB1BFD01C8
:10FC70000DC0AA1FBB1FEE1FFF1FA217B307E4078B
:10FC8000F50720F0A21BB30BE40BF50B661F771FE3
:10FC9000881F991F1A9469F76095709580959095C3
:10FCA0009B01AC01BD01CF01089597FB092E0526EC
:10FCB0000ED057FD04D0D7DF0AD0001C38F4509581
:10FCC0004095309521953F4F4F4F5F4F0895F6F780
:10FCD00090958095709561957F4F8F4F9F4F0895B8
:10FCE0008005453781054A3784034F3785037E37C2
:10FCF0008605AF378804F937890420388C034B38E0
:10FD00008D036438900382389403F13895022A39C0
:10FD100098024639990169399C026E399D039139DF
:10FD2000A001B839A201153AA4032E3AA501523A0E
:10FD3000A6015B3AA701613AC401673AC602E14BEA
:10FD4000C703D74BC8016A3AC901A73ACA01E93AC1
:10FD5000CB01823B000000002C20000000010000CD
:10FD6000FF00020000FF0000B559FF00030000FF84
:10FD70000000C85AFF0000A352FF0000374FFF00E9
:10FD8000007D4FFF01003351FF01008F4FFF010045
:10FD90005C50FF01000B52FF01005C52FF0200BBF0
:10FDA00055FF02002A55FF02003F56FF02009E56F3
:10FDB000FF0200CE55FF0200E155FF0200DB54FFB9
:10FDC00003040000FF0300645A17030500001E032C
:10FDD000007359FF030600001E0300AB57FF03002A
:10FDE000B057FF0400085CFF0400625CFF0500B52B
:10FDF00057FF0500AC5BFF0600CE57FF06001F58FB
:10FE0000FF06006B59FF06006F59FF2534642D254E
:0AFE100034643A2000253464000039
:00000001FF
